:1000000049C6000078C6000076C6000074C600002D
:1000100072C6000070C600006EC600006CC600000C
:100020006AC6000068C6000066C6000064C600001C
:1000300062C600000C941F7B5EC600005CC6000018
:100040005AC600000C94CA7856C6000054C6000078
:1000500052C6000050C600004EC600000C94F9774E
:100060004AC600000C940D750C94E37444C600005D
:1000700042C6000040C600003EC600003CC600006C
:100080000C949D7838C6000036C6000034C60000C7
:1000900032C6000030C600002EC600000C94CB7B98
:1000A0002AC6000028C600000C94707824C6000000
:1000B00022C6000020C600001EC600000C94437833
:1000C0001AC6000018C6000016C6000014C60000BC
:1000D00012C6000010C600000C94AD740C9483741A
:1000E0000AC600004E414E494E495459494E46CD2C
:1000F000CCCC3D0AD7233C17B7D13877CC2B3295DF
:1001000095E6241FB14F0A000020410000C84200BC
:10011000401C4620BCBE4CCA1B0E5AAEC59D740086
:10012000407A10F35A00A0724E18090010A5D4E8C6
:100130000000E87648170000E40B54020000CA9A59
:100140003B000000E1F505000080969800000040AB
:10015000420F000000A086010000001027000000F0
:1001600000E803000000006400000000000A000036
:100170000000000100000000002C76D888DC674FEA
:100180000823DFC1DFAE59E1B1B796E5E3E453C61A
:100190003AE651997696E8E6C28426EB898C9B6212
:1001A000ED407C6FFCEFBC9C9F40F2BAA56FA5F4BC
:1001B00090055A2AF75C936B6CF9676DC11BFCE0E4
:1001C000E40D47FEF520E6B500D0ED902E03009437
:1001D0003577050080841E080000204E0A000000CC
:1001E000C80C333333330F986E12831141EF8D21D6
:1001F00014893BE65516CFFEE6DB18D1844B381B3D
:10020000F77C1D901DA4BBE424203284725E228101
:1002100000C9F124ECA1E53D27485454502F312E5C
:10022000302034303020426164205265717565732E
:10023000740D0A5365727665723A2057656264756B
:10024000696E6F2F312E370D0A436F6E74656E74B1
:100250002D547970653A20746578742F68746D6CCC
:100260000D0A0D0A3C68313E45504943204641493C
:100270004C3C2F68313E00485454502F312E3020D2
:10028000323030204F4B0D0A5365727665723A203A
:100290005765626475696E6F2F312E370D0A4163A1
:1002A000636573732D436F6E74726F6C2D416C6C4C
:1002B0006F772D4F726967696E3A202A0D0A436F76
:1002C0006E74656E742D547970653A2000436F6EBC
:1002D0006E656374696F6E3A20636C6F73650D0AA7
:1002E000436F6E74656E742D547970653A20617039
:1002F000706C69636174696F6E2F782D7777772DD5
:10030000666F726D2D75726C656E636F64656400E7
:10031000506F7374206661696C65640055706C6F12
:100320006164204661696C65643A2000234E6F2049
:1003300073656E736F7220666F722074656D7020C6
:10034000262068756D696469747921004E6F2053A9
:10035000656E736F72210020666F722074656D7018
:1003600020262068756D69646974792100235365BE
:100370006E736F72204572726F72200053656E73D8
:100380006F72204572726F7221002357726F6E6711
:100390002073656E736F7220666F722074656D7066
:1003A00020262068756D6964697479210057726F21
:1003B0006E672053656E736F7221004320483D00C5
:1003C000543D0020202020202020202020202020FC
:1003D000202020002020202020202020202020203D
:1003E000202020002020202020202020202020202D
:1003F00020202000495020616464726573733A20A4
:1004000000416E676C654000496E76616C696420DE
:10041000534D2073746570732070657220616E6730
:100420006C653D00534D2073746570732070657268
:1004300020616E676C653D003C703E4C616D7020C4
:10044000616E64204F7468657220537461747573B3
:10045000EFBC9A3C2F703E003C703E54696D653A8B
:1004600020003C2F68333E0A003C62723E4254201A
:100470006E616D653D003C62723E506174683D0086
:100480003C68333E53797374656D3A2056657273D8
:10049000696F6E3D003C21646F63747970652068FC
:1004A000746D6C3E3C68746D6C3E3C686561643E86
:1004B0003C6D65746120636861727365743D22757B
:1004C00074662D38223E3C7469746C653E4F6E6CC8
:1004D000696E65206578706572696D656E7420203F
:1004E000506F6C6172697A6174696F6E20656666BF
:1004F00065637473206F66206C696768743C2F7441
:1005000069746C653E3C2F686561643E3C626F6453
:10051000793E3C68313E4F6E6C696E65206578703F
:100520006572696D656E742020506F6C6172697AB6
:100530006174696F6E2065666665637473206F66AB
:10054000206C696768743C2F68313E003C68343E1B
:10055000436F70797269676874284329323032308A
:1005600020456455484B204861732043656E747282
:10057000652E3C2F68343E3C2F626F64793E3C2FE1
:1005800068746D6C3E003C68313E43616E6E6F7402
:10059000206765742073656E736F72207265616485
:1005A000696E6773213C2F68313E00506172616D46
:1005B000657465727320726573657420646F6E650F
:1005C0002100736573757365722F736D6C6967684D
:1005D00074706F2F73312F00616E676C65206469D2
:1005E00072656374696F6E3A200043757272656E4E
:1005F0007420534D206973202300534D3A54616297
:100600006C652073746570732070657220616E670D
:100610006C653D00534D3A506F6C61726F69642098
:1006200073746570732070657220616E676C653DD0
:1006300000234448543D00236E65743D424C450000
:10064000236E65743D5769466900236E65743D42AB
:1006500054002366747020757365726E616D653A1F
:10066000003A0023486F73742073657276657220B8
:10067000495020616E6420506F72743A00235265B5
:100680006C617920646576696365733A002352650D
:100690006C617920737461747573206C6162656C30
:1006A000733A20002352656C61792073746174651C
:1006B000733A002352656C61792070696E733A0059
:1006C000234E6F2E206F662072656C6179733D003A
:1006D00046696E64696E6720576946692049500013
:1006E0004E45543D426C7565746F6F7468204C457F
:1006F000004E45543D426C7565746F6F7468004ED2
:1007000045543D57694669005344206F70656E201B
:100710006661696C004E6577206461746120636F67
:100720006C6C656374696F6E207374617274656458
:100730000043757272656E742073657474696E67B8
:10074000733A0053797374656D2072657365742014
:100750006174200023445320546865726D6F6D6589
:100760007465722063616C6962726174656420668D
:100770006F72202300496E76616C696420616E6738
:100780006C6520666F722000207374657073207032
:10079000657220616E676C653D00207374657073CF
:1007A0002070657220616E676C653D005461626CFB
:1007B0006520536574203000235475726E74616235
:1007C0006C6520536574203000506F6C6172697ADB
:1007D00065722053657420300023506F6C6172691C
:1007E0007A6572205365742030005461626C652014
:1007F000536574203000235475726E7461626C65A9
:1008000020536574203000506F6C6172697A657294
:100810002053657420300023506F6C6172697A65D3
:100820007220536574203000576946692049503A58
:10083000004C6F67676572204E616D653A2000520B
:1008400065626F6F74696E672E2E2E005365727627
:10085000657220506F7274207570646174656400F5
:1008600053504F52543D0049502075706461746577
:1008700064005349503D0074696D6520696E74656C
:100880007276616C3D00237765627365727665727E
:1008900020626567696E73005461626C6520536500
:1008A00074203000235475726E7461626C6520533D
:1008B0006574203000506F6C6172697A65722053E4
:1008C000657420300023506F6C6172697A65722004
:1008D00053657420300053797374656D20726573AD
:1008E00074617274656421002053797374656D209E
:1008F000726573746172746564210023436F6D6D5A
:10090000616E64400054657374204C616D70732F88
:1009100046616E73004448435020537563636573AA
:10092000730044484350204641494C454400776594
:1009300062736572766572202E2E2E006572726F5C
:1009400072206F70656E696E672066696C653A200B
:10095000004C616D70204F74686572002354696D9E
:100960006520202020202044617465202020202044
:100970005365636F6E647320506F6C61726F69644E
:10098000205461626C652054286F43292048282533
:1009900029202000646F6E652100696E69742E2025
:1009A000646F6E652E00534420696E69742E206654
:1009B00061696C65642100696E69742E20666169E5
:1009C0006C6564210057656C636F6D6520746F20E2
:1009D000456455484B00496E697469616C697A6970
:1009E0006E6720534420636172642E2E2E00757052
:1009F0006C6F616420627920465450206661696C96
:100A00006564210075706C6F6164206279204654C2
:100A100050204F4B21007C3C3E5E2B3D3F2F5B5DC9
:100A20003B2C2A225C0000002100240027002A0021
:100A30002D003000330001010000040107010A010C
:100A400000002200250028002B002E003100340079
:100A500002010000050108010B0100002000230035
:100A6000260029002C002F003200000100000301A5
:100A70000601090105050505070508080808020221
:100A800002020A0A08080404040401010101010128
:100A900001010303030303030303040707070C0C0B
:100AA0000C0C0C0C0C0C02020202060606060606D2
:100AB00006060B0B0B0B0B0B0B0B01021020200877
:100AC00008102040102040800201020108040201A9
:100AD0000102040810204080804020100804020118
:100AE0008004020180402010080402010804020171
:100AF00001020408102040800102040810204080F8
:100B000000000A0B02090C0D0E0807030401000087
:100B100000000000000000000000000000000000D5
:100B20000000000000000000000000001211100092
:100B300000000000000000000000000000000000B5
:100B40000000000000000000010001001010020081
:100B500001000100B00000001600000028000000A5
:100B60001000000020000000010001000000000053
:100B70000000000000000000000000000000000075
:100B80000000000000000000FF000000FFFF000068
:100B9000FFFF0000FFFF0000CFBF0000C7BF000045
:100BA000C3BF0000C1BF0000C0BF000000000000C4
:100BB000C0BF0000C1BF0000C3BF0000C7BF00002E
:100BC000CFBF0000FFFF0000FFFF0000000000009B
:100BD0000000000000000000000000000000000015
:100BE0000000000000000000000000000000000005
:100BF00000000000000000000000000000000000F5
:100C00000000000000000000000000005573657245
:100C10002D6167656E743A202A0D0A446973616C10
:100C20006C6F773A202F0D0A004E6574776F726BE8
:100C3000206D61696E7461696E6564206174200065
:100C4000417070656E64206D6561732E200053697C
:100C50006E676C65206D6561732E2000536176654B
:100C6000206D65617375726520746F3A00202020D5
:100C70002020202020202020202020202000202094
:100C800020202020202020202020202020200000A4
:100C90000B91B39011241FBECFEFD1E2DEBFCDBFC9
:100CA00000E00CBF1AE0A0E0B2E0E2EFF4E501E002
:100CB0000BBF02C007900D92A034B107D9F725E110
:100CC000A0E4BAE001C01D92A83DB207E1F716E02A
:100CD000C9E4D6E000E006C021970109802FFE019B
:100CE0000E94F0A4C834D10780E00807A9F70E9449
:100CF00085940C9468AA84C9CF93DF93EC01898D05
:100D00009A8D892B41F0E881F9810284F385E02DE9
:100D1000CE011995F4CFDF91CF910895CF93DF9352
:100D20001F92CDB7DEB76983DC01ED91FC910280A3
:100D3000F381E02D41E050E0BE016F5F7F4F1995D8
:100D40000F90DF91CF910895FC01818D928D0895D0
:100D5000FC0184899589089521E034E0FC01318308
:100D60002083FB014089518962897389FC01428398
:100D70005383648375830895DC01ED91FC91048CA9
:100D8000F58DE02D1994CF93DF931F92CDB7DEB789
:100D90006983DC01ED91FC910280F381E02D41E05B
:100DA00050E0BE016F5F7F4F19950F90DF91CF919B
:100DB0000895FC019485FB018485981303C081E0AC
:100DC000943009F480E0089521E0FC0184858430AA
:100DD00009F420E0822F08950895CF93DF931F92A6
:100DE000CDB7DEB76983DC01ED91FC910280F38120
:100DF000E02D41E050E0BE016F5F7F4F19950F90ED
:100E0000DF91CF910895DC01ED91FC91068CF78D77
:100E1000E02D199591E089270895862F089581E0A6
:100E2000862708950A96D9CF90E080E0089590E053
:100E3000982F882744E050E0845F9B4F0C94758D79
:100E4000DF92EF92FF920F931F93CF93DF93D82EF1
:100E50000CED1BE0E801EE24E394F12C2296809146
:100E6000A8029091A9028E159F059CF061E08881EF
:100E70000E9459766091D70B88810E94437564EF78
:100E800071E080E090E00E948A768FEFE81AF80A1D
:100E9000E5CFDD2009F45EC0CCEDDBE0EE24E39489
:100EA000F12C22968091A8029091A902E816F906E9
:100EB0002CF56091D90B88810E94437568EE73E030
:100EC00080E090E00E948A76AFEFEA1AFA0A609119
:100ED000D90B8A810E94437568EE73E080E090E050
:100EE0000E948A766091D70B88810E94437568EED4
:100EF00073E080E090E00E948A76D3CF68EE73E0E2
:100F000080E090E00E948A7693E4E92E92E0F92E48
:100F1000C1E0D0E0B2E0EB0EF11C0E5F1F4F8091FC
:100F2000A8029091A9028C179D07A4F0D701ED911A
:100F3000FC91EE0FFF1FE952F44F6081F8018081B0
:100F40000E94437568EC70E080E090E00E948A7631
:100F50002196E0CFDF91CF911F910F91FF90EF90FD
:100F6000DF9008959F92AF92BF92CF92DF92EF925F
:100F7000FF920F931F93CF93DF935C017B018B0153
:100F8000D0E0C0E0F80191908F016501CC0EDD1E2C
:100F9000C6010E9449A3981621F0692DC6010E943E
:100FA00051A32196CA32F1E0DF0761F7C701DF9153
:100FB000CF911F910F91FF90EF90DF90CF90BF9056
:100FC000AF909F90089581E08093DD028091DE02D2
:100FD000882341F088E08093E31160E088ED91E19F
:100FE0000C94F7780895CF93DF93EC01FB012481F3
:100FF00035810E940673CE01DF91CF9108958091D3
:10100000DE028823F9F08091DD028823D9F081E0A7
:101010000E9436798BE39FE10197F1F760E080E071
:101020000E94457964EE73E088ED91E10E9453746B
:1010300061E080E00E94457964ED73E088ED91E124
:101040000C94537408958F929F92AF92BF92CF9257
:10105000DF92EF92FF920F931F93CF93DF938C0158
:10106000862F0B30110509F09FC0909161119923D3
:1010700009F0F89462E10E94BD76EC018091611163
:10108000882309F07894209701F180E090ECA9E79B
:10109000B4EC8093541190935511A0935611B093D2
:1010A00057118093581190935911A0935A11B093EE
:1010B0005B11CE3F8FEFD80709F4A9C0CF3FDC0703
:1010C00009F462C0CCEFDFEF30C1C0915C11E09059
:1010D0005D116E2D70E090E080E00E9436A22DEC54
:1010E0003CEC4CEC5DE30E9495A24B015C016C2F43
:1010F00070E090E080E00E9436A29B01AC01C50147
:10110000B4010E94CCA36093541170935511809345
:10111000561190935711D0915E11F0905F116D2F81
:101120006F7770E090E080E00E9436A24B015C0196
:101130006F2D70E090E080E00E9436A22DEC3CEC38
:101140004CEC5DE30E9495A29B01AC01C501B4018A
:101150000E94CCA3D7FD26C06093581170935911FB
:1011600080935A1190935B11CE0DCD0FCF0D81E07E
:1011700090E020916011C21302C090E080E0892BC2
:1011800009F493C0CFEFDFEFCE01DF91CF911F9134
:101190000F91FF90EF90DF90CF90BF90AF909F9016
:1011A0008F9008959058D8CFCFEFDFEF063111051B
:1011B00009F0BBC090916111992309F0F89461E0A6
:1011C0000E94BD76EC0180916111882309F078942A
:1011D000209701F180E090ECA9E7B4EC80935411E2
:1011E00090935511A0935611B093571180935811B5
:1011F00090935911A0935A11B0935B11CF3FDC0724
:1012000019F2209709F451C0229609F05BCFCEEF76
:10121000DFEF8BC0C0915D11D0915C1160915C11CA
:1012200070915D1176276727762790E080E00E9415
:1012300034A22DEC3CEC4CEC5DE30E9495A2609353
:101240005411709355118093561190935711E0905B
:101250005F11F0905E116F2D6F77762F6E2D90E0FD
:1012600080E00E9434A22DEC3CEC4CEC5DE30E944B
:1012700095A2F7FC18C06093581170935911809390
:101280005A1190935B118C2F8D0F8E0D8F0DC1E035
:10129000D0E090916011891302C0D0E0C0E0D195F8
:1012A000C195D109ABCF9058E6CFC0905411D090E2
:1012B0005511E0905611F090571120E030E048ECC5
:1012C00052E4C701B6010E94C9A4D0E0C0E01816DC
:1012D00014F4CBEFDFEF20E030E0A901C701B60145
:1012E0000E9430A287FF02C0CAEFDFEFC090581102
:1012F000D0905911E0905A11F0905B1120E030E04D
:1013000048EC52ECC701B6010E9430A287FF02C030
:10131000C9EFDFEF20E030E040EF52E4C701B60153
:101320000E94C9A418160CF405C10C30110509F06F
:101330002BCF81E08093B50C8CE58093B70C109295
:10134000B60C1092B80C60E083EF9DE00E940B6D2C
:1013500081E00E94256E8091B40C8111FCCF81E068
:101360008093B40C8093B30C9FEF9093B20C1092C7
:10137000B10C94E09093B00C80938F0C80918F0C03
:10138000886B80938F0C80918E0C813009F0D5C0D2
:1013900010928E0C80918F0C8093BB008091BC00CA
:1013A00083FDF8CF85EC8093BC008091B40C813034
:1013B000E1F38091B10C95E0853010F49091B10C7F
:1013C000A0E9BCE0E3E2FCE080E08913B8C0109241
:1013D000740C8093730C082F10E0CEEFDFEF88239E
:1013E00009F4D2CECDEFDFEF053011050CF4CCCEF1
:1013F000C0E0DBE083EF9DE00E94C56C888721960A
:10140000CE0180509B4080179107A4F3C091080B38
:101410000091090B602F70E090E080E00E9436A2FE
:101420002DEC3CEC4CEC5DE30E9495A26B017C0141
:101430006C2F70E090E080E00E9436A29B01AC012E
:10144000C701B6010E94CCA36B017C01C092000BC6
:10145000D092010BE092020BF092030BD0910A0B99
:1014600010910B0B6D2F6F7770E090E080E00E9481
:1014700036A24B015C01612F70E090E080E00E9499
:1014800036A22DEC3CEC4CEC5DE30E9495A29B0156
:10149000AC01C501B4010E94CCA3D7FD54C0609338
:1014A000040B7093050B8093060B9093070BC00FF2
:1014B000CD0FC10F80910C0BC81364CE20E030E03B
:1014C00048EC52E4C701B6010E94C9A4D0E0C0E0D4
:1014D000181614F4CBEFDFEF20E030E040EA50E4E0
:1014E000C701B6010E9430A287FF02C0CAEFDFEF3A
:1014F000C090040BD090050BE090060BF090070B0A
:1015000020E030E040EF51ECC701B6010E9430A26C
:1015100087FF02C0C9EFDFEF20E030E040EF52E488
:10152000C701B6010E94C9A418160CF02DCEC8EF51
:10153000DFEF2ACEC8EFDFEFF8CE85EE34CF2D9166
:1015400021938F5F42CF9058AACF2C9A08952C9860
:1015500008958EBD00000DB407FEFDCF8EB5089531
:101560009B0190E00496982F8827642F820F931F89
:101570000C94028ECF93DF93C82FD62F472F60E1B4
:1015800070E0EEDF4D2F61E170E08C2FDF91CF91A5
:10159000E7CFCF93DF93C82FD0E02496DC2FCC2762
:1015A000C60FD71FD4DF8FE0D4DF8D2FD2DF8C2F73
:1015B000D0DF80E0CEDFC82FC8DF8C2FDF91CF9146
:1015C00008951F93CF93DF93182F66E270E0E1DF59
:1015D000C82F67E270E0812FDCDF9C2FDF91CF9175
:1015E0001F9108951F93CF93DF93182F60E270E04F
:1015F000D0DFC82F61E270E0812FCBDF9C2FDF911D
:10160000CF911F91089544E050E0BC018FE090E03D
:101610000C94758D08958CBD9DBD0895EF92FF9239
:101620000F931F93CF93C82F7B0180E590E0F3DFEA
:1016300068E270E08C2FADDF082F69E270E08C2F3C
:10164000A8DF282F302FB90121E030E0A7018C2F2F
:101650000E94F96F81E090E0CF911F910F91FF9070
:10166000EF900895CF93DF931F92CDB7DEB7FC01C3
:10167000218D328D8FEF9FEF232B39F0BE016F5FED
:101680007F4F808DCBDF898190E00F90DF91CF91EC
:1016900008950F931F93CF93DF931F92CDB7DEB7BB
:1016A0008C01DC01ED91FC910084F185E02D199510
:1016B000892B71F0BE016F5F7F4FF8018485AEDF2B
:1016C000898190E00F90DF91CF911F910F91089544
:1016D0008FEF9FEFF7CFFF920F931F93CF93DF937F
:1016E000F82E80E590E097DF10E000E08F2D69DFB5
:1016F000EC01892B19F08F2D64DF8C01C017D10705
:10170000A9F7CE01DF91CF911F910F91FF9008951E
:10171000FC018485843009F0DECF90E080E00895FC
:10172000AF92BF92CF92DF92EF92FF921F93CF932F
:10173000DF93182F6B017A0180E590E06CDFB12C0C
:10174000A12C812F3EDFEC01892B19F0812F39DF8D
:101750005C01CA15DB05A9F72097E1F463E070E0AE
:10176000812F17DF843159F0882349F0C1E0D0E0A0
:101770008C3111F4D0E0C0E0D195C195D109CE01F2
:10178000DF91CF911F91FF90EF90DF90CF90BF90AE
:10179000AF900895EC16FD060CF4E7011C161D062B
:1017A00074F768E270E0812FF4DEE82E69E270E001
:1017B000812FEFDE282F3E2D79019E01A601B70172
:1017C000812F0E94F96FEC0EFD1E4F2D68E270E034
:1017D000812FC6DE4E2D69E270E0812FC1DE60E40C
:1017E00070E0812F0E94C66ECACFCF93DF93FC01B9
:1017F000218D328D2115310529F48FEF9FEFDF9177
:10180000CF910895EC01808D4217530708F0A9018C
:1018100087DF181619068CF7298D3A8D281B390B8E
:101820003A8F298FECCF0F931F93CF93DF931F92A3
:10183000CDB7DEB7FC01218D328D232B41F48FEF24
:101840009FEF0F90DF91CF911F910F9108958C0121
:1018500041E050E0BE016F5F7F4FFC01808D60DF93
:101860001816190664F7F801818D928D0197928FF1
:10187000818F898190E0E5CF0F931F93CF93DF9302
:1018800000D000D01F921F92CDB7DEB78C01DC01D3
:10189000ED91FC910680F781E02D1995F801808D7E
:1018A0001ADF18161906ACF548E050E0BE016F5F6C
:1018B0007F4FD80158968C9133DF18161906F4F42F
:1018C000D801509684E0FE01319601900D928A95E0
:1018D000E1F78D8190E0982F88272E81820F911D4E
:1018E000F801958B848B8F81282F30E0322F2227AF
:1018F0008885820F932F911D928F818F28960FB626
:10190000F894DEBF0FBECDBFDF91CF911F910F9135
:10191000089590E080E0F2CFFC01848501CFCF9361
:10192000DF931F92CDB7DEB741E050E0BE016F5F9D
:101930007F4FFC018485F4DE1816190634F4898182
:1019400090E00F90DF91CF9108958FEF9FEFF9CF47
:10195000CF93C82F80E590E05EDE60E170E08C2FD1
:101960000E94C66E4FEF62E070E08C2FCF91F8CDF1
:10197000FF920F931F93CF93DF93C82FD62F8A0127
:10198000F22EE6DF80E590E046DE4D2F4F2970E035
:1019900060E08C2FE5DD01151105B1F0412F64E009
:1019A00070E08C2FDDDD402F65E070E08C2FD8DDFE
:1019B00061E070E08C2F0E94C66E81E0DF91CF91D4
:1019C0001F910F91FF9008950091210C1091220C0E
:1019D0000F5F1F4F1093220C0093210CDFCFBF929B
:1019E000CF92DF92EF92FF920F931F93CF93DF93EB
:1019F00000D000D0CDB7DEB7FC01208D243009F037
:101A000059C06A017B018C01B12C63E070E08B2D21
:101A1000C0DD811147C0F801B08EF801808D84309F
:101A200009F448C096E0E9EEF2E0DE01119601907B
:101A30000D929A95E1F7F70193819F779C839481AA
:101A40009D8395819E83B7016E5F7F4FF0D9B6016C
:101A5000F801808D8FDDF801808D90E0982F882728
:101A600046E050E0BE016F5F7F4F8A5F9B4F0E9450
:101A7000758DF801128E118E20E8A60162E0808D2E
:101A800077DF81E026960FB6F894DEBF0FBECDBF9C
:101A9000DF91CF911F910F91FF90EF90DF90CF904A
:101AA000BF900895883109F4B6CFB394F4E0BF1223
:101AB000ACCFB3CF80E0E6CFCF93DF93EC01888D3E
:101AC000843059F045DFE88DF0E0EE0FFF1FE05B5A
:101AD000F34F1182108284E0888FDF91CF910895B7
:101AE000CF93C82F80E590E096DD63E070E08C2F07
:101AF000CF914FCDEF92FF921F93CF93DF93FC01D5
:101B0000208D243039F080E0DF91CF911F91FF903C
:101B1000EF9008957B01EC0110E0812FE1DF81114E
:101B20000EC0188F888D843071F3FD86EC861A8E76
:101B3000198E20E0A70162E01BDF81E0E5CF88314C
:101B400081F31F5F143049F7EDCFFC0184858430A9
:101B500009F0C6CF80E00895CF93DF93FC01248580
:101B60002430D1F0EC01F1DF843189F0882379F061
:101B7000883169F021E08C3159F4E881F9810084E1
:101B8000F185E02DCE01199521E0892B09F420E0A3
:101B9000822FDF91CF91089580E0FBCFAF92BF926B
:101BA000CF92DF92FF920F931F93CF93DF938C011D
:101BB0005B01EA01FC01C688D788F08C80E590E0E3
:101BC0002ADD8F2D0E94D66E8C179D0720F48F2D55
:101BD0000E94D66EEC019E01A501B6018F2D0E94D8
:101BE000A48DF801868997898C0F9D1F978B868B12
:101BF000CE01DF91CF911F910F91FF90DF90CF9099
:101C0000BF90AF900895CF93FC01C08D80E590E028
:101C100002DD60E270E08C2F0E94C66E62E070E030
:101C20008C2FB7DC84FD13C062E070E08C2FB1DC38
:101C300083FF09C048E162E070E08C2F91DC90E006
:101C400080E0CF91089580E590E0E5DCE7CF40E1CA
:101C500062E070E08C2F84DC81E090E0F2CFFF92B4
:101C60000F931F93CF93DF93EB01FC01178A168A22
:101C70002A81211109C02B81211106C02C8121113B
:101C800003C02D812223C9F041155105B1F08A010D
:101C9000FC01F08C80E590E0BEDCBE016E5F7F4F02
:101CA0008F2DC5D8B8018F2D65DC81E090E0DF91E4
:101CB000CF911F910F91FF90089590E080E0F7CFB2
:101CC0004F925F926F927F928F929F92AF92BF924C
:101CD000CF92DF92EF92FF920F931F93CF93DF93F8
:101CE000CDB7DEB763970FB6F894DEBF0FBECDBF9A
:101CF0007C016B013A01FB0120E090E080E06AE0AA
:101D00003191332309F45EC040ED430F4A3008F0AF
:101D10004AC0689FA001699F500D1124CA01C09755
:101D2000830F911D37FD9A958F3F910549F340F33D
:101D3000F70142815381648175818091540E9091A5
:101D4000550EA091560EB091570E481759076A07C5
:101D50007B0709F416C28701085F1F4F0E94447772
:101D60006F7077277C5FC801C5DE813009F00EC235
:101D700081E094E09A838983F70182819381A48131
:101D8000B5818B839C83AD83BE8345E350E0BE0168
:101D90006F5F7F4FC80163DF892BA1F5D12CC12C68
:101DA000C8018ADE17C03E3209F0C2CF233009F4E1
:101DB000BFCFD301A20FB11D12968C932F5F90E07D
:101DC00080E09ECF233009F0B3CFF3018583CC248C
:101DD000C394D12CC60163960FB6F894DEBF0FBE34
:101DE000CDBFDF91CF911F910F91FF90EF90DF90CA
:101DF000CF90BF90AF909F908F907F906F905F90AB
:101E00004F9008950E944477F70177836683762781
:101E1000672776277A83698342E050E0BE016F5FCF
:101E20007F4FC801BBDE81E090E09E878D8742E056
:101E300050E0BE01635F7F4FC801B0DE80E091E0FB
:101E40009E878D8742E050E0BE01635F7F4FC801EF
:101E5000A5DE1E861D8642E050E0BE01635F7F4F17
:101E6000C8019CDE42E050E0BE01635F7F4FC801C5
:101E700095DE42E050E0BE01635F7F4FC8018EDE19
:101E80005601F60180818823F1F06501F601819108
:101E90002F01882311F08E32A1F446018A189B0885
:101EA0001814190464F48F8641E050E0BE01615FAC
:101EB0007F4FC80173DEA401B501C8016FDE520176
:101EC000E0CF6201E3CF1F8641E050E0BE01615FD9
:101ED0007F4FC80163DEC12CDD24D394DE86CD861E
:101EE00042E050E0BE01635F7F4FC80157DEDE86EF
:101EF000CD8642E050E0BE01635F7F4FC8014EDEF9
:101F0000C80181DE892B09F449CFF3E0AF2EB12C53
:101F1000230122E0420E511C5DC0F7014281538132
:101F200064817581808D918DA28DB38D481759077D
:101F30006A077B0709F01BC1848D958DC59709F051
:101F400016C181A192A10C970CF416C14CE050E08F
:101F5000BE016F5F7F4FC80148DC8B819C81982751
:101F6000892798279A8B898B29813A8132272327C1
:101F70003227F7014681578142175307D1F497FF63
:101F800018C08F709270892B09F041C06F807884DF
:101F9000762467247624D12CC12C6114710409F0B5
:101FA0004CC0C8010E947C066AEFC62EDD24DA947C
:101FB00007C0C8010E947C06ECEFCE2EDD24DA9427
:101FC00081E0A81AB10809F4EBCEFFEFCF16DF06C7
:101FD00009F0E6CE0E9444773B014C01C8014CDC7D
:101FE000181619060CF499CF0E94447766197709E0
:101FF00088099909693873418105910508F0B3C0D2
:1020000062E370E080E090E00E948A76E7CFC8014A
:102010000E947C067BEFC72EDD24DA94D1CF8D851C
:10202000811113C0C801FFDBC801FDDBC801FBDB68
:10203000C801F9DBFFEFCF1ADF0A8D819E81982757
:1020400089279827C816D90698F441E050E0BE01C8
:10205000635F7F4FC801C9DB8D85882301F38D85C0
:102060009FEF980F9D878823D1F2C801DCDBF7CF63
:10207000912C812C41E050E0BE016D5E7F4FC80184
:10208000B4DB8B89982F907C59F4882379F08B8965
:102090009FEF980F9B8B882331F0C801C4DBF7CFEB
:1020A000C801C1DB1B8A8B898111E4CF42E050E07B
:1020B000BE01615F7F4FC80198DB42E050E0BE0186
:1020C000635F7F4FC80191DBC801ADDBC801ABDBAB
:1020D000C801A9DBC801A7DB42E050E0BE016F5E8A
:1020E0007F4FC80182DB8F85988981159140E1F48B
:1020F000CD84DE84DC24CD24DC2481E0C816D10428
:1021000099F489899A898115944041F0C8010E9407
:102110007C0657EFC52EDD24DA9452CF44E050E020
:10212000B201C80162DB4CCFD12CC12C89899A89BC
:10213000982789279827C816D90630F4C80173DB79
:10214000FFEFCF1ADF0AF2CF2FEF821A920A68143C
:10215000790409F08FCFC8010E947C0646EFC42E97
:10216000DD24DA942DCFCC24CA94DC2C29CF2EEF99
:10217000C22EDD24DA9424CF9DEFC92EDD24DA941B
:102180001FCF8EEFC82EDD24DA9424CED12CC12CA3
:1021900021CECF92DF92EF92FF920F931F93CF93B6
:1021A000DF93CDB7DEB7AF970FB6F894DEBF0FBEA3
:1021B000CDBF7C016A0101E014E01A8309831C860B
:1021C0001B8688EE93E0A0E0B0E08D879E87AF8706
:1021D000B88B85E993E09A878987188F0F8B198EC2
:1021E0001A8E1B8E1C8E84E089A31BA70AA71CA62F
:1021F0001DA61EA61FA680914C0E90914D0EA0917B
:102200004E0EB0914F0E8EA39FA3A8A7B9A78B83A4
:102210009C83AD83BE8318861F82AE01465D5F4FEF
:10222000CE0101964DDD81309105B1F4D701ED91DC
:10223000FC910488F589E02D1DA30CA38CA59DA518
:10224000AEA5BFA58EA39FA3A8A7B9A7A601BE014F
:102250006C5D7F4FC7011995AF960FB6F894DEBF3E
:102260000FBECDBFDF91CF911F910F91FF90EF90E7
:10227000DF90CF900895CF92DF92EF92FF920F936D
:102280001F93CF93DF93CDB7DEB7AF970FB6F89418
:10229000DEBF0FBECDBF7C016A0101E014E01A83EE
:1022A00009831C861B8688EE93E0A0E0B0E08D8752
:1022B0009E87AF87B88B85E993E09A878987188FC7
:1022C0000F8B198E1A8E1B8E1C8E84E089A31BA780
:1022D0000AA71CA61DA61EA61FA680914C0E9091B3
:1022E0004D0EA0914E0EB0914F0E8EA39FA3A8A7A6
:1022F000B9A78B839C83AD83BE8318861F82AE01F2
:10230000465D5F4FCE010196DBDC81309105B1F473
:10231000D701ED91FC910684F785E02D1DA30CA358
:102320008CA59DA5AEA5BFA58EA39FA3A8A7B9A761
:10233000A601BE016C5D7F4FC7011995AF960FB620
:10234000F894DEBF0FBECDBFDF91CF911F910F91EB
:10235000FF90EF90DF90CF9008957F928F929F92A1
:10236000AF92BF92CF92DF92EF92FF920F931F93A3
:10237000CF93DF93CDB7DEB7A6970FB6F894DEBF45
:102380000FBECDBF8C01762E942E852E20E2A22E7C
:10239000CE0101967C01DC01EA2D1D92EA95E9F758
:1023A0006801F3E4CF0ED11C81E094E09AA389A3E5
:1023B0008FEF8BA38CA38DA38EA343E450E0BE01CB
:1023C0006F5D7F4FC6014BDC019609F4B8C081E018
:1023D00089838A8386E0B82EBB821C82D80114963A
:1023E0006D917D918D919C9117970E94F8A46D83BA
:1023F0007E838F83988789869A8680E890E09C8781
:102400008B874CE150E0B701C601C8DBFE0137966F
:102410008AE1DF011D928A95E9F74801B8E08B0E49
:10242000911CF401D70101900D92BA94E1F740E1BB
:1024300050E0B701C601B2DBF7011192AA94E9F7A7
:1024400096E0A92EB12C40E250E0B701C601A6DB10
:10245000F1E0AF1AB108B9F783E6898392E89A836D
:1024600093E59B838C8385E38D8381E08E837F82DC
:102470009DE3988797E099878A8786E0F401DE01DB
:102480001B9601900D928A95E1F78CE0898B8A8BDF
:1024900063E074E0CE0143960E9462A7D8011B96C8
:1024A0006C91CE0149960E943F70F8016485CE017F
:1024B0004B960E943F70D8011D966C91CE014D96AF
:1024C0000E943F704EE150E0B701C60167DBB3E008
:1024D0007B121DC082E3898384E08A83F80196859C
:1024E0009B8397859C8390899D8391899E8396E3A6
:1024F0009F838887828D8987838D8A87848D8B8748
:10250000858D8C874CE050E0B701C60147DB87E33F
:10251000898386E08A8391E09B8393E09C838D830B
:102520008FE08E838AE38F838BE388878FEF8987A1
:1025300049E050E0B701C60131DBC60164DBA69675
:102540000FB6F894DEBF0FBECDBFDF91CF911F91C4
:102550000F91FF90EF90DF90CF90BF90AF909F9042
:102560008F907F9008958F929F92AF92BF92CF925B
:10257000DF92EF92FF920F931F93CF93DF93CDB72C
:10258000DEB72D970FB6F894DEBF0FBECDBF7C012E
:1025900010E000E038EE832E33E0932EA12CB12C16
:1025A0004DEBC42E43E0D42E1C821B828D829E8272
:1025B000AF82B886DA82C9820D87CE010196C5DA6C
:1025C000811133C0F7014481558120E061E0802F03
:1025D000CFD980E590E01FD863E070E0802F0E94A3
:1025E000C90A833129F462E070E0802F0E94C66E30
:1025F000F70184819581000F111FF801E05BF34F13
:10260000918380832D960FB6F894DEBF0FBECDBFA9
:10261000DF91CF911F910F91FF90EF90DF90CF90BE
:10262000BF90AF909F908F9008950F5F1F4F043021
:10263000110509F0B9CFE6CFCF92DF92EF92FF926A
:102640001F93CF93DF93FC011485143079F1EC01D3
:1026500080E590E00E940B0B68E070E0812F0E9403
:10266000C66E0E9444776B017C01CE016EDA88232E
:1026700099F061E070E080E090E00E948A760E942C
:1026800044776C197D098E099F09683E7340810566
:10269000910558F38C855CD9EC85F0E0EE0FFF1FB7
:1026A000E05BF34F1182108284E08C87DF91CF9141
:1026B0001F91FF90EF90DF90CF9008954F925F921F
:1026C0006F927F928F929F92AF92BF92CF92DF9242
:1026D000EF92FF921F93CF93DF93CDB7DEB72D9785
:1026E0000FB6F894DEBF0FBECDBF7C0190E5A92EDA
:1026F0009CE0B92E10E0D12CC12C28EE422E23E014
:10270000522E612C712C3DEB832E33E0932E1C82D4
:102710001B824D825E826F8278869A8289821D87B3
:10272000D5012D913D915D01F70184819581281797
:10273000390799F4CE01019608DA843189F1CE0186
:10274000019603DA8C3149F4CE0101960E94880B80
:10275000892B19F4CE0101966FDF1F5F1430B9F693
:10276000CD2841F4D701ED91FC910084F185E02D55
:10277000C70119952D960FB6F894DEBF0FBECDBFD9
:10278000DF91CF911F91FF90EF90DF90CF90BF909E
:10279000AF909F908F907F906F905F904F90089533
:1027A000CC24C394D12CD9CF8F929F92AF92BF9259
:1027B000CF92DF92EF92FF920F931F93CF936C0112
:1027C0005B017A01FC01C485C430A1F481E090E092
:1027D000F60193838283F12CE12CC701CF911F91E5
:1027E0000F91FF90EF90DF90CF90BF90AF909F90B0
:1027F0008F9008958A014130584010F000E018E0B1
:1028000080E590E00E940B0B8C2F0E94D66E4C014D
:1028100063E070E08C2F0E94C90A873111F08C317F
:1028200021F58016910660F380E590E00E940B0B85
:102830009801A50170E060E08C2F0E94A48D60E2F9
:1028400070E08C2F0E94C66E62E070E08C2F0E94B8
:10285000C90A84FD12C063E070E08C2F0E94C90A8F
:10286000811106C08C2F74D8B1CF10E000E0DCCF0E
:1028700080E590E00E940B0BE7CF40E162E070E062
:102880008C2F0E94B00A012B09F0A7CF9FCF3F9257
:102890004F925F926F927F928F929F92AF92BF9270
:1028A000CF92DF92EF92FF920F931F93CF93DF931C
:1028B000CDB7DEB72D970FB6F894DEBF0FBECDBFF4
:1028C0006C015B014A01FADE80E5E82E8CE0F82E0F
:1028D000312C10E000E098EE492E93E0592E612C47
:1028E000712C1C821B824D825E826F8278868DEBFA
:1028F00093E09A8389833D86F701219131917F018D
:10290000F601848195812817390761F4CE0101967B
:102910001CD9873139F4A401B501CE01019644DFF9
:10292000080F191F3394F4E03F12DBCFC8012D9636
:102930000FB6F894DEBF0FBECDBFDF91CF911F91D0
:102940000F91FF90EF90DF90CF90BF90AF909F904E
:102950008F907F906F905F904F903F9008950A9670
:1029600023CFCF92DF92FF920F931F93CF93DF93EA
:10297000FC012485243051F090E080E0DF91CF917C
:102980001F910F91FF90DF90CF9008956A01EB01A6
:102990008C01F12C8F2DA4D8811129C0F801F48667
:1029A000F8018485843041F320919C0230919D028E
:1029B0002F5F3F4F21F130939D0220939C02409165
:1029C0009C0250919D0220E061E00E94B80C8A8137
:1029D0008F3FC1F48B818F3F01F58C818F3FE9F4EC
:1029E0008D818F3FD1F484E0F8018487C5CF8B7F40
:1029F0008831A1F2F394F4E0FF12CCCFD1CF20E0E4
:102A000030ECD9CF811109C08B81811106C08C8136
:102A1000811103C08D81882331F3C114D10419F3CE
:102A2000F801F48480E590E00E940B0BBE016E5F1C
:102A30007F4F8F2D0E941707B6018F2D0E94BA0A73
:102A400064E070E08F2D0E94C66EC8017ED8873189
:102A500059F061E070E080E090E00E948A76C80161
:102A600074D88111F2CFBFCF81E090E087CFCF93B0
:102A7000CFB7F8948091200C811127C0E9EAFAE0E1
:102A80008491EFEEFAE09491E82FF0E0EE0FFF1F53
:102A9000EA5DF54FA591B491EC91E92321F461E051
:102AA00085E30E94437561E085E30E9459768CB509
:102AB00080618CBD8CB580648CBD61E084E30E9434
:102AC000597661E083E30E9459768091200C8F5FF4
:102AD0008093200CCFBFCF9108954F925F926F9259
:102AE0007F928F929F92AF92BF92CF92DF92EF929E
:102AF000FF920F931F93CF93DF93EC018090A80276
:102B00009090A902E5E4F2E081E090E0512C412CA4
:102B10008816990654F0219131912130310519F42C
:102B20002FEF421A520A0196F3CF1C161D060CF025
:102B30004AC08C169D060CF446C04E018E01000F53
:102B4000111F7E01EE0CFF1CEE0CFF1C8C169D0667
:102B50000CF4D9C0C701895C9D4F6C01FC018081D8
:102B60009181A281B3819701215B3D4F59011816D4
:102B700019061A061B0654F50E94C179F501208139
:102B8000318142815381621B730B840B950BF601DB
:102B90002081318142815381261737074807590721
:102BA00058F410821182128213820E94C179F501B9
:102BB000608371838283938321960E5F1F4FF4E0BD
:102BC000EF0EF11CC3CFC1E0D0E0B8CF98012E5575
:102BD0003D4F3901F9018081918198012D5B3D4F75
:102BE0006901F9012081318182179307F1F0F3E047
:102BF0004F16510414F00097C1F4880F991FFC017F
:102C0000E952F44F6081F801E452F44F80810E9450
:102C10004375F30180819181F601918380836CE299
:102C200071E080E090E00E948A76F50180819181D8
:102C3000A281B381181619061A061B060CF0BCCF28
:102C40000E94C179F5012081318142815381621B4B
:102C5000730B840B950BF701E55AFD4F20813181F1
:102C600042815381261737074807590708F0A4CF38
:102C7000F50110821182128213829801275B3D4F69
:102C80005901F90180819181F601208131818217FA
:102C9000930709F491CF6091A8027091A902E5E42D
:102CA000F2E041E050E030E020E0641775074CF0BE
:102CB000A191B191119711F42F5F3F4F4F5F5F4F7B
:102CC000F4CF233031051CF0009709F075CF880F41
:102CD000991FFC01E952F44F6081F801E452F44F6E
:102CE00080810E944375F50180819181F601918375
:102CF0008083F301918380836CE271E080E090E057
:102D00000E948A7659CFDF91CF911F910F91FF904A
:102D1000EF90DF90CF90BF90AF909F908F907F907B
:102D20006F905F904F900895CF93DF93FC012481C3
:102D30003581232B69F0EC01BC0186E59DE00E9402
:102D40004174BE0189EB9CE0DF91CF910C944174FA
:102D5000DF91CF910895CF93DF93FC0124813581DA
:102D6000232B69F0EC01BC0186E59DE00E943374E1
:102D7000BE0189EB9CE0DF91CF910C943374DF911D
:102D8000CF910895CF93DF93FB0122813381DC0142
:102D900013963C932E9312974481558166817781D7
:102DA00014964D935D936D937C9317974085518551
:102DB0006285738518964D935D936D937C931B97F5
:102DC0001C96EF012C969C01275E3F4F49914D9335
:102DD000A217B307D9F7218D328DFC01328F218FD5
:102DE000DF91CF910895CF92DF92EF92FF920F93F0
:102DF0001F93CF93DF93CDB7DEB7A0970FB6F894AC
:102E0000DEBF0FBECDBF7C018B0150E040E06C0106
:102E10008AE0C80ED11CCA010196F8012491E1E0B4
:102E2000F0E0EC0FFD1FE40FF51F2083222381F05B
:102E30008032910549F440E250E0BE016F5F7F4F60
:102E4000C601B2DC90E080E00F5F1F4FAC01E3CF22
:102E5000029730F0BE016F5F7F4FC7010A96A4DC76
:102E6000A0960FB6F894DEBF0FBECDBFDF91CF9115
:102E70001F910F91FF90EF90DF90CF900895EF9208
:102E8000FF920F931F93CF93DF93EC018B017A0195
:102E900067E772E0A8DFB801CE010E942C748E01B2
:102EA000065F1F4F42E050E069EE79E0C8017CDC2C
:102EB000E114F10421F0B701CE010E942C7442E02C
:102EC00050E069EE79E0C801DF91CF911F910F9139
:102ED000FF90EF9069CC69E172E085CFCF92DF92ED
:102EE000EF92FF920F931F93CF93DF9300D000D008
:102EF000CDB7DEB77C01FB01848195818A01081B77
:102F0000190B101611069CF0C7010E94DA72C70156
:102F100026960FB6F894DEBF0FBECDBFDF91CF91DE
:102F20001F910F91FF90EF90DF90CF900895CE0109
:102F300001960E94EA72CC24C394D12C62EE75E013
:102F4000CE0101960E94DD71FFEFCF1ADF0A0C154A
:102F50001D05A4F7BE016F5F7F4FC7010E94DA72A3
:102F6000CE0101960E945D72D2CFDF92EF92FF9266
:102F70000F931F93CF93DF93CDB7DEB762970FB652
:102F8000F894DEBF0FBECDBF2091DE02222379F17F
:102F90002091DD02222359F17A018C016F3F7F4F8E
:102FA000A1F560E080E00E944579D12CB80188ED60
:102FB00091E10E94337463EC73E088ED91E10E942B
:102FC0005374F801848160E08D0D0E9445790E9460
:102FD000447760937A0C70937B0C80937C0C909375
:102FE0007D0CB701FF0C880B990B0E948A766296C4
:102FF0000FB6F894DEBF0FBECDBFDF91CF911F910A
:103000000F91FF90EF90DF90089560E080E00E94C4
:1030100045790E94447728EE33E040E050E00E947A
:103020006EA3CA01B90120E831E541E050E00E94F9
:1030300090A3AB01BC0120E0CE0101960E949672E4
:10304000BE016F5F7F4FCE0107960E94EA7268E76C
:1030500078E0CE0107960E947071BC01CE010D96FA
:103060000E94EA72CE0107960E945D72CE0101961F
:103070000E945D72BE01635F7F4F88ED91E10E9407
:103080003374D98860E08D2D0E944579CE010D966C
:103090000E945D728BCFEF92FF920F931F93CF939D
:1030A000DF9300D000D0CDB7DEB78C017B0165ED9A
:1030B00078E00E94F2728AE0E816F1042CF468E9E4
:1030C00076E0C8010E94DD71B701CE0101960E9431
:1030D0005A70BE016F5F7F4FC8010E94E671CE013A
:1030E00001960E945D72C80126960FB6F894DEBF65
:1030F0000FBECDBFDF91CF911F910F91FF90EF9049
:103100000895CF92DF92EF92FF920F931F93CF9388
:10311000DF93CDB7DEB7C455D1090FB6F894DEBF43
:103120000FBECDBF65965FAF4EAF65972091590C2E
:1031300030915A0C2F5F3F4F30935A0C2093590C0B
:103140002091580C2111C9C08B016C0181E0809342
:10315000580C10925A0C1092590C65ED78E0CE0183
:10316000895B9F4F0E94F27265ED78E0CE01835B30
:103170009F4F0E94F27250E040E06AE074E0C601A6
:103180007EDE0130110509F097C065ED78E088EF2B
:103190009FE00E94517065ED78E084ED9FE00E9411
:1031A00051706596EEADFFAD65978081882309F477
:1031B0007DC000E210E09E012F5F3F4F40E250E0F3
:1031C000BE016F5D7F4FCE018D5A9F4F0E94F26E00
:1031D000049739F3BE016F5D7F4FCE018F5B9F4F28
:1031E0000E94F272BE016F5B7F4FCE01895B9F4FE1
:1031F0000E942472CE018F5B9F4F0E945D72BE01C0
:103200006F5F7F4FCE018F5B9F4F0E94F272BE01B6
:103210006F5B7F4FCE01835B9F4F0E942472CE0174
:103220008F5B9F4F0E945D7270E060E0CE01895B12
:103230009F4F0E942471823569F42D968EAD9FAD0B
:103240002D970297029730F463E274E084ED9FE0DB
:103250000E945170BE01695B7F4F88EF9FE00E9422
:10326000E67163968EAD9FAD6397892B09F499CF74
:1032700065EE75E0CE018F5B9F4F0E94F272BE013A
:10328000635B7F4FCE018F5B9F4F0E94847162EE24
:1032900075E00E947071BC0188EF9FE00E94E671AA
:1032A000CE018F5B9F4F0E945D727BCF68EF7FE006
:1032B00084ED9FE00E94E6711092580CCE01835B72
:1032C0009F4F0E945D72CE01895B9F4F0E945D728D
:1032D0000FB6F894DEBF0FBECDBFCC5ADF4F0FB68E
:1032E000F894DEBF0FBECDBFDF91CF911F910F913C
:1032F000FF90EF90DF90CF9008950F931F93CF939F
:10330000DF93CDB7DEB72C970FB6F894DEBF0FBEB4
:10331000CDBF2C893D893093A9022093A802FE01DC
:103320007496ACEDBBE090E080E032962817390748
:1033300034F0408151814D935D930196F6CF8C8D91
:103340009D8D9093D80B8093D70B8E8D9F8D9093EE
:10335000DA0B8093D90BAD968FADAD97BE01645952
:103360007F4F8F3209F0B9C1CE0107960E94F272E9
:103370006AE274E0CE0101960E94F272BE01695FBA
:103380007F4FCE0101960E948471BC0180E891E1DB
:103390000E940F72CE0101960E945D72CE010796C7
:1033A0000E945D7260E871E1CE0101960E94EA72AE
:1033B000CE010196B9DCCE0101960E945D7260E4F7
:1033C00074E0CE0101960E94F272BE016F5F7F4FE2
:1033D00080E891E10E943571182FCE0101960E947C
:1033E0005D724091841150918511112309F47CC1C3
:1033F000BA016250710980E891E10E942471682F3E
:10340000CE0101960E94C272BE016F5F7F4F82E6BD
:1034100091E10E942472CE0101960E945D726AE5DC
:1034200070E1CE0107960E94F27262E474E0CE0170
:1034300001960E94F272BE01695F7F4FCE01019634
:103440000E948471BC018AE791E10E940F72CE0153
:1034500001960E945D72CE0107960E945D722496CD
:103460008FAD24971F928F9323968FAD23971F9232
:103470008F9322968FAD22971F928F9321968FADB7
:1034800021971F928F9388E494E09F938F938EE00F
:103490009CE09F938F930E94A0A7CE52DF4F88811C
:1034A0009981C25DD0409093840280938302BE01D3
:1034B0006C527F4FCE0101960E94F272BE016F5F87
:1034C0007F4F84E791E10E942472CE0101960E9411
:1034D0005D72BE0161527F4FCE0101960E94F27271
:1034E000BE016F5F7F4F8EE691E10E942472CE0194
:1034F00001960E945D724091721150917311425079
:1035000051096EE671E1CE0101960E94F307CE01EA
:1035100001960E94BC706C596093B502CE01019671
:103520000E945D72CC5EDE4F688179818A819B81C9
:10353000C451D1400E9436A20FB6F894DEBF0FBE30
:10354000CDBF9B01AC010E94CDA4882389F08CE300
:1035500090E0A0E0B0E0CC5EDE4F88839983AA8340
:10356000BB83C451D140CD5EDE4F1882C351D140E0
:10357000CD5EDE4F8881C351D140882399F0CC5E67
:10358000DE4F88819981AA81BB81C451D14080934B
:10359000AC029093AD02A093AE02B093AF0281E073
:1035A0008093770CC85EDE4F688179818A819B8128
:1035B000C851D1409B01AC010E94CDA4882361F089
:1035C00080E090E0A0E7B2E4C85EDE4F8883998394
:1035D000AA83BB83C851D140C45EDE4F6881798124
:1035E000CC51D140072E000C880B990B0E9436A2BB
:1035F0009B01AC010E94CDA4882341F082E090E0C1
:10360000C45EDE4F99838883CC51D140C45CDE4FC9
:1036100008811981CC53D140B801012E000C880BD0
:10362000990B0E9436A29B01AC010E94CDA481118E
:1036300003C01016110644F080E590E0C45CDE4F34
:1036400099838883CC53D140C45CDE4F88819981B3
:10365000CC53D140909336028093350288E2FE012C
:10366000E551FF4FA2EEBBE001900D928A95E1F784
:10367000CE5CDE4F88819981AA81BB81C253D14043
:103680008093200290932102A0932202B093230200
:10369000CA5CDE4F88819981AA81BB81C653D14023
:1036A00080931C0290931D02A0931E02B0931F02F0
:1036B000C65CDE4F88819981CA53D14090936802DD
:1036C000809367022C960FB6F894DEBF0FBECDBF75
:1036D000DF91CF911F910F910895CE0107960E941F
:1036E000F2726FE274E046CE4150510960E871E138
:1036F000CE0101960E94F307BE016F5F7F4F82E605
:1037000091E10E942472CE0101960E945D7260E8F0
:1037100071E1CE0101960E94EA7260E474E0CE018C
:1037200001960E947071BC0180E891E10E940F72C5
:1037300072CE0F931F93CF93DF9300D000D0CDB7FD
:10374000DEB72091DB0B2223A9F08C016EE877E035
:10375000CE0101960E94F272B801CE0101960E943C
:103760008471BC0186E59DE00E944174CE01019602
:103770000E945D7226960FB6F894DEBF0FBECDBFD5
:10378000DF91CF911F910F910895DF92EF92FF92F9
:103790000F931F93CF93DF93CDB7DEB762970FB62A
:1037A000F894DEBF0FBECDBF8C0110920D0B65EDFE
:1037B00078E0CE010D960E94F272FF24F39486E524
:1037C0009DE00E94FA6A20910D0B1816190674F5F7
:1037D00021112CC086E59DE00E94D86A8A3009F04C
:1037E0007DC089899A89892B09F480C0F0920D0BDC
:1037F00064E574E0CE0101960E94F272BE01635F3F
:103800007F4FCE0101960E948471BC01CE010796C4
:103810000E94EA72CE0107968CDFCE0107960E94C5
:103820005D72CE0101960E945D7260C0F12CE12CA8
:10383000DD24D394222309F460C089899A890197F1
:1038400009F045C063ED74E0CE0107960E94F27264
:10385000BE01695F7F4FCE010D960E945571F12C1C
:10386000811115C064E674E0CE0101960E94F272E7
:10387000BE016F5F7F4FCE010D960E945571FF24F0
:10388000F3948111F12CCE0101960E945D72CE015C
:1038900007960E945D72FF20A1F050E040E0BE015B
:1038A000635F7F4FCE0101960E94F307BE016F5FF9
:1038B0007F4F8BE99FE00E942472CE0101960E9407
:1038C0005D7264E170E080E090E00E948A76BE0163
:1038D000635F7F4FC8010E94DA728CC08D3009F49B
:1038E00080CF682FCE010D960E94BE716AE070E015
:1038F00080E090E00E948A7662CF89EB9CE00E9493
:10390000FA6A1816190614F589EB9CE00E94D86A29
:103910008A30A9F08D3099F090910D0B91110FC064
:10392000682FCE010D960E94BE718FEFE81AF80A3B
:1039300065E070E080E090E00E948A76DECF8989C1
:103940009A89892BA9F3D0920D0BF2CF64E170E034
:1039500080E090E00E948A76EF2809F43DC08989D2
:103960009A89892BC9F18091DB0B882379F16EE864
:1039700077E0CE0101960E94F272BE016F5F7F4F29
:10398000CE010D960E945571F82ECE0101960E942F
:103990005D72F1101BC06DE574E0CE0101960E94CE
:1039A000F272CE010196D7D9CE0101960E945D72C6
:1039B000BE01635F7F4FCE0101960E94EA72CE0185
:1039C0000196B2D9CE0101960E945D7264E170E069
:1039D00080E090E00E948A7689899A8920910D0B77
:1039E00021112DCF009709F02ACF65ED78E0C801AD
:1039F0000E94F272CE010D960E945D72C80162961D
:103A00000FB6F894DEBF0FBECDBFDF91CF911F91EF
:103A10000F91FF90EF90DF9008950F931F93CF9336
:103A2000DF93CDB7DEB72C970FB6F894DEBF0FBE8D
:103A3000CDBF8C010E94197BBC01C8012CDB0E9408
:103A4000137BBC01CE01079626DB66EC76E0CE0147
:103A500001960E94F272BE01695F7F4FCE0101960E
:103A60000E948471BC01C8010E94E671CE010196DA
:103A70000E945D72CE0107960E945D7262EE75E053
:103A8000C8010E94DD710E940D7BBC01CE01019630
:103A900002DBBE016F5F7F4FC8010E94E671CE015D
:103AA00001960E945D7266E674E0C8010E94DD71B5
:103AB0000E94077BBC01CE010196EDDABE016F5F6B
:103AC0007F4FC8010E94E671CE0101960E945D728F
:103AD00066E674E0C8010E94DD710E94FF7ABC01B5
:103AE000CE010196D8DABE016F5F7F4FC8010E94F8
:103AF000E671CE0101960E945D72C8012C960FB648
:103B0000F894DEBF0FBECDBFDF91CF911F910F9113
:103B10000895CF93DF9300D000D0CDB7DEB70E94D9
:103B2000FF07CE01019679DF4AE050E06FEF7FEFAB
:103B3000CE0101961ADACE0101960E945D7261E013
:103B400080E00E944579CE0101960E94B66F68ED33
:103B500071E1CE0101960E94BE7368E674E088EDC3
:103B600091E10E942C740E9444776093630C7093DF
:103B7000640C8093650C9093660C26960FB6F894AF
:103B8000DEBF0FBECDBFDF91CF9108950F931F937E
:103B9000CF93DF9300D000D0CDB7DEB78C01CE013C
:103BA00001963BDF4AE050E06FEF7FEFCE010196D8
:103BB000DCD9CE0101960E945D72B801CE0101965A
:103BC0000E94EA726AE070E0CE0101960E9471796B
:103BD000CE0101960E945D7226960FB6F894DEBF64
:103BE0000FBECDBFDF91CF911F910F9108950F931D
:103BF0001F93CF93DF93CDB7DEB72C970FB6F89412
:103C0000DEBF0FBECDBF8C010E94197BBC01C80175
:103C100042DA0E94137BBC01CE0107963CDA66ECC7
:103C200076E0CE0101960E94F272BE01695F7F4F7D
:103C3000CE0101960E948471BC01C8010E94E67108
:103C4000CE0101960E945D72CE0107960E945D72C0
:103C50000E94C1790E94067A6091430C70E0CE0107
:103C6000079619DA66EC76E0CE0101960E94F272B0
:103C7000BE01695F7F4FCE0101960E948471BC0135
:103C8000C8010E94E671CE0101960E945D72CE01CC
:103C900007960E945D7262EE75E0C8010E94DD71B8
:103CA0000E940D7BBC01CE010196F5D9BE016F5F6C
:103CB0007F4FC8010E94E671CE0101960E945D729D
:103CC00066E674E0C8010E94DD710E94077BBC01BA
:103CD000CE010196E0D9BE016F5F7F4FC8010E94FF
:103CE000E671CE0101960E945D7266E674E0C8013D
:103CF0000E94DD710E94FF7ABC01CE010196CBD9F2
:103D0000BE016F5F7F4FC8010E94E671CE01019630
:103D10000E945D72C8012C960FB6F894DEBF0FBEEC
:103D2000CDBFDF91CF911F910F910895611571055E
:103D300019F00A960C944F7390E080E008952F924A
:103D40003F924F925F926F927F928F929F92AF922B
:103D5000BF92DF92EF92FF920F931F93CF93DF9367
:103D6000CDB7DEB7E4970FB6F894DEBF0FBECDBF78
:103D70007C014A015B0119010E9444772B013C013F
:103D800087010D5B1F4FC8010E943C0C18161906D5
:103D90009CF00E9444776419750986099709861674
:103DA0009706A806B90608F490C162E370E080E0C7
:103DB00090E00E948A76E7CF42E250E0BE016F5F5A
:103DC0007F4FC8010E94F50B8981823009F078C1CC
:103DD000F801848995898334910509F071C16D8159
:103DE0007E818F8198850E94F8A42B013C01F1010E
:103DF000408251826282738246E050E0B701685F80
:103E00007F4FCE014D960E9420A7892B99F4F70190
:103E100080819181A281B381481659066A067B068A
:103E200048F084819581A681B78184159505A60502
:103E3000B705E8F4C8010E947C06D12C8D2DE496CC
:103E40000FB6F894DEBF0FBECDBFDF91CF911F91AB
:103E50000F91FF90EF90DF90BF90AF909F908F9069
:103E60007F906F905F904F903F902F900895898939
:103E70009A89AB89BC8986879787A08BB18B8EEC9A
:103E8000A82EB12CC8010E94130CF1E0AF1AB108A2
:103E9000C9F7D12CC70182969AA789A7F701B696D0
:103EA000FCA7EBA708969EA78DA73C974F01899684
:103EB00098AB8FA73897FAABE9AB1701F6E12F0E55
:103EC000311CC5979CAB8BABF801818D928D181678
:103ED00019060CF0F6C0C8010E94130C833391053B
:103EE00009F4D4C0A4F58130910509F474C074F4C8
:103EF000892B51F3C8010E94130CB82EBA94FFEF1E
:103F0000BF1611F3C8010E94130CF8CF833091053E
:103F100009F46CC0069771F7C8010E94130CA82E13
:103F200044E050E06BA97CA9C8010E94F50B712CFC
:103F3000612CEA2DE450FF0B5F016A147B0424F628
:103F4000C8010E94130CFFEF6F1A7F0AF6CF8A3365
:103F5000910509F46FC074F585339105A1F1C697F9
:103F600049F6C8010E94130CB82EF701828D811109
:103F700009C0838D811106C0848D811103C0858D98
:103F80008823A1F0EFA5F8A940805180628073805A
:103F9000B401CE0183960E9477748DA19EA1AFA13A
:103FA000B8A584159505A605B705D9F544E050E0F8
:103FB000B40118C08B33910509F452C08F3F9105AD
:103FC00009F482CF97CFC8010E94130CC8010E9448
:103FD000130CD82E79CFC8010E94130C44E050E096
:103FE00069A97AA9C8010E94F50B6ECFC8010E9489
:103FF000130CA82E44E050E0B101C8010E94F50B5B
:10400000712C612C8A2D8450990B5C016A147B04FD
:104010000CF05ACFC8010E94130C9FEF691A790A5D
:10402000F5CFBA94FFEFBF1609F44ECFC8010E9436
:10403000130CF7CFC8010E94130C44E050E06BA5AD
:104040007CA5C8010E94F50BF70166A177A180A5A8
:1040500091A50E94F8A466A377A380A791A734CF67
:10406000C8010E94130C44E050E06DA57EA5C80174
:104070000E94F50BF70162A573A584A595A50E9482
:10408000F8A462A773A784A795A71ECFC8010E94B2
:10409000130C44E050E069A57AA5C8010E94F50B15
:1040A000F70162A173A184A195A10E94F8A462A363
:1040B00073A384A395A366A777A780AB91AB04CF26
:1040C000D12CC8010E947C06B9CEDD24DA94B6CE8C
:1040D0002F923F924F925F926F927F928F929F9218
:1040E000AF92BF92CF92DF92EF92FF920F931F9306
:1040F000CF93DF9300D000D0CDB7DEB78C010E9404
:10410000599C2FEC37E040E050E00E9490A3DC0186
:10411000CB010196A11DB11DF80184839583A6836F
:10412000B78380839183A283B3835801F3E4AF0EF6
:10413000B11CC5010E945C0D64E470E0C5010E94E1
:104140007A0D882309F443C10E9444772B013C0176
:10415000480182E4880E911C48EEC42E43E0D42E20
:10416000E12CF12C52E0252E1E821D82D4018C916F
:104170008330B1F1811166C0F80184819581A681F7
:10418000B7810196A11DB11D84839583A683B78352
:104190000E9444776419750986099709A701960159
:1041A0000E946EA3A90161E0C8010E94AD1181E0E7
:1041B000D4018C938D819E810197C1F20E94447736
:1041C0006419750986099709D801D6962D913D91F4
:1041D0004D915C91D997261737074807590720F664
:1041E000C5010E945C0DF80184819581A681B7818B
:1041F0000196A11DB11D84839583A683B7830E9478
:104200004477F801FE9660837183828393838D8166
:104210009E8126960FB6F894DEBF0FBECDBFDF910C
:10422000CF911F910F91FF90EF90DF90CF90BF90B3
:10423000AF909F908F907F906F905F904F903F9046
:104240002F9008958430F1F4F80184819581A6813E
:10425000B7810196A11DB11D84839583A683B78381
:104260000E9444776419750986099709A701960188
:104270000E946EA3A90163E0C8010E94AD11D401A0
:104280002C9298CF813049F5F80142AD53AD64AD21
:1042900075AD9E012F5F3F4FC80151DD382EF2E012
:1042A0008F138FC089819A81AB81BC81F80184838F
:1042B0009583A683B7830E9444776419750986099C
:1042C0009709A70196010E946EA3A90163E0C801A6
:1042D0000E94AD11D4013C926DCF823009F06ACFBB
:1042E000F80142AD53AD64AD75AD9E012F5F3F4FF8
:1042F000C80125DD382EF5E08F135DC0E3E0D40161
:10430000EC93F80182A193A1A4A1B5A1892B8A2BDA
:104310008B2B41F484E893E0A0E0B0E082A393A368
:10432000A4A3B5A3F80186A197A1A0A5B1A5892B47
:104330008A2B8B2B61F482A193A1A4A1B5A1B69580
:10434000A7959795879586A397A3A0A7B1A7F801EE
:1043500082A593A5A4A5B5A5892B8A2B8B2BA9F49F
:1043600082A193A1A4A1B5A1AC01BD0123E07695E2
:104370006795579547952A95D1F7841B950BA60B02
:10438000B70B82A793A7A4A7B5A7F80186A197A109
:10439000A0A5B1A586A797A7A0ABB1AB82A593A511
:1043A000A4A5B5A582AB93ABA4ABB5AB81E090E07F
:1043B0009E838D83FFCE96E0891303C0D4011C92A7
:1043C000F9CEBFEF3B12F6CEF4011082F3CE1E827F
:1043D0001D821DCF7F928F929F92AF92BF92CF92FC
:1043E000DF92EF92FF920F931F93CF93DF93CDB79E
:1043F000DEB762970FB6F894DEBF0FBECDBF10E0F8
:1044000000E03EE0C32E3BE0D32E40E3E42E53EE2B
:10441000B52E66E0A62E7CEE972EE1E3FE2EFEE49E
:104420008F2EA4E37A2E68EB72E28DEA9FE00E9461
:104430007A0DF6018E2D11928A95E9F7B0920E0B46
:10444000A092100B9092110BF0921A0B80921B0B02
:10445000F0921C0B70921D0B60E072E0CE01019691
:104460000E9477744BE750E0BE016F5F7F4F8DEA8B
:104470009FE00E942F0E40E350E06EE07BE08DEA6B
:104480009FE00E94CE0D8DEA9FE00E94030E68EE31
:1044900073E080E090E00E948A768DEA9FE00E94BF
:1044A0003C0C892B31F50A30110509F05DC16CE631
:1044B00074E0CE0101960E94F272CE0101960E9434
:1044C0009416CE0101960E945D7262960FB6F89422
:1044D000DEBF0FBECDBFDF91CF911F910F91FF9037
:1044E000EF90DF90CF90BF90AF909F908F907F9094
:1044F000089540E350E06EE07BE08DEA9FE00E948B
:10450000F50B6091360B7091370B7627672776276E
:1045100090E080E0CB0177276627C090380BD090E1
:10452000390BDC24CD24DC24F12CE12C6C297D29F1
:104530008E299F297E508A4A93480E949D790E9425
:10454000C17960933E0B70933F0B8093400B909327
:10455000410B0A30110509F4AACF0E94C17960937A
:10456000670C7093680C8093690C90936A0C0E949E
:10457000C17960936B0C70936C0C80936D0C90936D
:104580006E0CCE01019633DBCE0101960E9494168B
:10459000CE0101960E945D720E940D7BBC01CE018E
:1045A00007960E944B1866E674E0CE0107960E94BB
:1045B000DD710E94077BBC01CE0101960E944B1861
:1045C000BE016F5F7F4FCE0107960E94E671CE015C
:1045D00001960E945D7266E674E0CE0107960E9425
:1045E000DD710E94FF7ABC01CE0101960E944B183A
:1045F000BE016F5F7F4FCE0107960E94E671CE012C
:1046000001960E945D7266E774E0CE0101960E94F9
:10461000F272BE01695F7F4FCE0101960E948471E4
:10462000BC01CE010D960E94EA724AE050E06FEFA5
:104630007FEFCE010D960E94B517CE010D960E9418
:104640005D72CE0101960E945D72CE0107960E94B6
:104650005D7268EE73E080E090E00E948A760E94CE
:10466000197BBC01CE010D960E944B180E94137B52
:10467000BC01CE0101960E944B1866EC76E0CE019B
:1046800007960E94F272BE016F5F7F4FCE010796C0
:104690000E948471BC01CE010D960E94E671CE018C
:1046A00007960E945D72CE0101960E945D720E9483
:1046B000C1790E94067A6091430C70E0CE010196A8
:1046C0000E944B1866EC76E0CE0107960E94F272CB
:1046D000BE016F5F7F4FCE0107960E948471BC01BF
:1046E000CE010D960E94E671CE0107960E945D7282
:1046F000CE0101960E945D726CE774E0CE010196D6
:104700000E94F272BE01635F7F4FCE0101960E944C
:104710008471BC01CE0107960E94EA724AE050E023
:104720006FEF7FEFCE0107960E94B517CE01079677
:104730000E945D72CE0101960E945D72CE010D96BF
:104740000E945D7268EE73E080E090E00E948A76DD
:10475000CE01019662D94AE050E06FEF7FEFCE01C3
:1047600001960E94B517ADCE0F5F1F4F68EE73E044
:1047700080E090E00E948A7640913E0B50913F0B82
:104780006091400B7091410BCE0101960E948570A3
:10479000CE0101960E949416CE0101960E945D7290
:1047A00042CEEF92FF920F931F93CF93DF93CDB73B
:1047B000DEB7E8970FB6F894DEBF0FBECDBF65ED4C
:1047C00078E0CE0187960E94F27265ED78E0CE0126
:1047D0008D960E94F27282E0E82EF12C2496FFAEB4
:1047E000EEAE249786E0EFEEF2E0DE01D396019084
:1047F0000D928A95E1F786E0FE01F396DE01AC5B4F
:10480000BF4F01900D928A95E1F72C961FAE1EAE18
:104810002C9701E010E02E961FAF0EAF2E9788E088
:10482000E5EFF2E0DE01599601900D928A95E1F7ED
:1048300088E0FE017996DE01A25BBF4F01900D92E8
:104840008A95E1F788E1EDEFF2E0DE011196019043
:104850000D928A95E1F788E1FE013196DE01AA5AB0
:10486000BF4F01900D928A95E1F7809115039091C9
:104870001603A0911703B0911803E2968CAF9DAF79
:10488000AEAFBFAFE29762E874E0CE0187960E94B8
:10489000517060E0CE0187960E94BE714BA55CA569
:1048A000BE016E587F4FCE0187960E94D36F62EC97
:1048B00075E0CE018D960E94EC716AEC74E082E6A0
:1048C00091E10E94517060E0CE018D960E94BE7110
:1048D00049A95AA9BE0166567F4FCE018D960E9406
:1048E000D36F65ED78E0CE0187960E94517065ED3B
:1048F00078E0CE018D960E945170C250DF4F198230
:104900001882CE5FD0408091830290918402C05083
:10491000DF4F99838883C050D14080E090E0A0E7CA
:10492000B2E4CA5BDE4F88839983AA83BB83C654F3
:10493000D140C65BDE4FF982E882CA54D14080E0A4
:1049400090E0A0E2B2E4C45BDE4F88839983AA833F
:10495000BB83CC54D14080E090E0A4E3B2E4C05BE0
:10496000DE4F88839983AA83BB83C055D14084EBF3
:1049700090E0CC5ADE4F99838883C455D14088E7B4
:1049800090E0CA5ADE4F99838883C655D1408CE2A5
:1049900091E0A0E0B0E0C85ADE4F88839983AA83F3
:1049A000BB83C855D140C45ADE4F19830883CC5508
:1049B000D140C25ADE4FF982E882CE55D14060E044
:1049C00084E791E10E94BE7160E08EE691E10E9471
:1049D000BE714091781150917911BE016E5F7E4F8A
:1049E00084E791E10E94D36F40917211509173114D
:1049F000BE01635F7E4F8EE691E10E94D36F88E235
:104A0000E2EEFBE0DE01A75EBE4F01900D928A95BB
:104A1000E1F78CE390E0A0E0B0E0CE5BDE4F88836E
:104A20009983AA83BB83C254D140CF5BDE4F1882E7
:104A3000C154D14084EE98E3AEE8B2E4C05ADE4FF0
:104A400088839983AA83BB83C056D14084EE98E3C0
:104A5000AEE8B1E4CC59DE4F88839983AA83BB8347
:104A6000C456D140C859DE4F19830883C856D14077
:104A700080E590E0C659DE4F99838883CA56D140BD
:104A800084EF91E090939B0280939A02BE016E5B4B
:104A90007F4F0E94B20764EF71E080E090E00E94D7
:104AA0008A766BEA75E0CE0181960E94E272CE01B1
:104AB00081960E949416CE0181960E945D72CE016D
:104AC0008D960E945D72CE0187960E945D72E89677
:104AD0000FB6F894DEBF0FBECDBFDF91CF911F910F
:104AE0000F91FF90EF9008959F92AF92BF92CF9257
:104AF000DF92EF92FF920F931F93CF93DF93CDB787
:104B0000DEB7C859D1090FB6F894DEBF0FBECDBFCE
:104B10005C017B016A0162E870E1CE0189579F4F19
:104B20000E94F27260E474E08E010F5F1F4FC801B3
:104B30000E94F272B801CE0189579F4F0E945571B1
:104B4000982EC8010E945D72911014C060E474E058
:104B5000C8010E94F272BE0169577F4FC8010E94CE
:104B60008471BC01CE0189579F4F0E940F72C8010A
:104B70000E945D72B501CE0183579F4F0E94F27271
:104B80006AE874E021E0E216F10441F065E974E0BE
:104B900032E0E316F10411F06DE974E0CE018957BB
:104BA0009F4F0E94DD7160E0CE0189579F4F0E94A8
:104BB000BE71B601C8010E94EA726AE0C8010E9493
:104BC000D171BC01CE018D569F4F0E94EA72C8017F
:104BD0000E945D72C557DF4F48815981CB58D04044
:104BE000B801CE0189579F4F0E94D36F8091780CF6
:104BF000882399F165EA74E0CE018F579F4F0E9498
:104C0000F272CE018F579F4F0E94AB16CE018F5785
:104C10009F4F0E945D72BE0169577F4FCE018F5733
:104C20009F4F0E94EA72CE018F579F4F0E94AB1692
:104C3000CE018F579F4F0E945D72B801CE018F57F2
:104C40009F4F0E94F272CE018F579F4F0E94AB166A
:104C5000CE018F579F4F0E945D72CC56DF4F8881E7
:104C6000C459D0408F93CD56DF4F8881C359D0406F
:104C70008F93C257DF4F8881CE58D0408F93C35750
:104C8000DF4F8881CD58D0408F9385EB94E09F9380
:104C90008F9380E4E82E8AE0F82EFF92EF920E9434
:104CA000A0A740913502509136026EE07CE08BE087
:104CB00090E10E943B110FB6F894DEBF0FBECDBF4E
:104CC000019709F07CC01F930F938BEB94E09F93A7
:104CD0008F9302E41BE01F930F930E94A0A7B801DB
:104CE0008BE090E10E941A748EE09CE09F938F937A
:104CF0008CEC94E09F938F931F930F930E94A0A737
:104D0000B8018BE090E10E941A746DEC72E08BE0C8
:104D100090E10E94537469EE79E08BE090E10E948B
:104D20004F73F70101900020E9F7CF0181549A40B9
:104D30009F938F9385ED94E09F938F931F930F9391
:104D40000E94A0A7B8018BE090E10E941A74B701FD
:104D50008BE090E10E942C7462E370E080E090E0D0
:104D60000E948A768BE090E10E941C130FB6F894A3
:104D7000DEBF0FBECDBF11E0CE018D569F4F0E940A
:104D80005D72CE0183579F4F0E945D72CE0189579D
:104D90009F4F0E945D72812FC856DF4F0FB6F89467
:104DA000DEBF0FBECDBFDF91CF911F910F91FF905E
:104DB000EF90DF90CF90BF90AF909F90089560E10B
:104DC00073E0CE018F579F4F0E94E272CE018F5742
:104DD0009F4F0E949416CE018F579F4F0E945D7285
:104DE0006CE173E0CE018F579F4F0E94E272CE01BB
:104DF0008F579F4F0E94AB16CE018F579F4F0E9437
:104E00005D7260E47AE0CE018F579F4F0E94F2728C
:104E1000CE018F579F4F0E949416CE018F579F4F00
:104E20000E945D7210E0A8CF8F929F92AF92BF92C6
:104E3000EF92FF920F931F93CF93DF93CDB7DEB71F
:104E40006E970FB6F894DEBF0FBECDBF0091500E27
:104E50001091510E0115110509F4D6C00E94447736
:104E60004B015C0178012EE3E20EF11CF701808119
:104E70009181A281B381A5019401281B390B4A0BB2
:104E80005B0BCA01B901683E33E0730781059105E8
:104E9000A0F128EE33E040E050E00E946EA3861AB5
:104EA000970AA80AB90AD7018D929D92AD92BC9239
:104EB0001397F80186A597A5A0A9B1A949015A01A0
:104EC000880C991CAA1CBB1C88159905AA05BB0552
:104ED00008F0C0C016A617A610AA11AAF80182A948
:104EE00093A9A4A9B5A988159905AA05BB0508F039
:104EF000BAC012AA13AA14AA15AAF80186A597A5E2
:104F0000A0A9B1A9892B8A2B8B2B09F0B5C0EE5B28
:104F1000FF4F8081833009F0AFC084E08083C801F7
:104F2000D7D80196D801D2964D915D916D917C9123
:104F3000D597452B462B472B99F4F801EE5BFF4F95
:104F40002081233011F021110BC01082F8013E9610
:104F500084E1DF011D928A95E9F7C801B9D803966B
:104F60008230910519F0049709F04EC080E590E079
:104F70000E940B0B6091500E7091510E625F7F4F3B
:104F8000CE0101960E947774CE0103960E94030B16
:104F90006091500E7091510E6A5E7F4FCE01019666
:104FA0000E94777444E050E0BE016D5F7F4F81E066
:104FB00090E00E94758D6091500E7091510E6E5E62
:104FC0007F4FCE0101960E94777444E050E0BE010D
:104FD0006D5F7F4F85E090E00E94758D6091500E6F
:104FE0007091510E625E7F4FCE0101960E947774E0
:104FF0008B819C81AD81BE8180934C0E90934D0E30
:10500000A0934E0EB0934F0E60ED77E080E090E0FD
:105010000E948A760E941D8E7C0168EE73E080E01B
:1050200090E00E948A7605E110E0EF28B1F501508A
:10503000110929F160ED77E080E090E00E948A7626
:105040000E941D8E7C0168EE73E080E090E00E947B
:105050008A76EBCF821B930BA40BB50B86A797A781
:10506000A0ABB1AB3BCF821B930BA40BB50B82ABB8
:1050700093ABA4ABB5AB41CF90E080E053CF809130
:10508000670C9091680CA091690CB0916A0C892B07
:105090008A2B8B2B11F0F801199582EF9EE00E946C
:1050A000B3120E94891D65ED78E0CE010D960E9435
:1050B000F27264EF73E0CE0143960E94E272CE0179
:1050C00049960E94B66F8E8D1F928F938D8D1F9281
:1050D0008F938C8D1F928F938B8D1F928F9388E46B
:1050E00094E09F938F9382E49BE09F938F930E9421
:1050F000A0A762E47BE0CE0101960E94F272BE019D
:105100006F5F7F4FCE010D960E942472CE010196F3
:105110000E945D72BE016D5E7F4FCE0101960E94BE
:10512000EA72BE01635F7F4FCE0101960E948471D7
:10513000BC01CE0107960E94EA72CE0107960E943A
:105140009416CE0107960E945D72CE0101960E94D0
:105150005D72BE01635F7F4FCE0101960E94EA72CD
:10516000AE014F5F5F4F63E070E085E892E0BCDC2A
:10517000182FCE0101960E945D720FB6F894DEBF23
:105180000FBECDBF111122C06AEE74E0CE010196B0
:105190000E94F272BE016D5E7F4FCE0101960E94A9
:1051A00084716AED7FE00E948471BC01CE01079694
:1051B0000E94EA72CE0107960E949416CE010796CD
:1051C0000E945D72CE0101960E945D72CE014396EF
:1051D0000E945D72CE010D960E945D726E960FB6B2
:1051E000F894DEBF0FBECDBFDF91CF911F910F911D
:1051F000FF90EF90BF90AF909F908F900895CF92C7
:10520000DF92EF92FF920F931F93CF93DF93CDB76F
:10521000DEB768970FB6F894DEBF0FBECDBF65ED61
:1052200078E0CE0143960E94F27260EC76E0CE0107
:1052300001960E94E272CE0101960E94AB16CE0149
:1052400001960E945D726CA17DA1CE0101960E9423
:105250005A70CE0101960E949416CE0101960E94CA
:105260005D7263EB76E0CE0101960E94E272CE01A0
:1052700001960E94AB16CE0101960E945D727E01DE
:1052800088E2E80EF11C01E010E08CA19DA18017DE
:1052900091070CF1F701619171917F01CE010196A7
:1052A0000E945A70CE0101960E94AB16CE01019663
:1052B0000E945D7262EE75E0CE0101960E94F2726C
:1052C000CE0101960E94AB16CE0101960E945D723E
:1052D0000F5F1F4FDACF62EE75E0CE0101960E949C
:1052E000F272CE0101960E949416CE0101960E94A0
:1052F0005D7264EA76E0CE0101960E94E272CE0110
:1053000001960E94AB16CE0101960E945D726091DB
:10531000D70B7091D80BCE0101960E945A70CE0126
:1053200001960E94AB16CE0101960E945D7262EE5C
:1053300075E0CE0101960E94F272CE0101960E94A4
:10534000AB16CE0101960E945D726091D90B7091EF
:10535000DA0BCE0101960E945A70CE0101960E948E
:105360009416CE0101960E945D726DE876E0CE0142
:1053700001960E94E272CE0101960E94AB16CE0108
:1053800001960E945D72BE01605D7F4FCE01019665
:105390000E94F272CE0101960E94AB16CE010196D8
:1053A0000E945D7262EE75E0CE0101960E94F2727B
:1053B000CE0101960E94AB16CE0101960E945D724D
:1053C000BE016C5C7F4FCE0101960E94F272CE014D
:1053D00001960E949416CE0101960E945D726DE7BF
:1053E00076E0CE0101960E94E272CE0101960E9403
:1053F0009416CE0101960E945D728E010C5D1F4FC6
:10540000EE24E394F12C6801F8E0CF0ED11C8CA1BE
:105410009DA18E159F050CF449C0B701CE010796DA
:105420000E945A706EE877E0CE0101960E94F272F7
:10543000BE01695F7F4FCE0101960E948471BC015D
:10544000CE010D960E94EA72CE010D960E94AB1617
:10545000CE010D960E945D72CE0101960E945D7292
:10546000CE0107960E945D7266EC76E0CE01019651
:105470000E94F272CE0101960E94AB16CE010196F7
:105480000E945D72B801645E7F4FCE0101960E945A
:10549000F272CE0101960E949416CE0101960E94EE
:1054A0005D728FEFE81AF80A8601ADCF63E676E009
:1054B000CE0101960E94E272CE0101960E94AB16C7
:1054C000CE0101960E945D726EE07CE0CE010196F5
:1054D0000E94F272CE0101960E94AB16CE01019697
:1054E0000E945D7261E676E0CE0101960E94E27252
:1054F000CE0101960E94AB16CE0101960E945D720C
:105500006091350270913602CE0101960E945A7068
:10551000CE0101960E949416CE0101960E945D7202
:1055200062E576E0CE0101960E94E272CE0101961C
:105530000E94AB16CE0101960E945D72BE016C5AAC
:105540007F4FCE0101960E94F272CE0101960E9419
:105550009416CE0101960E945D7263EF74E0CE0155
:1055600001960E94F272CE0101960E94AB16CE0106
:1055700001960E945D72BE0164587F4FCE01019674
:105580000E94F272CE0101960E949416CE010196FD
:105590000E945D72C052DF4F88819981C05ED04009
:1055A000892B71F46AE476E0CE0101960E94E272E2
:1055B000CE0101960E949416CE0101960E945D7262
:1055C000C052DF4F88819981C05ED040019771F44D
:1055D00060E476E0CE0101960E94E272CE0101966F
:1055E0000E949416CE0101960E945D72C052DF4F58
:1055F00088819981C05ED040029771F467E376E0BC
:10560000CE0101960E94E272CE0101960E9494168C
:10561000CE0101960E945D7261E376E0CE010196B3
:105620000E94E272CE0101960E94AB16CE01019655
:105630000E945D72CE51DF4F68817981C25ED04099
:10564000CE0101960E945A70CE0101960E949416D6
:10565000CE0101960E945D7240915F0C5091600CEA
:105660006091610C7091620C21E0CE0107960E945E
:1056700062726EEF74E0CE0101960E94F272BE017A
:10568000695F7F4FCE0101960E94847168E075E0EA
:105690000E947071BC01CE010D960E94EA72CE018B
:1056A0000D960E949416CE010D960E945D72CE0159
:1056B00001960E945D72CE0107960E945D72409134
:1056C0005B0C50915C0C60915D0C70915E0C21E064
:1056D000CE0107960E9462726DE075E0CE010196E0
:1056E0000E94F272BE01695F7F4FCE0101960E9457
:1056F000847168E075E00E947071BC01CE010D9666
:105700000E94EA72CE010D960E949416CE010D966B
:105710000E945D72CE0101960E945D72CE010796D5
:105720000E945D7264E176E0CE0101960E94E27211
:10573000CE0101960E94AB16CE0101960E945D72C9
:105740004091200250912102609122027091230227
:1057500025E0CE0101960E946272CE0101960E9460
:105760009416CE0101960E945D726AEF75E0CE013B
:1057700001960E94E272CE0101960E94AB16CE0104
:1057800001960E945D7240911C0250911D02609131
:105790001E0270911F0225E0CE0101960E946272E6
:1057A000CE0101960E949416CE0101960E945D7270
:1057B0006AEE75E0CE0101960E94E272CE0101967A
:1057C0000E94AB16CE0101960E945D726091AA0202
:1057D0007091AB02CE0101960E945A70CE010196E3
:1057E0000E949416CE0101960E945D7268ED75E0EC
:1057F000CE0101960E94E272CE0101960E94AB1684
:10580000CE0101960E945D72C65BDE4F6881798190
:10581000CA54D140CE0101960E945A70CE01019621
:105820000E949416CE0101960E945D72CE014396AD
:105830000E945D7268960FB6F894DEBF0FBECDBFB2
:10584000DF91CF911F910F91FF90EF90DF90CF905C
:1058500008952F923F924F925F926F927F928F9214
:105860009F92AF92BF92CF92DF92EF92FF920F93EF
:105870001F93CF93DF93CDB7DEB7EC970FB6F894B5
:10588000DEBF0FBECDBF9CA78BA71B0170E060E001
:105890000E942471182F65ED78E0CE0149960E9490
:1058A000F2722091AA023091AB022130310509F049
:1058B00091C088E090E090931B0280931A0289E0E7
:1058C00090E090931902809318028091D50B9091EB
:1058D000D60B9093D40B8093D30B809114029091AC
:1058E0001502A0911602B0911702809310029093B6
:1058F0001102A0931202B093130280912C02909196
:105900002D02A0912E02B0912F028093300290932D
:105910003102A0933202B09333028091D20B809374
:10592000D10B8091CD0B9091CE0BA091CF0BB0916C
:10593000D00B8093C90B9093CA0BA093CB0BB09361
:10594000CC0B8AE390E090930F0280930E0280913B
:105950005F0C9091600CA091610CB091620C8093EF
:105960000A0C90930B0CA0930C0CB0930D0C80912F
:105970000C0290910D0290930B0280930A02809189
:10598000200290912102A0912202B09123028093E3
:10599000240290932502A0932602B0932702133588
:1059A00009F08AC01092D40B1092D30B8091DB0BBC
:1059B000882371F064E175E0CE0101960E94F272D5
:1059C000CE0101960E949416CE0101960E945D724E
:1059D000E12C5AC12230310511F78AE090E0909312
:1059E0001B0280931A028BE090E09093190280933F
:1059F00018028091C70B9091C80B9093D40B8093A1
:105A0000D30B8091060290910702A0910802B091F9
:105A100009028093100290931102A0931202B09396
:105A200013028091280290912902A0912A02B0913C
:105A30002B028093300290933102A0933202B093F4
:105A400033028091C60B8093D10B8091C20B909151
:105A5000C30BA091C40BB091C50B8093C90B90935D
:105A6000CA0BA093CB0BB093CC0B8BE390E090933D
:105A70000F0280930E0280915B0C90915C0CA091C0
:105A80005D0CB0915E0C80930A0C90930B0CA0936C
:105A90000C0CB0930D0C8091040290910502909330
:105AA0000B0280930A0280911C0290911D02A0912A
:105AB0001E02B0911F026BCFC1010197029708F03F
:105AC00003C281E090E0A0E0B0E0809310029093E8
:105AD0001102A0931202B0931302ABA5BCA51496B9
:105AE0008D919C911597029750F141E050E0BD01D6
:105AF000CE0101960E94F307BE016F5F7F4FCE017A
:105B000049960E942472CE0101960E945D72CE01D8
:105B10004996B1E02B16310479F50E94B17020E06E
:105B200030E040E251E40E9495A20E9498A4609364
:105B3000100270931102809312029093130281E07D
:105B400090E09093D40B8093D30B113401F58091A6
:105B5000DB0B882309F43CCF69E175E0CE010196A7
:105B60000E94F272CE0101960E949416CE01019617
:105B70000E945D72E12C55C00E94B17020912402F8
:105B8000309125024091260250912702CCCF163445
:105B900009F055C161E080911A020E94437564E6E4
:105BA00070E080E090E00E948A7661E080911A02C5
:105BB0000E94437564E670E080E090E00E948A767F
:105BC000E2E02E163104C1F4CE0149960E94B17074
:105BD0009B01AC0160910A0C70910B0C80910C0C34
:105BE00090910D0C0E94CBA360930A0C70930B0C48
:105BF00080930C0C90930D0C8091DB0B882371F03B
:105C000062E275E0CE0101960E94F272CE01019629
:105C10000E94AB16CE0101960E945D72EE24E394C1
:105C2000F12C8091DB0B882379F140911002509187
:105C3000110260911202709113022AE0CE010196C6
:105C40000E949672BE016F5F7F4FCE0107960E9441
:105C5000EA7266E375E0CE0107960E947071BC019E
:105C6000CE010D960E94EA72CE010D960E94941606
:105C7000CE010D960E945D72CE0107960E945D7264
:105C8000CE0101960E945D728091100290911102E6
:105C9000A0911202B0911302181619061A061B06DB
:105CA0000CF0E0C5163409F4E6C4123509F4E7C473
:105CB0006E2D80911A020E94437564E670E080E0C8
:105CC00090E00E948A766091D30B809118020E9426
:105CD000437561E070E080E090E00E948A7660E0C9
:105CE000809118020E94437568EC70E080E090E0BB
:105CF0000E948A76C12CD12C7601C3948091100227
:105D000090911102A0911202B0911302C816D90607
:105D1000EA06FB060CF0B5C46091D30B8091180223
:105D20000E94437561E070E080E090E00E948A7616
:105D300060E0809118020E9443756091300270917A
:105D4000310280913202909133020E948A768091D2
:105D5000300290913102A0913202B09133020B9740
:105D6000A105B1050CF465C0609124027091250273
:105D700080912602909127029B01AC010E94CCA346
:105D80000E9498A49B01AC01C701B6010E9490A398
:105D9000672B682B692B09F04CC032E023163104C5
:105DA0000CF447C061E074E08FE89FE00E94EC7162
:105DB000C701B6010E9436A220912402309125022B
:105DC00040912602509127020E9430A4AB01BC01F1
:105DD00020E0CE0107960E9462726FE87FE0CE015C
:105DE00001960E94EA72BE01695F7F4FCE01019663
:105DF0000E94847168E075E00E947071BC018FE8B8
:105E00009FE00E940F72CE0101960E945D72CE014A
:105E100007960E945D726FE87FE0CE0101960E94B6
:105E2000EA72CE0101960E94C61DCE0101960E9423
:105E30005D724FEFC41AD40AE40AF40A5FCF123538
:105E400009F098CE60E080911A020E94437564E6E2
:105E500070E080E090E00E948A7660E080911A0213
:105E60000E94437564E670E080E090E00E948A76CC
:105E7000F2E02F163104C1F4CE0149960E94B170B0
:105E80009B01AC0160910A0C70910B0C80910C0C81
:105E900090910D0C0E94CCA360930A0C70930B0C94
:105EA00080930C0C90930D0C8091DB0B882309F4EC
:105EB0008FCD6CE275E0CE0101960E94F272CE01A8
:105EC00001960E94AB1652CE2114310429F043E012
:105ED0002416310409F07CCD80E197E2A0E0B0E027
:105EE0002130310521F480E49CE9A0E0B0E08FA7E7
:105EF00098ABA9ABBAAB81E090E09093D40B8093C0
:105F0000D30B909368028093670280915011909117
:105F100051112230310521F4909368028093670279
:105F2000A0916702B0916802BEA7ADA70B2F001F1A
:105F30000027001F919581959109909351118093AD
:105F4000501181E090E09093680280936702602F87
:105F500080911A020E94437564E670E080E090E050
:105F60000E948A76602F80911A020E94437564E62F
:105F700070E080E090E00E948A768FEF9FEF909330
:105F80000B0280930A02812C912C54011FA218A6A7
:105F900019A61AA61BA21CA21DA21EA21F8E18A221
:105FA00019A21AA2412C512C320119AE1AAE1BAE05
:105FB0001CAE1DAA1EAA1FAA18AE61E0809118028D
:105FC0000E94437561E070E080E090E00E948A7674
:105FD00060E0809118020E94437561E070E080E00B
:105FE00090E00E948A76C501B40123E030E040E0F1
:105FF00050E00E9490A3672B682B692B09F0F8C032
:1060000043E050E05CAB4BABC12CD12C76018091CE
:106010000E02863308F0865320917B00982F9870EB
:10602000277F922B90937B008770806480937C0005
:1060300080917A00806480937A0080917A0086FD56
:10604000FCCF8091780060917900762F682F072E21
:10605000000C880B990B0E9436A29B01AC01C70172
:10606000B6010E94CCA36B017C0162E070E080E08D
:1060700090E00E948A768BA99CA901979CAB8BAB80
:10608000892B29F620E030ED4FE355E4C701B60136
:106090000E9430A46B017C018091DB0B882399F175
:1060A0002DEC3CEC4CE45EE3C701B6010E94C9A4B0
:1060B00087FD29C022E0B701A601CE0107960E9404
:1060C00062726DE375E0CE0101960E94F272BE012C
:1060D000695F7F4FCE0101960E948471BC01CE01A1
:1060E0000D960E94EA72CE010D960E949416CE0182
:1060F0000D960E945D72CE0101960E945D72CE01E6
:1061000007960E945D722AE939E949E95EE3C70111
:10611000B6010E94C9A487FD13C041145104610453
:10612000710411F4240135012BA13CA14DA15EA104
:10613000232B242B252B21F48BA29CA2ADA2BEA243
:106140002DEC3CEC4CE45EE3C701B6010E9430A2AA
:1061500018160CF448C0411451046104710409F488
:1061600047C08F8D98A1A9A1BAA1892B8A2B8B2B0F
:1061700069F42FA138A549A55AA5232B242B252B3B
:1061800009F402C18F8E98A2A9A2BAA28F8D98A1FC
:10619000A9A1BAA1481659066A067B064CF580915A
:1061A0000A0290910B0297FFF4C010920B0210921A
:1061B0000A022F8D38A149A15AA1420E531E641E16
:1061C000751ED301C201B595A7959795879589AF9F
:1061D0009AAFABAFBCAF1F8E18A219A21AA2412C66
:1061E000512C320105C0411451046104710471F64F
:1061F000E0900A02F0900B0292E0E916F1043CF400
:10620000F7FCE3C0A3E02A16310409F0DEC08FA436
:1062100098A8A9A8BAA8BAE08B0E911CA11CB11C21
:106220002FA538A949A95AA982169306A406B5062E
:106230000CF4C3CEF2E0EF16F1040CF479C06DA9B2
:106240007EA98FA998AD29AD3AAD4BAD5CAD621B6F
:10625000730B840B950B0E9436A24B015C01B701B6
:10626000FF0C880B990B0E9436A29B01AC01C50163
:10627000B4010E9430A420E030E044EB53E40E94DB
:1062800030A46B017C01C0922402D0922502E092DE
:106290002602F092270220E030E040E85FE30E940F
:1062A000C9A487FDACC08091AA029091AB02813055
:1062B000910509F090C0C0924811D0924911E09226
:1062C0004A11F0924B11C0922002D0922102E0922A
:1062D0002202F092230264E274E0CE0101960E9451
:1062E000E272CE0101960E94AB16CE0101960E9489
:1062F0005D724091240250912502609126027091B6
:10630000270225E0CE0101960E946272CE0101961D
:106310000E949416CE0101960E945D7284EF91E076
:1063200090939B0280939A026AE270E10E94B20706
:1063300033E02316310429F0E02E2114310409F052
:10634000A3CC8BA59CA50E94B1706B017C01C0926F
:106350000A0CD0920B0CE0920C0CF0920D0C20E089
:1063600030E044EB53E4C701B6010E94C9A487FDA5
:106370006AC020E030E044EB53E4C701B6010E945C
:10638000CBA36B017C01EBCF8FA298A6A9A6BAA6DE
:10639000F9CE2114310409F02BCF019690930B0212
:1063A00080930A022F8D38A149A15AA1420E531E93
:1063B000641E751ED301C201B595A7959795879563
:1063C0008DAB9EABAFABB8AF06CFEFEF8E1A9E0A88
:1063D000AE0ABE0A25CF029709F07DCFC0924C11BC
:1063E000D0924D11E0924E11F0924F11C0921C02CA
:1063F000D0921D02E0921E02F0921F026CCF68E064
:1064000074E0CE0101960E94E272CE0101960E94D4
:10641000AB16CE0101960E945D724091240250910C
:106420002502609126027091270225E0CE01019697
:106430000E946272CE0101960E949416CE010196CE
:106440000E945D7275CF20E030E0A901C701B6015E
:106450000E9430A287FF0BC020E030E044EB53E401
:10646000C701B6010E94CCA36B017C01ECCFC092A6
:10647000C90BD092CA0BE092CB0BF092CC0B4FA081
:1064800058A469A47AA48BA19CA1ADA1BEA1481A6D
:10649000590A6A0A7B0A21143104D9F41092C90BF3
:1064A0001092CA0B1092CB0B1092CC0BADA5BEA5CF
:1064B000812C912C54018394C12CD12C7601B7FFEF
:1064C00026C0C12CD12C760188248A94982C5401A2
:1064D0001EC0EDA5FEA5812C912C54018394F7FFDD
:1064E00004C088248A94982C5401C090C90BD09081
:1064F000CA0BE090CB0BF090CC0B20E030E044E3F3
:1065000053E4C701B6010E9430A287FF93C0C701C0
:10651000B601905820912402309125024091260224
:10652000509127020E9495A26B017C01A301920168
:10653000C501B4010E945FA30E9436A220E030E0B2
:1065400040E05FE30E9495A29B01AC01C701B60148
:106550000E94CBA30E9498A4609310027093110232
:1065600080931202909313028091DB0B882309F42D
:1065700041C02AE04FA158A569A57AA5CE010D9684
:106580000E9496722AE04BA15CA16DA17EA1CE0172
:1065900007960E94967264E475E0CE0101960E940F
:1065A000F272BE01695F7F4FCE0101960E94847135
:1065B00062EE75E00E947071BE01635F7F4F0E94C2
:1065C0008471BC01CE0143960E94EA72CE014396CB
:1065D0000E949416CE0143960E945D72CE010196F0
:1065E0000E945D72CE0107960E945D72CE010D96EB
:1065F0000E945D728091100290911102A09112028E
:10660000B0911302E12C12E5B7FF3ECBB095A095F7
:10661000909581959F4FAF4FBF4F809310029093FD
:106620001102A0931202B0931302EE24E394F12C12
:1066300016E42ACB209124023091250240912602B3
:10664000509127022F8F38A349A35AA3A70196017F
:1066500060E070E084EB93E40E94CBA36093C90BED
:106660007093CA0B8093CB0B9093CC0B2F8D38A1DA
:1066700049A15AA157CFEE24E394F12C19CBE12C78
:1066800017CB52E02516310424F42114310409F00B
:10669000E1C061E080E00E94457982E02816310483
:1066A00024F42114310409F09CC0C0900A0CD0904D
:1066B0000B0CE0900C0CF0900D0C20E030E044EB63
:1066C00053E4C701B6010E94C9A487FD0BC020E0B6
:1066D00030E044EB53E4C701B6010E94CBA36B0149
:1066E0007C01EBCF20E030E0A901C701B6010E9498
:1066F00030A287FF0BC020E030E044EB53E4C70139
:10670000B6010E94CCA36B017C01ECCFC0920A0CB5
:10671000D0920B0CE0920C0CF0920D0C8091AA021E
:106720009091AB020197B1F46EEF74E08FE89FE0B7
:106730000E94517080910A0C90910B0CA0910C0C4E
:10674000B0910D0C80935F0C9093600CA093610C42
:10675000B093620C8091AA029091AB020297B1F4BF
:106760006DE075E08FE89FE00E94517080910A0C07
:1067700090910B0CA0910C0CB0910D0C80935B0CC4
:1067800090935C0CA0935D0CB0935E0C40910A0C4E
:1067900050910B0C60910C0C70910D0C20E0CE010F
:1067A00007960E9462726FE87FE0CE0101960E9418
:1067B000EA72BE01695F7F4FCE0101960E9484712B
:1067C00069E075E00E947071BC018FE89FE00E9453
:1067D0000F72CE0101960E945D72CE0107960E9453
:1067E0005D7291E02916310439F540911002509103
:1067F0001102609112027091130221E0CE010796FE
:106800000E9496726CE475E0CE0101960E94F272CD
:10681000BE01695F7F4FCE0101960E948471BC0169
:106820008FE89FE00E940F72CE0101960E945D7278
:10683000CE0107960E945D726FE87FE0CE0101965F
:106840000E94EA72CE0101960E94C61DCE010196F9
:106850000E945D72109210021092110210921202A8
:10686000109213028091AA029091AB02813091059F
:1068700009F083C08091D30B9091D40B9093D60BE9
:106880008093D50B8091100290911102A091120279
:10689000B09113028093140290931502A0931602F4
:1068A000B09317028091300290913102A091320290
:1068B000B091330280932C0290932D02A0932E026C
:1068C000B0932F028091D10B8093D20B8091C90B92
:1068D0009091CA0BA091CB0BB091CC0B8093CD0BB8
:1068E0009093CE0BA093CF0BB093D00B80910A0C5A
:1068F00090910B0CA0910C0CB0910D0C80935F0C3F
:106900009093600CA093610CB093620C80910A028A
:1069100090910B0290930D0280930C02232881F436
:106920008091240290912502A0912602B091270225
:106930008093200290932102A0932202B09323021D
:10694000CE0149960E945D72EC960FB6F894DEBFB8
:106950000FBECDBFDF91CF911F910F91FF90EF90B0
:10696000DF90CF90BF90AF909F908F907F906F906F
:106970005F904F903F902F900895029709F7809174
:10698000D30B9091D40B9093C80B8093C70B80913D
:10699000100290911102A0911202B0911302809303
:1069A000060290930702A0930802B0930902809117
:1069B000300290913102A0913202B0913302809363
:1069C000280290932902A0932A02B0932B0280916F
:1069D000D10B8093C60B8091C90B9091CA0BA091EB
:1069E000CB0BB091CC0B8093C20B9093C30BA093B5
:1069F000C40BB093C50B80910A0C90910B0CA09125
:106A00000C0CB0910D0C80935B0C90935C0CA093DC
:106A10005D0CB0935E0C80910A0290910B029093F2
:106A2000050280930402232809F08ACF8091240272
:106A300090912502A0912602B091270280931C021A
:106A400090931D02A0931E02B0931F0279CF4F9224
:106A50005F926F927F928F929F92AF92BF92CF92EE
:106A6000DF92EF92FF920F931F93CF93DF93CDB7F7
:106A7000DEB7ED970FB6F894DEBF0FBECDBF67EA65
:106A80007FE0CE01C4960E94EA720CA91DA90115EF
:106A9000110571F0F80181918F01882349F0082ECA
:106AA000000C990B0E9418A7F80131978083F2CF50
:106AB00063E575E0CE0101960E94F272BE016F5F40
:106AC0007F4FCE01C4960E945571182FCE010196BA
:106AD0000E945D72112309F4FFC045E050E067EAAF
:106AE0007FE0CE0101960E94F307BE016F5F7F4FEA
:106AF00089E89FE00E942472CE0101960E945D7297
:106B000089E89FE00E94C77060E089E89FE00E94EA
:106B1000BE7140918D0F50918E0F62E870E189E84F
:106B20009FE00E94D36F60E474E0CE0101960E9462
:106B3000F272BE016F5F7F4F89E89FE00E9455713E
:106B4000182FCE0101960E945D726AE274E0111165
:106B500002C06FE274E0CE0101960E94F27269E811
:106B60007FE0CE0101960E948471BC0180E891E132
:106B70000E940F72CE0101960E945D7280E891E141
:106B80000E94C77040918411509185114150510964
:106B900060E871E1CE0101960E94F307BE016F5FCC
:106BA0007F4F82E691E10E942472CE0101960E94FD
:106BB0005D7282E691E10E94BC700E9436A29B0148
:106BC000AC010E94CDA4882309F448C060918411CF
:106BD000709185116250710980E891E10E942471E1
:106BE000682FCE0101960E94C272BE016F5F7F4F77
:106BF00082E691E10E942472CE0101960E945D72AC
:106C000060E474E0CE0101960E94F272BE016F5FF3
:106C10007F4F82E691E10E945571182FCE010196B7
:106C20000E945D721123D1F06091841170918511E1
:106C30006350710980E891E10E942471682FCE01B0
:106C400001960E94C272BE016F5F7F4F82E691E1A2
:106C50000E942472CE0101960E945D7284EF91E041
:106C600090939B0280939A026AE270E10E94B207BD
:106C700064E670E080E090E00E948A7680913402C1
:106C8000882371F067EA7FE0CE0101960E94EA72E4
:106C9000CE0101960E94991BCE0101960E945D7261
:106CA000CE01C4960E945D7281E0ED960FB6F89415
:106CB000DEBF0FBECDBFDF91CF911F910F91FF902F
:106CC000EF90DF90CF90BF90AF909F908F907F908C
:106CD0006F905F904F90089569E575E0CE01019641
:106CE0000E94F272BE016F5F7F4FCE01C4960E9478
:106CF0005571182FCE0101960E945D72112309F47F
:106D000047C045E050E067EA7FE0CE0101960E946F
:106D1000F307BE016F5F7F4F89E89FE00E942472F6
:106D2000CE0101960E945D7289E89FE00E94C770C3
:106D300060E089E89FE00E94BE7140918D0F509104
:106D40008E0F6AE570E189E89FE00E94D36F6AE5E3
:106D500070E1CE014C960E94F27262E474E0CE01C2
:106D600001960E94F272BE01645E7F4FCE010196D1
:106D70000E948471BC018AE791E10E940F72CE01EA
:106D800001960E945D72CE014C960E945D7266CFA4
:106D90006FE575E0CE0101960E94F272BE016F5F51
:106DA0007F4FCE01C4960E945571182FCE010196D7
:106DB0000E945D721123E1F043E050E067EA7FE05A
:106DC000CE0101960E94F307BE016F5F7F4F89E8F5
:106DD0009FE00E942472CE0101960E945D7269E8D4
:106DE0007FE0CE0101960E94EA72CE010196CDCFDE
:106DF00063E675E0CE0101960E94F272BE016F5FFC
:106E00007F4FCE01C4960E945571182FCE01019676
:106E10000E945D72112301F144E050E067EA7FE0D7
:106E2000CE0101960E94F307BE016F5F7F4F89E894
:106E30009FE00E942472CE0101960E945D7289E853
:106E40009FE00E94BC707093E9106093E81070930B
:106E500084026093830202CF68E675E0CE0101965A
:106E60000E94F272BE016F5F7F4FCE01C4960E94F6
:106E70005571182FCE0101960E945D72112309F4FD
:106E800049C045E050E067EA7FE0CE0101960E94EC
:106E9000F307BE016F5F7F4F89E89FE00E94247275
:106EA000CE0101960E945D7289E89FE00E94BC704D
:106EB000709345116093441184EF91E090939B028D
:106EC00080939A026AE270E10E94B20764E670E081
:106ED00080E090E00E948A766EE877E0CE0101962D
:106EE0000E94F27267EA7FE0CE0101960E948471EF
:106EF000BC01CE014C960E94EA72CE014C960E94D3
:106F00009416CE014C960E945D72CE0101960E94AD
:106F10005D72B4CE6EE675E0CE0101960E94F2720B
:106F2000BE016F5F7F4FCE01C4960E945571182F2E
:106F3000CE0101960E945D721123E1F044E050E021
:106F400067EA7FE0CE0101960E94F307BE016F5F02
:106F50007F4F89E89FE00E942472CE0101960E9433
:106F60005D7289E89FE00E94BC7070934711609346
:106F70004611A2CF63E775E0CE0101960E94F2723E
:106F8000BE016F5F7F4FCE01C4960E945571182FCE
:106F9000CE0101960E945D721123A1F044E050E001
:106FA00067EA7FE0CE0101960E94F307BE016F5FA2
:106FB0007F4F89E89FE00E942472CE0101960E94D3
:106FC0005D7284CF68E775E0CE0101960E94F2728F
:106FD000BE016F5F7F4FCE01C4960E945571182F7E
:106FE000CE0101960E945D721123A1F047E050E0AE
:106FF00067EA7FE0CE0101960E94F307BE016F5F52
:107000007F4F89E89FE00E942472CE0101960E9482
:107010005D722ECE60E875E0CE0101960E94F2729C
:10702000BE016F5F7F4FCE01C4960E945571182F2D
:10703000CE0101960E945D721111D8CF68E875E00B
:10704000CE0101960E94F272BE016F5F7F4FCE01AA
:10705000C4960E945571182FCE0101960E945D7250
:10706000112321F081E00E94200702CE62E975E041
:10707000CE0101960E94F272BE016F5F7F4FCE017A
:10708000C4960E945571182FCE0101960E945D7220
:10709000112319F00E941427EBCD69E975E0CE01A8
:1070A00001960E94F272BE016F5F7F4FCE01C496BF
:1070B0000E945571182FCE0101960E945D72112316
:1070C00009F454C04AE050E067EA7FE0CE0101963F
:1070D0000E94F307BE016F5F7F4F89E89FE00E9427
:1070E0002472CE0101960E945D7289E89FE00E94A1
:1070F000BC700E949D790E94C1796093670C709367
:10710000680C8093690C90936A0C0E94C17960931B
:107110006B0C70936C0C80936D0C90936E0CCE0185
:107120004C960E94F71D64EA75E0CE0101960E941C
:10713000F272BE01645E7F4FCE0101960E9484719F
:10714000BC01CE0182960E94EA72CE0182960E9414
:107150009416CE0182960E945D72CE0101960E9425
:107160005D72CE014C960E945D7288CD6AE077E038
:10717000CE0101960E94F272BE016F5F7F4FCE0179
:10718000C4960E945571182FCE0101960E945D721F
:10719000112309F46CC045E050E067EA7FE0CE01BE
:1071A00001960E94F307BE016F5F7F4F89E89FE061
:1071B0000E942472CE0101960E945D720E94C179E4
:1071C0006093670C7093680C8093690C90936A0CC1
:1071D00089E89FE00E94BC706093AC027093AD029E
:1071E0008093AE029093AF0260932A1170932B119B
:1071F00080932C1190932D11209129112093770CBD
:10720000672B682B692B11F41092770C84EF91E0B7
:1072100090939B0280939A026AE270E10E94B20707
:1072200064E670E080E090E00E948A7667E778E0AC
:10723000CE0101960E94E272CE0101960E94AB1629
:10724000CE0101960E945D724091AC025091AD0258
:107250006091AE027091AF02CE0101960E948570DE
:10726000CE0101960E949416CE0101967CCF65EB6B
:1072700075E0CE0101960E94F272BE016F5F7F4FF2
:10728000CE01C4960E945571182FCE0101960E941E
:107290005D721123D9F14AE050E067EA7FE0CE0148
:1072A00001960E94F307BE016F5F7F4F89E89FE060
:1072B0000E942472CE0101960E945D7289E89FE0CF
:1072C0000E94BC70613071058105910519F481E05F
:1072D0008093291189E89FE00E94BC70672B682B7E
:1072E000692B11F410922911809129118093770C48
:1072F000882309F4E1CD0E94C1796093670C7093F3
:10730000680C8093690C90936A0CD6CD60EC75E0A4
:10731000CE0101960E94F272BE016F5F7F4FCE01D7
:10732000C4960E945571182FCE0101960E945D727D
:107330001123A1F048E050E067EA7FE0CE0101961A
:107340000E94F307BE016F5F7F4F89E89FE00E94B4
:107350002472CE0101960E945D72BECD69EC75E08B
:10736000CE0101960E94F272BE016F5F7F4FCE0187
:10737000C4960E945571182FCE0101960E945D722D
:10738000112321F145E050E067EA7FE0CE0101964C
:107390000E94F307BE016F5F7F4F89E89FE00E9464
:1073A0002472CE0101960E945D7289E89FE00E94DE
:1073B000BC706130710521F481E08093780C5ECC63
:1073C000672B09F05BCC1092780C58CC6FEC75E011
:1073D000CE0101960E94F272BE016F5F7F4FCE0117
:1073E000C4960E945571182FCE0101960E945D72BD
:1073F000112309F472C066E070E087EA9FE00E9402
:107400002471682FCE0101960E94C272BE016F5F87
:107410007F4F89E89FE00E942472CE0101960E946E
:107420005D7289E89FE00E94C77060E089E89FE094
:107430000E94BE7189E89FE00E94BC706B01CB0185
:10744000181619060CF01ACC2091A8023091A90246
:10745000261737070CF412CC48E050E067EA7FE0CB
:10746000CE0101960E94F307BE016F5F7F4F89E84E
:107470009FE00E942472CE0101960E945D7289E80D
:107480009FE00E94C77080918D0F90918E0F099799
:10749000A8F028E030E050E040E069E87FE0CE016D
:1074A00001960E940673BE016F5F7F4F89E89FE0DF
:1074B0000E942472CE0101960E945D72B601E3E043
:1074C000660F771FEA95E1F7625C7F4E48E050E077
:1074D00089E89FE00E94D36FC1CB63E274E0CE01E4
:1074E0004C960E94F272BE01645E7F4FCE01C4963C
:1074F0000E94557111E0811115C066ED75E0CE0155
:1075000001960E94F272BE016F5F7F4FCE01C4965A
:107510000E94557111E0811101C010E0CE01019669
:107520000E945D72CE014C960E945D72112309F497
:10753000D3C162EE75E0CE014C960E94F2726DED01
:1075400075E0CE0101960E94F272AE01445E5F4F7B
:10755000BE016F5F7F4FCE01C4960E948D9ACE010F
:1075600001960E945D72CE014C960E945D7262EEA1
:1075700075E0CE014C960E94F2726FED75E0CE017F
:1075800001960E94F272AE01445E5F4FBE016F5FD2
:107590007F4FCE01C4960E948D9ACE0101960E9423
:1075A0005D72CE014C960E945D7262EE75E0CE0176
:1075B0004C960E94F27261EE75E0CE0101960E9437
:1075C000F272AE01445E5F4FBE016F5F7F4FCE012E
:1075D000C4960E948D9ACE0101960E945D72CE01E2
:1075E0004C960E945D7265EE75E0CE014C960E944D
:1075F000F27264EE75E0CE0101960E94F272AE0165
:10760000445E5F4FBE016F5F7F4FCE01C4960E9404
:107610008D9ACE0101960E945D72CE014C960E9419
:107620005D7265EE75E0CE014C960E94F27262E3E7
:1076300078E0CE0101960E94F272AE01445E5F4F87
:10764000BE016F5F7F4FCE01C4960E948D9ACE011E
:1076500001960E945D72CE014C960E945D72CE0131
:10766000C4960E94C7700E94C17960934C0C7093BD
:107670004D0C80934E0C90934F0C36E0E32EF12C82
:1076800044E6442E512C612C712C88248394912C37
:107690005701F3E0AF0EB11C88AD99AD0197A81664
:1076A000B90608F0EBCAB701CE01C4960E94247156
:1076B000682FCE014C960E94C272670182E0C80E0C
:1076C000D11C9FEFE91AF90A9601A701BE016C5C73
:1076D0007F4FCE0101960E940673CE0101960E9453
:1076E000BC708B01CE0101960E945D7201301105C4
:1076F00021F400914411109145110330110521F43A
:10770000009146111091471162EE75E0CE0101968D
:107710000E94F272A601BE016F5F7F4FCE01C49638
:107720000E94859B6C01CE0101960E945D7265ED01
:1077300078E0CE0101960E94F2721C141D0424F51B
:107740009601A501BE016C5C7F4FCE0182960E941E
:107750000673BE016E5D7F4FCE0101960E942472BA
:10776000CE0182960E945D72101611061CF1760100
:10777000EFEFEE1AFE0ACE0101960E945D72CE0175
:107780004C960E945D7284CFA501BE016C5C7F4F58
:10779000CE0182960E94F307BE016E5D7F4FCE013F
:1077A00001960E942472CE0182960E945D7210168C
:1077B00011060CF78091A8029091A90280179107F9
:1077C0000CF445C070E060E0CE014C960E9424713C
:1077D000823509F041C0CE0101960E94BC70672B32
:1077E000682B692B39F4F801EE0FFF1FEE55FD4FA2
:1077F00011821082CE0101960E94BC706130710529
:107800008105910521F5F801EE0FFF1FEE55FD4FA3
:1078100091828082000F111F000F111FF801E55A9D
:10782000FD4F80819181A281B381181619061A0635
:107830001B0624F040825182628273820E94C179C9
:10784000015B1D4FF80160837183828393831C1455
:107850001D040CF48CCF8FCF8634F1F4CE01019649
:107860000E94BC70672B682B692B39F4F801EE0F6E
:10787000FF1FE75BFD4F11821082CE0101960E942F
:10788000BC70613071058105910521F6F801EE0F9C
:10789000FF1FE75BFD4FBCCF843481F4CE0101961E
:1078A0000E94BC70000F111F000F111FF801E95C4E
:1078B000FD4F6083718382839383C0CF843539F613
:1078C000CE0101960E94BC70000F111F000F111F06
:1078D000F801E55AFD4FEDCF62E778E0CE01019661
:1078E0000E94E272BE016F5F7F4FCE01C4960E947C
:1078F0005571082FCE0101960E945D72002309F494
:1079000013C144E050E067EA7FE0CE0101960E9497
:10791000F307BE016F5F7F4F89E89FE00E942472EA
:10792000CE0101960E945D7289E89FE00E94C770B7
:1079300060E089E89FE00E94BE7140918D0F5091F8
:107940008E0F6EE07CE089E89FE00E94D36F60EECE
:1079500078E0CE018E960E94F27269E87FE0CE0157
:1079600088960E94EA728CA59DA5892BA9F065EDE9
:1079700078E0CE0182960E94F2728AA99BA9892B97
:1079800009F05CC0CE0188960E94BC706AAFCE013F
:1079900082960E945D7211E0CE0188960E945D720F
:1079A000CE018E960E945D72112309F467C98E0183
:1079B000065C1F4F56E5E52E50E1F52E6E018EE375
:1079C000C80ED11CF80181918F01F70181937F01CD
:1079D0001D8E1C8E1F8E1E8E19A218A24AE0BE019B
:1079E0006F5F7F4F90E00E94479EBE016F5F7F4FA9
:1079F000CE014C960E945170CE014C960E94941676
:107A0000CE014C960E945D72C016D106D9F684EF65
:107A100091E090939B0280939A026AE270E10E9447
:107A2000B20764E670E080E090E00E948A7667E644
:107A300078E0CE0101960E94E27212CC50E040E064
:107A4000BE01625D7F4FCE0188960E94859B8C01AE
:107A5000892B11F40CA51DA565ED78E0CE014C969F
:107A60000E94F2724E01FAE38F0E911C5401F12C28
:107A7000E12C6501C818D9081016110684F5980183
:107A8000A701BE01685D7F4FCE0101960E9406737B
:107A9000BE016F5F7F4FCE014C960E942472CE01D3
:107AA00001960E945D72CE014C960E94BC70F50159
:107AB00061935F017801FFEFEF1AFF0AA701BE0192
:107AC000625D7F4FCE0188960E94859B8C018CA5BC
:107AD0009DA5E816F90668F210E000E0CACF8CA573
:107AE0009DA5E816F906D8F4A701BE01685D7F4F91
:107AF000CE0101960E94F307BE016F5F7F4FCE015A
:107B00004C960E942472CE0101960E945D72CE01B5
:107B10004C960E94BC70FE01EC0DFD1D62AFCE01C3
:107B20004C960E945D7233CF60E678E0CE010196FC
:107B30000E94E272BE016F5F7F4FCE01C4960E9429
:107B40005571182FCE0101960E945D721123E9F143
:107B500046E050E067EA7FE0CE0101960E94F3071D
:107B6000BE016F5F7F4F89E89FE00E942472CE01C3
:107B700001960E945D7289E89FE00E94C770809123
:107B80008D0F90918E0F892B09F478C889E89FE0BA
:107B90000E94BC707093531160935211709336021F
:107BA0006093350284EF91E090939B0280939A0258
:107BB0006AE270E10E94B20764E670E080E090E063
:107BC0000E948A766CE478E034CF67EE75E0CE01EF
:107BD00001960E94F272BE016F5F7F4FCE01C49684
:107BE0000E945571182FCE0101960E945D721123DB
:107BF000A1F06FE378E0CE0101960E94E27264E6A4
:107C000070E0CE0101960E947179CE0101960E942A
:107C10005D72F0E0E0E0199531C86EEE75E0CE01DE
:107C20004C960E94F272BE01645E7F4F87EA9FE02D
:107C30000E94557111E0811115C066EF75E0CE010B
:107C400001960E94F272BE016F5F7F4F87EA9FE04C
:107C50000E94557111E0811101C010E0CE01019622
:107C60000E945D72CE014C960E945D72112389F1D3
:107C70006EEF75E0CE0101960E94F27268E671E146
:107C8000CE0101960E948471BC018FE89FE00E94A2
:107C90000F72CE0101960E945D726EE877E0CE0110
:107CA00001960E94F2726FE87FE0CE0101960E9479
:107CB0008471BC01CE014C960E94EA72CE014C96B2
:107CC0000E949416CE014C960E945D72CE010196E0
:107CD0006BC568E076E0CE014C960E94F272BE0160
:107CE000645E7F4F87EA9FE00E94557111E0811129
:107CF00015C06FE076E0CE0101960E94F272BE01DF
:107D00006F5F7F4F87EA9FE00E94557111E08111FC
:107D100001C010E0CE0101960E945D72CE014C962A
:107D20000E945D72112369F061E378E08FE89FE0C3
:107D30000E94EC716EE671E18FE89FE00E94E671AF
:107D4000ACCF66E176E0CE0101960E94F272BE01F0
:107D50006F5F7F4FCE01C4960E945571182FCE01E0
:107D600001960E945D72112331F00E94EA21109267
:107D700034020C943E366FE176E0CE014C960E94C0
:107D8000F272BE01645E7F4F87EA9FE00E945571E8
:107D900011E0811115C064E276E0CE0101960E94E7
:107DA000F272BE016F5F7F4F87EA9FE00E945571BC
:107DB00011E0811101C010E0CE0101960E945D72B8
:107DC000CE014C960E945D72112309F441C065EE0C
:107DD00075E0CE0101960E94F2724091AB0F509176
:107DE000AC0F8D819E81481B590BBE016F5F7F4F89
:107DF00087EA9FE00E943F9AAC014F5F5F4F67EABE
:107E00007FE0CE014C960E94F307BE01645E7F4F77
:107E100089E89FE00E942472CE014C960E945D7218
:107E2000CE0101960E945D7289E89FE00E94BC70BD
:107E30006115710531F481E08093DE020E94588F54
:107E400096CF6130710509F092CF1092DE02F6CF25
:107E500069E276E0CE0101960E94F272BE016F5F88
:107E60007F4FCE01C4960E945571182FCE01019606
:107E70000E945D72112309F43AC143E050E067EAC1
:107E80007FE0CE0101960E94F307BE016F5F7F4F36
:107E900089E89FE00E942472CE0101960E945D72E3
:107EA00069E87FE0CE0101960E94EA72CE01019658
:107EB0000E94991BCE0101960E945D7284EF91E0B1
:107EC00090939B0280939A0269E87FE0CE0101962D
:107ED0000E94EA7260E0CE0101960E94D171BC015D
:107EE00084E791E10E940F72CE0101960E945D72BB
:107EF00069E87FE0CE0101960E94EA7260E0CE015F
:107F000001960E94D171BC018EE691E10E940F7230
:107F1000CE0101960E945D724091781150917911C5
:107F20006AEE70E184E791E10E94D36F4091721193
:107F30005091731165EF70E18EE691E10E94D36F6D
:107F40006AE270E180919A0290919B020E94B207CE
:107F50006DE276E0CE0101960E94F27269E87FE060
:107F6000CE0101960E948471BC01CE0182960E94CE
:107F7000EA72CE0101960E945D728091E6109091A6
:107F8000E710892B39F4BE016E5D7F4F89EB9CE0D1
:107F90000E94337468EB7BE080E090E00E948A7678
:107FA0008091E6109091E710029709F087C069E888
:107FB0007FE0CE0188960E94EA7265E376E0CE010A
:107FC00001960E94F272CE0101960E94848FCE012A
:107FD00001960E945D7264EF71E080E090E00E9483
:107FE0008A7668E376E0CE0101960E94F272CE01B5
:107FF00001960E94848FCE0101960E945D726CED05
:1080000075E080E090E00E948A7661E476E0CE013F
:1080100001960E94F272CE0101960E94848FCE01D9
:1080200001960E945D7264EF71E080E090E00E9432
:108030008A766FE476E0CE0101960E94F272CE015C
:1080400001960E94848FCE0101960E945D7264EFBA
:1080500071E080E090E00E948A766DE276E0CE01E9
:1080600001960E94F272BE01685D7F4FCE010196BB
:108070000E948471BC01CE014C960E94EA72CE012E
:1080800001960E945D72CE014C960E94C770BE019F
:10809000645E7F4FCE0101960E94EA72CE01019686
:1080A0000E94848FCE0101960E945D72CE014C9693
:1080B0000E945D72CE0188960E945D7268EB7BE043
:1080C00080E090E00E948A766AEE70E1CE0101962F
:1080D0000E94F272CE0101960E94991BCE01019678
:1080E0000E945D7210923402CE0182963CC86DE50A
:1080F00076E0CE0101960E94F272BE016F5F7F4F63
:10810000CE01C4960E945571182FCE0101960E948F
:108110005D72112309F486C044E050E067EA7FE015
:10812000CE0101960E94F307BE016F5F7F4F89E881
:108130009FE00E942472CE0101960E945D7262E669
:1081400076E0CE0101960E94F27269E87FE0CE01EE
:1081500001960E948471BC01CE014C960E94EA7285
:10816000CE0101960E945D728091E6109091E71019
:10817000892B39F4BE01645E7F4F89EB9CE00E943D
:10818000337468E873E180E090E00E948A76809121
:10819000E6109091E710029759F569E676E0CE0176
:1081A00001960E94F27280918D0F90918E0F892B13
:1081B00019F562E776E0CE0101960E945170BE018A
:1081C000645E7F4FCE0182960E94EA72CE01829653
:1081D0000E94848FCE0182960E945D7268E873E1EE
:1081E00080E090E00E948A76CE0101960E945D7246
:1081F000109234020C94B138BE016F5F7F4FCE01F4
:1082000082960E94EA72CE0182960E94848FCE01ED
:1082100082960E945D7260E777E180E090E00E94C4
:108220008A76CDCF6BE776E0CE0101960E94F2729E
:10823000BE016F5F7F4FCE01C4960E945571182F0B
:10824000CE0101960E945D72112309F462C067EAB3
:108250007FE089E89FE00E940F7281E08093340202
:1082600067EA7FE0CE0101960E94EA72CE01019694
:108270000E94991BCE0101960E945D728091E610CA
:108280009091E710029709F169E87FE089EB9CE0A3
:108290000E94337468EB7BE080E090E00E948A7675
:1082A000CE0101960E941D90BE016F5F7F4F87EA4D
:1082B0009FE00E942472CE0101960E945D7260EDE3
:1082C00077E080E090E00E948A768091E6109091BD
:1082D000E710029771F469E87FE0CE0101960E94F1
:1082E000EA72CE0101960E94848FCE0101960E940F
:1082F0005D728091AB0F9091AC0F892B09F437CD53
:108300006EE877E0CE0101960E94F27267EA7FE0A4
:10831000CCCC6FE776E0CE0101960E94F272BE01EE
:108320006F5F7F4FCE01C4960E945571182FCE010A
:1083300001960E945D72112309F492C18091E610AA
:108340009091E710019709F012CD65E876E0CE0133
:1083500088960E94F272BE01685D7F4F89EB9CE0B7
:108360000E9433746CE271E080E090E00E948A76B3
:10837000CE0182960E941D9064E670E080E090E05D
:108380000E948A7610E000E035E0C32ED12C4AE04E
:10839000A42EB12C60E976E0CE0101960E94F27223
:1083A00050E040E0BE016F5F7F4FCE0182960E9499
:1083B000859B7C01CE0101960E945D72A7014F5FF3
:1083C0005F4FBE016E5D7F4FCE0101960E94F307A5
:1083D000BE016F5F7F4FCE0188960E942472CE014E
:1083E00001960E945D728CA59DA5892B09F170E014
:1083F00060E0CE0188960E942471082E000C990B33
:10840000C0970A97A8F462E976E0CE0101960E942F
:10841000F272BE016F5F7F4FCE0188960E94557148
:10842000E82ECE0101960E945D72FF24F394E110C4
:10843000F12C60ED76E0CE0101960E94E27264E1DB
:1084400070E0CE0101960E94A19BCE0101960E9490
:108450005D720F5F1F4F62E370E080E090E00E946A
:108460008A76C801B6010E94DDA40197C1F4CE014D
:1084700001960E94C51B8D819E81892B09F4BBC08A
:10848000BE016F5F7F4F87EA9FE00E940F720E94DC
:108490002735FF24F394CE0101960E945D72CE0130
:1084A00001960E941D90BE016F5F7F4FCE018296A4
:1084B0000E942472CE0101960E945D7262E370E018
:1084C00080E090E00E948A760436110519F0FF20C2
:1084D00009F460CF8091DB0B8823F1F06EE877E040
:1084E000CE014C960E94F272BE01685D7F4FCE01B4
:1084F0004C960E948471BC01CE0101960E94EA72E2
:10850000CE0101960E949416CE0101960E945D72E2
:10851000CE014C960E945D728CA59DA5892B69F0B9
:1085200070E060E0CE0188960E942471082E000C55
:10853000990BC0970A9708F477C06AE976E0CE01F4
:1085400001960E94F272CE0182960E945D72CE0167
:1085500088960E945D728D819E81009709F446C0C5
:10856000E981FA812081222309F440C00797F0F1C4
:1085700068E278E0CE014C960E94E27268EC70E00E
:10858000CE014C960E94A19BCE014C960E945D723A
:10859000BE016F5F7F4FCE014C960E94EA7260ED84
:1085A00077E0CE014C960E947179CE014C960E94E4
:1085B0005D7266EA76E0CE014C960E94F27267EA3E
:1085C0007FE0CE014C960E948471BC01CE01829660
:1085D0000E94EA72CE0182960E949416CE01829683
:1085E0000E945D72CE014C960E945D72CE01019692
:1085F0000E945D72BCCB043111050CF44CCFC80154
:10860000B5010E94DDA4892B09F045CFBE01685D4C
:108610007F4F89EB9CE00E94337468EC70E080E04F
:1086200090E00E948A7637CF62E976E0CE0101962B
:108630000E94F272BE016F5F7F4FCE0188960E944A
:108640005571182FCE0101960E945D72111175CFE0
:10865000BE01685D7F4FCE0101960E94DA7273CF32
:1086600064EB76E0CE0101960E94F272BE016F5F6C
:108670007F4FCE01C4960E945571182FCE010196EE
:108680000E945D72112309F4E8C025E030E044E067
:1086900050E067EA7FE0CE0101960E940673BE01BA
:1086A0006F5F7F4F89E89FE00E942472CE010196A0
:1086B0000E945D7267EA7FE0CE0101960E94EA7235
:1086C000CE0101960E94991BCE0101960E945D7217
:1086D00089E89FE00E94BC706130710509F067C0B5
:1086E0007093E7106093E6106FEF76E0CE0101968D
:1086F0000E94E272CE0101960E94991BCE01019662
:108700000E945D7269EB76E0CE014C960E94F27297
:108710006EE671E1CE014C960E948471BC01CE01DF
:1087200001960E94EA7248EC50E06FEF7FEFCE01B5
:1087300001960E94B517CE0101960E945D72CE018E
:108740004C960E945D720E94229A40E052EC61E0D9
:1087500070E089EB9CE00E94826E84EF91E0909340
:108760009B0280939A026AE270E10E94B20768EC71
:1087700076E0CE014C960E94F27268E671E1CE017D
:108780004C960E948471BC01CE0101960E94EA724F
:1087900060ED77E0CE0101960E947179CE010196DD
:1087A0000E945D72CE014C960E945D72E0CA611516
:1087B0007105D1F51092E7101092E61061EF76E0A6
:1087C000CE0101960E94E272CE0101960E94991B91
:1087D000CE0101960E945D726FEB76E0CE014C9661
:1087E0000E94F2726EE671E1CE014C960E94847195
:1087F000BC01CE0101960E94EA7248EC50E06FEF96
:108800007FEFCE0101960E94B517CE0101960E941E
:108810005D72CE014C960E945D720E94229A40E8E1
:1088200055E260E070E095CF6230710509F09FCAB3
:108830007093E7106093E61060EE76E0CE0101964B
:108840000E94E272CE0101960E94991BCE01019610
:108850000E945D7263EC76E0C1CF6DEC76E0CE01F4
:1088600001960E94F272BE016F5F7F4FCE01C496E7
:108870000E945571182FCE0101960E945D7211233E
:1088800009F441C047E050E067EA7FE0CE0101967D
:108890000E94F307BE016F5F7F4F89E89FE00E944F
:1088A0002472CE0101960E945D7268E976E0CE01E5
:1088B00001960E94F272BE016F5F7F4F89E89FE0D0
:1088C0000E945571182FCE0101960E945D72111100
:1088D0001092760C6AEC74E0CE0101960E94F2725E
:1088E000BE016F5F7F4F89E89FE00E945571182F8E
:1088F000CE0101960E945D72112309F401CD81E041
:108900008093760CFDCC65ED76E0CE0101960E9459
:10891000F272BE016F5F7F4FCE01C4960E94557107
:10892000182FCE0101960E945D72112381F146E05D
:1089300050E067EA7FE0CE0101960E94F307BE0196
:108940006F5F7F4F89E89FE00E942472CE010196FD
:108950000E945D7289E89FE00E94B17060932E11C1
:1089600070932F11809330119093311184EF91E027
:1089700090939B0280939A026AE270E10E94B20790
:1089800064E670E080E090E00E948A76B9CC6CEDFD
:1089900076E0CE0101960E94F272BE016F5F7F4FBA
:1089A000CE01C4960E945571182FCE0101960E94E7
:1089B0005D72112301F148E050E067EA7FE0CE01EB
:1089C00001960E94F307BE016F5F7F4F89E89FE029
:1089D0000E942472CE0101960E945D7289E89FE098
:1089E0000E94B170609334117093351180933611E9
:1089F00090933711BBCF65EE76E0CE0101960E94D1
:108A0000F272BE016F5F7F4FCE01C4960E94557116
:108A1000182FCE0101960E945D72112301F149E0E9
:108A200050E067EA7FE0CE0101960E94F307BE01A5
:108A30006F5F7F4F89E89FE00E942472CE0101960C
:108A40000E945D7289E89FE00E94B17060933811C6
:108A50007093391180933A1190933B1187CF6FEE49
:108A600076E0CE0101960E94F272BE016F5F7F4FE9
:108A7000CE01C4960E945571182FCE0101960E9416
:108A80005D721123F1F049E050E067EA7FE0CE012A
:108A900001960E94F307BE016F5F7F4F89E89FE058
:108AA0000E942472CE0101960E945D7289E89FE0C7
:108AB0000E94B1700E9498A470933F1160933E1180
:108AC00055CF69EF76E0CE0101960E94F272BE01A9
:108AD0006F5F7F4FCE01C4960E945571182FCE0153
:108AE00001960E945D721123F1F04AE050E067EABE
:108AF0007FE0CE0101960E94F307BE016F5F7F4FBA
:108B000089E89FE00E942472CE0101960E945D7266
:108B100089E89FE00E94B1700E9498A470933D1173
:108B200060933C1123CF64E077E0CE0101960E9470
:108B3000F272BE016F5F7F4FCE01C4960E945571E5
:108B4000182FCE0101960E945D72112311F14BE0A6
:108B500050E067EA7FE0CE0101960E94F307BE0174
:108B60006F5F7F4F89E89FE00E942472CE010196DB
:108B70000E945D7289E89FE00E94B1700E9498A4F3
:108B8000609340117093411180934211909343116F
:108B9000EDCE60E177E0CE0101960E94F272BE0157
:108BA0006F5F7F4FCE01C4960E945571182FCE0182
:108BB00001960E945D721123E1F045E050E067EA02
:108BC0007FE0CE0101960E94F307BE016F5F7F4FE9
:108BD00089E89FE00E942472CE0101960E945D7296
:108BE00089E89FE00E94BC7070933311609332114A
:108BF000BDCE66E177E0CE0101960E94F272BE0121
:108C00006F5F7F4FCE01C4960E945571182FCE0121
:108C100001960E945D72112359F00E94C179609300
:108C20004C0C70934D0C80934E0C90934F0C9FC83E
:108C30006CE177E0CE0101960E94F272BE016F5F97
:108C40007F4FCE01C4960E945571182FCE01019618
:108C50000E945D72112389F143E050E0BE016C5C1B
:108C60007F4FCE0101960E94F307BE016F5F7F4FD9
:108C700089E89FE00E942472CE0101960E945D72F5
:108C800080918D0F90918E0F892B41F089E89FE0A4
:108C90000E94BC707093AB026093AA028091AA02FA
:108CA0009091AB020197029708F42ACB81E090E003
:108CB0009093AB028093AA0223CB6DEF76E0CE01B6
:108CC0004C960E94F272BE01645E7F4FCE01C49644
:108CD0000E94557111E0811115C063E677E0CE0165
:108CE00001960E94F272BE016F5F7F4FCE01C49663
:108CF0000E94557111E0811101C010E0CE01019672
:108D00000E945D72CE014C960E945D72112309F49F
:108D100068C06DEF76E0CE0101960E94F272BE014E
:108D20006F5F7F4FCE01C4960E945571182FCE0100
:108D300001960E945D721123A1F046E050E0BE0151
:108D40006C5C7F4FCE0101960E94F307BE016F5FFE
:108D50007F4F89E89FE00E942472CE0101960E9415
:108D60005D7263E677E0CE0101960E94F272BE0169
:108D70006F5F7F4FCE01C4960E945571182FCE01B0
:108D800001960E945D721123A1F042E050E0BE0105
:108D90006C5C7F4FCE0101960E94F307BE016F5FAE
:108DA0007F4F89E89FE00E942472CE0101960E94C5
:108DB0005D7280918D0F90918E0F892B09F4A0CA5E
:108DC00069E87FE0CE0101960E94EA7261E070E0FE
:108DD000CE0101960E94292CCE0101960E945D725F
:108DE0008FCA69E277E0CE0182960E94F272BE01DC
:108DF0006E5D7F4FCE01C4960E94557111E08111C6
:108E000029C060E277E0CE014C960E94F272BE016A
:108E1000645E7F4FCE01C4960E94557111E08111AE
:108E200015C068E277E0CE0101960E94F272BE01A1
:108E30006F5F7F4FCE01C4960E94557111E0811182
:108E400001C010E0CE0101960E945D72CE014C96E9
:108E50000E945D72CE0182960E945D72112309F418
:108E6000E6C069E277E0CE0101960E94F272BE018F
:108E70006F5F7F4FCE01C4960E945571182FCE01AF
:108E800001960E945D72112309F466C046E050E02D
:108E9000BE016C5C7F4FCE0101960E94F307BE01BC
:108EA0006F5F7F4F89E89FE00E942472CE01019698
:108EB0000E945D7289E89FE00E94B1706B017C01A5
:108EC00020E030E0A9010E94C9A418160CF08EC061
:108ED000A701960160E070E08AE794E40E9430A464
:108EE0000E9498A460933002709331028093320202
:108EF000909333028091300290913102A09132021E
:108F0000B0913302181619061A061B0664F081E0A8
:108F100090E0A0E0B0E08093300290933102A09303
:108F20003202B09333028091AA029091AB02813059
:108F3000910509F068C08091300290913102A091B2
:108F40003202B091330280932C0290932D02A093B1
:108F50002E02B0932F02D4C947E050E0BE016C5CF2
:108F60007F4FCE0101960E94F307BE016F5F7F4FD6
:108F700089E89FE00E942472CE0101960E945D72F2
:108F80006AE674E0CE0101960E94F272BE016F5F44
:108F90007F4FCE01C4960E945571182FCE010196C5
:108FA0000E945D72112331F081E090E09093AB025A
:108FB0008093AA0266E376E0CE0101960E94F272E7
:108FC000BE016F5F7F4FCE01C4960E945571182F6E
:108FD000CE0101960E945D72112309F46BCF82E0ED
:108FE00090E09093AB028093AA0264CF81E090E07E
:108FF000A0E0B0E08093300290933102A09332025F
:10900000B093330277CF029709F07AC9809130028A
:1090100090913102A0913202B091330280932802E4
:1090200090932902A0932A02B0932B0269C960E3AE
:1090300077E0CE014C960E94F272BE01645E7F4FD3
:10904000CE01C4960E94357111E0811115C065E30F
:1090500077E0CE0101960E94F272BE016F5F7F4FF2
:10906000CE01C4960E94557111E0811101C010E03B
:10907000CE0101960E945D72CE014C960E945D72F7
:10908000112309F469C26EEB77E0CE0101960E94CC
:10909000F272BE016F5F7F4FCE01C4960E94557180
:1090A000182FCE0101960E945D72112309F4E7C0CA
:1090B00001E010E01093AB020093AA021093680243
:1090C000009367026CE377E089E89FE00E945170AB
:1090D000109368020093670269E87FE0CE01019671
:1090E0000E94EA7262E070E0CE0101960E94292C93
:1090F000CE0101960E945D7267E178E0CE01019693
:109100000E94E272CE0101960E949416CE01019651
:109110000E945D7267E078E0CE0101960E94E272E3
:10912000CE0101960E94C61DCE0101960E945D727D
:1091300068E976E089E89FE00E94517069E87FE085
:10914000CE0101960E94EA7263E070E0CE010196C2
:109150000E94292CCE0101960E945D7282E090E06F
:109160009093AB028093AA0266EF77E0CE0101965E
:109170000E94E272CE0101960E949416CE010196E1
:109180000E945D726AEE77E0CE0101960E94E27263
:10919000CE0101960E94C61DCE0101960E945D720D
:1091A0006CE377E089E89FE00E9451708091501154
:1091B0009091511197FF06C060E477E089E89FE045
:1091C0000E94517069E87FE0CE0101960E94EA7228
:1091D00062E070E0CE0101960E94292CCE0101963A
:1091E0000E945D7268E976E089E89FE00E94517014
:1091F00082E090E09093AB028093AA0269E87FE05E
:10920000CE0101960E94EA7263E070E0CE01019601
:109210000E94292CCE0101960E945D7284EF91E09C
:1092200090939B0280939A026AE270E10E94B207D7
:1092300064E670E080E090E00E948A7681E090E051
:109240009093AB028093AA021092A5021092A402FE
:1092500082E090E0A0E0B0E080935F029093600233
:10926000A0936102B09362020E94C179609353029D
:1092700070935402809355029093560241C860E364
:1092800077E0CE0101960E94F272BE016F5F7F4FC0
:10929000CE01C4960E945571182FCE0101960E94EE
:1092A0005D7211112DC86AE674E0CE0101960E942C
:1092B000F272BE016F5F7F4FCE01C4960E9455715E
:1092C000182FCE0101960E945D72112331F081E0CA
:1092D00090E09093AB028093AA0266E376E0CE0121
:1092E00001960E94F272BE016F5F7F4FCE01C4965D
:1092F0000E945571182FCE0101960E945D721123B4
:1093000031F082E090E09093AB028093AA0281E07A
:1093100090E0A0E0B0E08093300290933102A093FF
:109320003202B09333028091AA029091AB02813055
:10933000910509F099C0909368028093670265E3F4
:1093400077E0CE0101960E94F272BE016F5F7F4FFF
:10935000CE01C4960E945571182FCE0101960E942D
:109360005D72112319F146E050E0BE016C5C7F4F45
:10937000CE014C960E94F30764E477E0CE0101969B
:109380000E94F272BE01645E7F4FCE0101960E9480
:109390008471BC0189E89FE00E940F72CE010196A2
:1093A0000E945D72CE014C960E945D7280913002E7
:1093B00090913102A0913202B091330280932C023D
:1093C00090932D02A0932E02B0932F026CE377E0CE
:1093D00089E89FE00E94517069E87FE0CE01019624
:1093E0000E94EA7262E070E0CE0101960E94292C90
:1093F000CE0101960E945D7269ED77E0CE01019683
:109400000E94E272CE0101960E949416CE0101964E
:109410000E945D7281E090E0909368028093670201
:1094200068E976E089E89FE00E94517069E87FE092
:10943000CE0101960E94EA7263E070E0CE010196CF
:109440000E94292CCE0101960E945D7269EC77E0A2
:10945000CE0101960E94E272CE0101960E94C61DC5
:10946000CE0101960E945D728091AA029091AB029A
:10947000029711F00C9480416CE377E089E89FE05B
:109480000E945170809150119091511197FF06C028
:1094900060E477E089E89FE00E94517001E010E00D
:1094A000109368020093670269E87FE0CE0101969D
:1094B0000E94EA7262E070E0CE0101960E94292CBF
:1094C000CE0101960E945D7268E976E089E89FE02E
:1094D0000E94517068EB77E0CE0101960E94E27223
:1094E000CE0101960E949416CE0101960E945D72F3
:1094F00069E87FE0CE0101960E94EA7263E070E0C5
:10950000CE0101960E94292CCE0101960E945D7227
:109510006CEA77E0CE0101960E94E272CE010196DC
:109520000E94C61DCE0101960E945D7284EF91E0FB
:1095300090939B0280939A026AE270E10E94B207C4
:1095400064E670E080E090E00E948A761093AB02BF
:109550000093AA020C94804166E477E0CE018896DD
:109560000E94F272BE01685D7F4FCE01C4960E94D8
:10957000557101E081113DC063E977E0CE0182962B
:109580000E94F272BE016E5D7F4FCE01C4960E94B2
:10959000557101E0811129C062E977E0CE014C9656
:1095A0000E94F272BE01645E7F4FCE01C4960E949B
:1095B000557101E0811115C06DE477E0CE0101968F
:1095C0000E94F272BE016F5F7F4FCE01C4960E946F
:1095D000557101E0811101C000E0CE0101960E94A9
:1095E0005D72CE014C960E945D72CE0182960E9401
:1095F0005D72CE0188960E945D72002309F46AC1F3
:1096000066E477E0CE0101960E94F272BE016F5FC0
:109610007F4FCE01C4960E945571082FCE0101964E
:109620000E945D7246E050E0011117C063E977E0E7
:10963000CE0101960E94F272BE016F5F7F4FCE0194
:10964000C4960E945571082FCE0101960E945D724A
:10965000002309F467C042E050E0BE016C5C7F4F1C
:10966000CE0101960E94F307BE016F5F7F4F89E82C
:109670009FE00E942472CE0101960E945D7280914B
:109680008D0F90918E0F892B11F40C94804164E41E
:1096900077E0CE014C960E94F272BE01645E7F4F6D
:1096A00089E89FE00E945571811114C06AE679E053
:1096B000CE0101960E94F272BE016F5F7F4F89E872
:1096C0009FE00E94557111E0811110E0CE010196DA
:1096D0000E945D72CE014C960E945D72112309F4C6
:1096E000E2C089E89FE00E94B17020910A0C30919D
:1096F0000B0C40910C0C50910D0C0E94CCA36B01F3
:109700007C0120E030E044EB53E40E94C9A487FDD3
:1097100053C020E030E044EB53E4C701B6010E949F
:10972000CBA3EDCF43E050E0BE016C5C7F4FCE0198
:1097300001960E94F307BE016F5F7F4F89E89FE0AB
:109740000E942472CE0101960E945D726AE674E066
:10975000CE0101960E94F272BE016F5F7F4FCE0173
:10976000C4960E945571082FCE0101960E945D7229
:10977000002331F081E090E09093AB028093AA0245
:1097800066E376E0CE0101960E94F272BE016F5F41
:109790007F4FCE01C4960E945571082FCE010196CD
:1097A0000E945D72002309F46ACF82E090E09093FA
:1097B000AB028093AA0263CF20E030E0A901C70189
:1097C000B6010E9430A287FF0BC020E030E044EBDE
:1097D00053E4C701B6010E94CCA36B017C01ECCF1E
:1097E000C0920A0CD0920B0CE0920C0CF0920D0C73
:1097F00089E89FE00E94B17020E030E0A9010E945A
:10980000C9A487FD15C06AE679E0CE0101960E94E1
:10981000F27269E87FE0CE0101960E948471BC017A
:1098200089E89FE00E940F72CE0101960E945D724E
:1098300089E89FE00E94B17020E030E0A9010E9419
:1098400030A287FF30C089E89FE00E94B17020E01D
:1098500030E0A9010E94C9A41816A4F589E89FE088
:109860000E94B170AB01BC0122E0CE014C960E9477
:10987000627264E477E0CE0101960E94F272BE014A
:10988000645E7F4FCE0101960E948471BC0189E81D
:109890009FE00E940F72CE0101960E945D72CE0180
:1098A0004C960E945D7281E090E0909368028093F4
:1098B000670269E87FE0CE0101960E94EA7262E0E9
:1098C00070E086CA89E89FE00E94B170AB01BC01DC
:1098D0007058CACF62E577E0CE0182960E94F2729C
:1098E000BE016E5D7F4FCE01C4960E94557111E09E
:1098F000811129C061E577E0CE014C960E94F27299
:10990000BE01645E7F4FCE01C4960E94557111E086
:10991000811115C068E577E0CE0101960E94F272D0
:10992000BE016F5F7F4FCE01C4960E94557111E05A
:10993000811101C010E0CE0101960E945D72CE013E
:109940004C960E945D72CE0182960E945D72112338
:1099500009F49BC0CE01C4960E94C7706CE377E007
:1099600089E89FE00E9451706AE674E0CE0101969A
:109970000E94F272BE016F5F7F4FCE01C4960E94BB
:109980005571182FCE0101960E945D72112331F09E
:1099900081E090E09093AB028093AA0266E376E0C8
:1099A000CE0101960E94F272BE016F5F7F4FCE0121
:1099B000C4960E945571182FCE0101960E945D72C7
:1099C000112391F082E090E09093AB028093AA0281
:1099D000809150119091511197FF06C060E477E09B
:1099E00089E89FE00E94517081E090E090936802C6
:1099F0008093670269E87FE0CE0101960E94EA72D7
:109A000062E070E0CE0101960E94292CCE01019601
:109A10000E945D7262E577E0CE0101960E94F272CB
:109A2000BE016F5F7F4FCE01C4960E945571182F03
:109A3000CE0101960E945D7245E050E0111102C016
:109A400046E050E0BE016C5C7F4FCE0101960E9463
:109A5000F307BE016F5F7F4F89E89FE00E94247289
:109A6000CE0101960E945D7280918D0F90918E0FB4
:109A7000892B11F40C94804169E87FE0CE010196B6
:109A80000E94EA7263E070E0A3C960E677E0CE016D
:109A900082960E94F272BE016E5D7F4FCE01C49627
:109AA0000E94557111E0811129C06FE577E0CE0168
:109AB0004C960E94F272BE01645E7F4FCE01C49646
:109AC0000E94557111E0811115C066E677E0CE0164
:109AD00001960E94F272BE016F5F7F4FCE01C49665
:109AE0000E94557111E0811101C010E0CE01019674
:109AF0000E945D72CE014C960E945D72CE018296EC
:109B00000E945D72112309F425C160E677E0CE0161
:109B100001960E94F272BE016F5F7F4FCE01C49624
:109B20000E945571182FCE0101960E945D7211237B
:109B300009F443C045E050E0BE016C5C7F4FCE01AC
:109B400001960E94F307BE016F5F7F4F89E89FE097
:109B50000E942472CE0101960E945D7280918D0F49
:109B600090918E0F892B61F089E89FE00E94B1707F
:109B700060930A0C70930B0C80930C0C90930D0C5B
:109B8000C0900A0CD0900B0CE0900C0CF0900D0CD7
:109B900020E030E044EB53E4C701B6010E94C9A4C1
:109BA00087FD55C020E030E044EB53E4C701B60127
:109BB0000E94CBA36B017C01EBCF46E050E0BE01DD
:109BC0006C5C7F4FCE0101960E94F307BE016F5F70
:109BD0007F4F89E89FE00E942472CE0101960E9487
:109BE0005D726AE674E0CE0101960E94F272BE01D7
:109BF0006F5F7F4FCE01C4960E945571182FCE0122
:109C000001960E945D72112331F081E090E0909303
:109C1000AB028093AA0266E376E0CE0101960E9431
:109C2000F272BE016F5F7F4FCE01C4960E945571E4
:109C3000182FCE0101960E945D72112309F48ECF78
:109C400082E090E09093AB028093AA0287CF20E05D
:109C500030E0A901C701B6010E9430A287FF0BC006
:109C600020E030E044EB53E4C701B6010E94CCA3EE
:109C70006B017C01ECCFC0920A0CD0920B0CE092ED
:109C80000C0CF0920D0C8091AA029091AB020197FE
:109C900071F4C0925F0CD092600CE092610CF09273
:109CA000620C6EEF74E08FE89FE00E94517080912B
:109CB0000A0C90910B0CA0910C0CB0910D0C209102
:109CC000AA023091AB022230310571F480935B0C13
:109CD00090935C0CA0935D0CB0935E0C6DE075E00E
:109CE0008FE89FE00E94517040910A0C50910B0C3C
:109CF00060910C0C70910D0C21E0CE014C960E94ED
:109D000062726FE87FE0CE0101960E94EA72BE01A6
:109D1000645E7F4FCE0101960E94847168E075E019
:109D20000E947071BC018FE89FE00E940F72CE010B
:109D300001960E945D72CE014C960E945D726FE8A2
:109D40007FE0CE0101960E94EA72CE0101960E9448
:109D5000C61D42C86EE677E0CE0182960E94F2727E
:109D6000BE016E5D7F4FCE01C4960E94557111E019
:109D7000811129C06DE677E0CE014C960E94F27207
:109D8000BE01645E7F4FCE01C4960E94557111E002
:109D9000811115C063E777E0CE0101960E94F2724F
:109DA000BE016F5F7F4FCE01C4960E94557111E0D6
:109DB000811101C010E0CE0101960E945D72CE01BA
:109DC0004C960E945D72CE0182960E945D721123B4
:109DD00009F412C2C0903002D0903102E0903202F9
:109DE000F090330269E777E0CE0101960E94F272AB
:109DF000BE016F5F7F4FCE01C4960E945571182F30
:109E0000CE0101960E945D72112309F465C044E001
:109E100050E0BE016C5C7F4FCE0101960E94F307BB
:109E2000BE016F5F7F4F89E89FE00E942472CE01E0
:109E300001960E945D728091AA029091AB028130DE
:109E4000910509F093C0C0902C02D0902D02E090B3
:109E50002E02F0902F0281E090E0A0E0B0E080932D
:109E60002C0290932D02A0932E02B0932F0280918A
:109E70008D0F90918E0F892B09F090C06EE777E0DF
:109E800089E89FE00E94517080918D0F90918E0F14
:109E9000892B81F069E87FE0CE0101960E94EA7289
:109EA00070E060E0CE0101960E94292CCE0101965F
:109EB0000E945D728091AA029091AB02813091055F
:109EC00009F08CC1C0922C02D0922D02E0922E0299
:109ED000F0922F020C94804145E050E0BE016C5C92
:109EE0007F4FCE0101960E94F307BE016F5F7F4F47
:109EF00089E89FE00E942472CE0101960E945D7263
:109F00006AE674E0CE0101960E94F272BE016F5FB4
:109F10007F4FCE01C4960E945571182FCE01019635
:109F20000E945D72112331F081E090E09093AB02CA
:109F30008093AA0266E376E0CE0101960E94F27257
:109F4000BE016F5F7F4FCE01C4960E945571182FDE
:109F5000CE0101960E945D72112309F46CCF82E05C
:109F600090E09093AB028093AA0265CF029709F02C
:109F70007ECFC0902802D0902902E0902A02F09073
:109F80002B0281E090E0A0E0B0E080932802909363
:109F90002902A0932A02B0932B0269CF64E877E0EC
:109FA000CE0101960E94F272BE016F5F7F4F89E879
:109FB0009FE00E943571182FCE0101960E945D72BC
:109FC000112309F477CF89E89FE00E94B17020E067
:109FD00030E0A9010E9430A2811128C08091AA021C
:109FE0009091AB02019731F467E877E089E89FE050
:109FF0000E9451708091AA029091AB02029731F4B5
:10A000006EE777E089E89FE00E94517080918D0FA4
:10A0100090918E0F892B09F44DCF69E87FE0CE0136
:10A0200001960E94EA7261E070E03CCF65EE75E057
:10A03000CE0101960E94F272BE016F5F7F4F89E8E8
:10A040009FE00E943571182FCE0101960E945D722B
:10A05000112309F42FCF41E050E069E87FE0CE0101
:10A0600001960E94F307CE0101960E94B1704B0148
:10A070005C01CE0101960E945D7220E030E0A901F2
:10A08000C501B4010E9430A2181634F0812C912C25
:10A0900020E8A22E2FE3B22E0091AA021091AB026B
:10A0A0000130110509F075C0A501940160E070E46C
:10A0B0008CE995E40E9430A46093240270932502F9
:10A0C0008093260290932702609348117093491160
:10A0D00080934A1190934B11609320027093210258
:10A0E0008093220290932302B801CE014C960E94E5
:10A0F0005A706CE877E0CE0101960E94F272BE01C0
:10A10000645E7F4FCE0101960E948471BC01CE0136
:10A1100082960E94EA72CE0182960E94AB16CE0110
:10A1200082960E945D72CE0101960E945D72CE0100
:10A130004C960E945D726AE977E0CE0101960E941A
:10A14000E272CE0101960E94AB16CE0101960E94EA
:10A150005D72409124025091250260912602709117
:10A16000270225E0CE0101960E946272CE0101967F
:10A170000E949416CE0101960E945D7284EF91E0D8
:10A1800090939B0280939A026AE270E10E94B20768
:10A1900091CE0230110509F0A7CFA501940160E02E
:10A1A00070E48CE196E40E9430A4609324027093E2
:10A1B0002502809326029093270260934C1170939E
:10A1C0004D1180934E1190934F1160931C02709328
:10A1D0001D0280931E0290931F0286CF029711F0FA
:10A1E0000C948041C0922802D0922902E0922A0267
:10A1F000F0922B020C94804161E977E0CE018296C7
:10A200000E94F272BE016E5D7F4FCE01C4960E9425
:10A21000557111E0811129C060E977E0CE014C96BB
:10A220000E94F272BE01645E7F4FCE01C4960E940E
:10A23000557111E0811115C066E977E0CE010196F4
:10A240000E94F272BE016F5F7F4FCE01C4960E94E2
:10A25000557111E0811101C010E0CE0101960E94FC
:10A260005D72CE014C960E945D72CE0182960E9474
:10A270005D72112309F429C188AD99AD059710F4D9
:10A280000C94804144E050E0BE016C5C7F4FCE01F5
:10A2900001960E94F307BE016F5F7F4F89E89FE040
:10A2A0000E942472CE0101960E945D7261E977E0FE
:10A2B000CE0101960E94F272BE016F5F7F4FCE0108
:10A2C000C4960E945571182FCE0101960E945D72AE
:10A2D000112309F49BC044E050E0BE016C5C7F4F49
:10A2E000CE0101960E94F307BE016F5F7F4F89E8A0
:10A2F0009FE00E942472CE0101960E945D7289E85F
:10A300009FE00E94B17020E030E0A9010E94C9A442
:10A31000181614F00C94804189E89FE00E94B170F7
:10A320006093240270932502809326029093270263
:10A330002091AA023091AB022130310509F0B0C062
:10A34000609348117093491180934A1190934B1177
:10A350006093200270932102809322029093230243
:10A36000B901CE014C960E945A706CE877E0CE019C
:10A3700001960E94F272BE01645E7F4FCE0101968B
:10A380000E948471BC01CE0182960E94EA72CE01C5
:10A3900082960E94AB16CE0182960E945D72CE011B
:10A3A00001960E945D72CE014C960E945D7268E833
:10A3B00077E0CE0101960E94E272CE0101960E94E2
:10A3C000AB16CE0101960E945D724091240250911D
:10A3D0002502609126027091270225E0CE010196A8
:10A3E0000E946272CE0101960E949416CE010196DF
:10A3F0000E945D7284EF91E090939B0280939A0299
:10A400006AE270E10E94B2070C94804145E050E09E
:10A41000BE016C5C7F4FCE0101960E94F307BE0126
:10A420006F5F7F4F89E89FE00E942472CE01019602
:10A430000E945D726AE674E0CE0101960E94F2729B
:10A44000BE016F5F7F4FCE01C4960E945571182FD9
:10A45000CE0101960E945D72112331F081E090E0FF
:10A460009093AB028093AA0266E376E0CE01019658
:10A470000E94F272BE016F5F7F4FCE01C4960E94B0
:10A480005571182FCE0101960E945D72112309F4B7
:10A4900036CF82E090E09093AB028093AA022FCF58
:10A4A0002230310509F05CCF60934C1170934D114F
:10A4B00080934E1190934F1160931C0270931D0274
:10A4C00080931E0290931F024BCF60E775E0CE0190
:10A4D0004C960E94F272BE01645E7F4FCE01C4961C
:10A4E0000E94557111E0811115C06CE977E0CE0131
:10A4F00001960E94F272BE016F5F7F4FCE01C4963B
:10A500000E94557111E0811101C010E0CE01019649
:10A510000E945D72CE014C960E945D72112309F477
:10A5200063C060E775E0CE0101960E94F272BE0141
:10A530006F5F7F4FCE01C4960E945571182FCE01D8
:10A5400001960E945D72112399F042E050E067EAA3
:10A550007FE0CE0101960E94F307BE016F5F7F4F3F
:10A5600089E89FE00E942472CE0101960E945D72EC
:10A570006CE977E0CE0101960E94F272BE016F5F36
:10A580007F4FCE01C4960E945571182FCE010196BF
:10A590000E945D72112399F043E050E067EA7FE08A
:10A5A000CE0101960E94F307BE016F5F7F4F89E8DD
:10A5B0009FE00E942472CE0101960E945D7289E89C
:10A5C0009FE00E94BC70653B710510F40C948041C3
:10A5D00065E777E0CE0101960E94E272CE01019616
:10A5E0000E94AB160C94EC4660EA77E0CE0101962F
:10A5F0000E94F272BE016F5F7F4FCE01C4960E942F
:10A600005571182FCE0101960E945D72112309F435
:10A610007EC026E030E044E050E067EA7FE0CE0113
:10A6200001960E940673BE016F5F7F4F89E89FE02D
:10A630000E942472CE0101960E945D7265EE75E063
:10A64000CE0101960E94F2724091AB0F5091AC0F77
:10A650008D819E81481B590BBE016F5F7F4F87EA3A
:10A660009FE00E943F9AAC014F5F5F4F67EA7FE037
:10A67000CE014C960E94F307BE01645E7F4F89E8CD
:10A680009FE00E942472CE014C960E945D72CE0122
:10A6900001960E945D7289E89FE00E94B17088E295
:10A6A000E2EEFBE0A1E0B1E101900D928A95E1F7C5
:10A6B00084EF91E090939B0280939A026AE270E1AA
:10A6C0000E94B20764E577E08FE89FE00E94EC719A
:10A6D00044E050E067EA7FE0CE0101960E94F30774
:10A6E000BE016F5F7F4F8FE89FE00E94E671CE0151
:10A6F00001960E945D726FE87FE0CE0101960E9494
:10A70000EA72CE0101960E9494160C94F64264EA15
:10A7100077E0CE0101960E94F272BE016F5F7F4F1B
:10A72000CE01C4960E945571182FCE0101960E9449
:10A730005D7211110C9442446CEA77E0CE010196EF
:10A740000E94F272BE016F5F7F4FCE01C4960E94DD
:10A750005571182FCE0101960E945D72112371F17F
:10A7600041E066EB72E0CE0101960E94DB8ABE01F9
:10A770006F5F7F4F86E891E10E94C21686E891E103
:10A780000E94898A811104C068E077E00C94193D29
:10A7900086E891E10E94396D892B51F086E891E1BC
:10A7A0000E946D84682F86E59DE00E943A6BF0CF91
:10A7B00086E891E10E94958A0C943E3663EB77E03F
:10A7C000CE0101960E94F272BE016F5F7F4FCE01F3
:10A7D000C4960E945571182FCE0101960E945D7299
:10A7E0001123E9F08DB79EB78A5291400FB6F894C5
:10A7F0009EBF0FBE8DBFADB7BEB711968AE291E086
:10A80000EAE2F0E101900D920197E1F70E94FF2842
:10A810000FB6F894DEBF0FBECDBF0C943E366CEB86
:10A8200077E0CE0101960E94F272BE016F5F7F4F0A
:10A83000CE01C4960E945571182FCE0101960E9438
:10A840005D72112309F459C08DB79EB78A529140A9
:10A850000FB6F8949EBF0FBE8DBFADB7BEB71196B1
:10A860008AE291E0EAE2F0E101900D920197E1F7CE
:10A870000E94D1230FB6F894DEBF0FBECDBF63E4B4
:10A8800077E0CE0101960E94E2728DB79EB78A52A0
:10A8900091400FB6F8949EBF0FBE8DBFADB7BEB747
:10A8A00011968AE291E0EAE2F0E101900D920197BF
:10A8B000E1F70E947D190FB6F894DEBF0FBECDBF41
:10A8C0008DB79EB78A5291400FB6F8949EBF0FBEC7
:10A8D0008DBFADB7BEB711968AE291E0EAE2F0E132
:10A8E00001900D920197E1F70E94FF280FB6F894AE
:10A8F000DEBF0FBECDBF0C9434396EEB77E0CE01D6
:10A9000001960E94F272BE016F5F7F4FCE01C49626
:10A910000E945571182FCE0101960E945D7211237D
:10A92000B1F061E377E0CE0101960E94E272BE01D0
:10A930006F5F7F4FCE014C960E94EA72CE014C961B
:10A940000E949416CE014C960E945D72B9CF62ECC3
:10A9500077E0CE0101960E94F272BE016F5F7F4FD9
:10A96000CE01C4960E945571182FCE0101960E9407
:10A970005D72112309F4F5C065E177E0CE0182969E
:10A980000E94E272BE016E5D7F4FCE0101960E9471
:10A99000EA72AE014F5F5F4F62E070E086E792E0DF
:10A9A0000E947425182FCE0101960E945D7211112C
:10A9B00022C0BE016E5D7F4FCE014C960E94EA72AE
:10A9C00066EC77E0CE014C960E9470716AED7FE0F4
:10A9D0000E948471BC01CE0101960E94EA72CE01F0
:10A9E00001960E949416CE0101960E945D72CE01DE
:10A9F0004C960E945D7268EE73E080E090E00E94E9
:10AA00008A76BE016E5D7F4FCE0101960E94EA728A
:10AA1000AE014F5F5F4F63E070E089E692E00E9415
:10AA20007425182FCE0101960E945D72111122C06B
:10AA3000BE016E5D7F4FCE014C960E94EA7266EDBC
:10AA400077E0CE014C960E9470716AED7FE00E9423
:10AA50008471BC01CE0101960E94EA72CE0101967A
:10AA60000E949416CE0101960E945D72CE014C9612
:10AA70000E945D7268EE73E080E090E00E948A764A
:10AA80006EEC7FE0CE0101960E94EA72AE014F5F4C
:10AA90005F4F61E070E080ED92E00E947425182F16
:10AAA000CE0101960E945D72111121C06EEC7FE013
:10AAB000CE014C960E94EA7266ED77E0CE014C968C
:10AAC0000E9470716AED7FE00E948471BC01CE012A
:10AAD00001960E94EA72CE0101960E949416CE0160
:10AAE00001960E945D72CE014C960E945D7268EEE6
:10AAF00073E080E090E00E948A768091760C882353
:10AB000011F40C94744043E160ED72E0CE010196C3
:10AB10000E94DB8ABE016F5F7F4F8CEB91E10E9448
:10AB2000C2168CEB91E10E94898A882311F40C945F
:10AB300074406EEC7FE08CEB91E10E94417466E919
:10AB400070E080E090E00E948A768CEB91E10E94B8
:10AB5000958A62E370E080E090E00E948A760C942F
:10AB6000744062EE77E0CE0101960E94F272BE015F
:10AB70006F5F7F4FCE01C4960E945571182FCE0192
:10AB800001960E945D72112301F19CEDE92E9BE07C
:10AB9000F92E01E010E0F2E0EF0EF11C8091A80226
:10ABA0009091A9028017910714F40C943E3660E04E
:10ABB000F70180810E9443756CE271E080E090E0D3
:10ABC0000E948A760F5F1F4FE6CF66EE77E0CE01D8
:10ABD00001960E94F272BE016F5F7F4FCE01C49654
:10ABE0000E945571182FCE0101960E945D721123AB
:10ABF00001F18CEDE82E8BE0F82E01E010E0F2E0A0
:10AC0000EF0EF11C8091A8029091A9028017910784
:10AC100014F40C943E3661E0F70180810E94437584
:10AC20006CE271E080E090E00E948A760F5F1F4F37
:10AC3000E6CF6BEE77E0CE0101960E94F272BE0184
:10AC40006F5F7F4FCE01C4960E945571182FCE01C1
:10AC500001960E945D72112311F40C943E3627E098
:10AC600030E046E050E067EA7FE0CE0101960E94C6
:10AC70000673BE016F5F7F4F89E89FE00E942472D8
:10AC8000CE0101960E945D7289E89FE00E94BC702F
:10AC9000672B71F41092DB0B67EA7FE0CE0101961F
:10ACA0000E94EA72CE0101960E94991B0C94F64212
:10ACB00081E08093DB0BF0CF4F925F926F927F9297
:10ACC0008F929F92AF92BF92CF92DF92EF92FF92BC
:10ACD0000F931F93CF93DF93CDB7DEB72C970FB6AB
:10ACE000F894DEBF0FBECDBF67E370E080918302B2
:10ACF000909184020E94230884E1482E512C612CFB
:10AD0000712CD12CC12CAFEFCA1ADA0AC301B201DF
:10AD10000E948A76E0908302F090840267E370E0FC
:10AD2000C7010E9423088C01B3E0CB16D10434F094
:10AD30008EE1C816D10444F4012B51F094E1490E80
:10AD4000511C611C711CDFCF0115110509F0AEC04B
:10AD50008BE0E816F10409F08EC0809058119090B5
:10AD60005911A0905A11B0905B118091541190919B
:10AD70005511A0915611B091571189879A87AB87C9
:10AD8000BC8764E670E080E090E00E948A7660EC28
:10AD900073E0CE0101960E94E272CE0101960E94FC
:10ADA000C61DCE0101960E945D7261E082E00E94A4
:10ADB000457921E0B501A401CE0101960E9462729D
:10ADC000BE016F5F7F4F88ED91E10E943374CE0129
:10ADD00001960E945D726FED88ED91E10E942179EC
:10ADE0006BEB73E088ED91E10E94537420E049859C
:10ADF0005A856B857C85CE0101960E946272BE01E8
:10AE00006F5F7F4F88ED91E10E943374CE01019610
:10AE10000E945D7262EF77E088ED91E10E942C74F0
:10AE200089829A82AB82BC8289859A85AB85BC85F2
:10AE30008D839E83AF83B88729813A814B815C8162
:10AE40006D817E818F8198852C960FB6F894DEBF38
:10AE50000FBECDBFDF91CF911F910F91FF90EF906B
:10AE6000DF90CF90BF90AF909F908F907F906F902A
:10AE70005F904F90089596E1E916F10409F46DCFC3
:10AE8000ACE0EA16F10409F07CCF8090040B9090BE
:10AE9000050BA090060BB090070B8091000B9091D2
:10AEA000010BA091020BB091030B67CF0F3F9FEFF7
:10AEB0001907CCF06DEA73E0CE0101960E94E272B0
:10AEC0004AE050E070E060E0CE0101960E94B517C4
:10AED000CE0101960E945D726AE873E08FE89FE000
:10AEE0000E94EC7132C00E3FAFEF1A07B9F16CE768
:10AEF00073E0CE0101960E94E2724AE050E070E0F9
:10AF000060E0CE0101960E94B517CE0101960E9425
:10AF10005D726DE673E08FE89FE00E94EC71B8010E
:10AF2000CE0101960E945A70BE016F5F7F4F8FE87D
:10AF30009FE00E94E671CE0101960E945D7267E576
:10AF400073E08FE89FE00E94957119821A821B823C
:10AF50001C821D821E821F8218866ECF6CE473E0F5
:10AF6000CE0101960E94E2724AE050E070E060E09B
:10AF7000CE0101960E94B517CE0101960E945D7226
:10AF80006CE273E0ABCF2F923F924F925F926F9241
:10AF90007F928F929F92AF92BF92CF92DF92EF9269
:10AFA000FF920F931F93CF93DF93CDB7DEB7AC978C
:10AFB0000FB6F894DEBF0FBECDBF8C017B01809130
:10AFC000590C90915A0C019690935A0C8093590CFD
:10AFD0002091580C222341F06AE070E00E94DDA429
:10AFE000181619060CF4B9C281E08093580C10921F
:10AFF0005A0C1092590C50E040E06AE074E0C8012D
:10B000000E943F1782E0E816F10409F4BFC265ED23
:10B0100078E088EC9FE00E94517067E370E08091D7
:10B020008302909184020E9423081C0165E974E068
:10B03000C8010E94F31664EF77E0C8010E942C74E7
:10B0400062E671E1CE0101960E94EA72BE016F5F75
:10B050007F4FC8010E943374CE0101960E945D7239
:10B060006DEF77E0C8010E942C7460E874E0C801BD
:10B070000E94537468E671E1CE0101960E94EA7263
:10B08000BE016F5F7F4FC8010E94337466E774E0B2
:10B09000C8010E94537462E870E1CE0109960E94D3
:10B0A000F272BE01675F7F4FC8010E94337469E688
:10B0B00074E0C8010E9453746AEE70E1CE010F96ED
:10B0C0000E94F272BE01615F7F4FC8010E9433741B
:10B0D00062E674E0C8010E945374CE010F960E948C
:10B0E0005D72CE0109960E945D72CE0101960E94AA
:10B0F0005D720E94447728EE33E040E050E00E9409
:10B100006EA329013A0168E574E0C8010E945374F6
:10B11000CE0101960E94F71DBE016F5F7F4FC801EF
:10B120000E943374CE0101960E945D72C301B20188
:10B1300020E13EE040E050E00E9490A34B015C0122
:10B14000B901CE0187960E944B184CE3C42ED12C36
:10B15000E12CF12CC501B401A70196010E9490A336
:10B16000B901CE0101960E944B1866EC76E0CE0143
:10B1700009960E94F272BE016F5F7F4FCE01099661
:10B180000E948471BC01CE0187960E94E671CE01B7
:10B1900009960E945D72CE0101960E945D72C30104
:10B1A000B201A70196010E9490A3CE0101960E94D0
:10B1B0004B1866EC76E0CE0109960E94F272BE0151
:10B1C0006F5F7F4FCE0109960E948471BC01CE0152
:10B1D00087960E94E671CE0109960E945D72CE01AB
:10B1E00001960E945D7263E078E0CE0109960E94AC
:10B1F000F272BE01695D7F4FCE0109960E94847193
:10B2000066E078E00E947071BC01CE0101960E9458
:10B21000EA72BE016F5F7F4FC8010E943374CE0196
:10B2200001960E945D72CE0109960E945D7264E1F2
:10B2300078E0C8010E942C74CE0101960E94B66F7E
:10B24000B801CE0101960E94BE736FE078E0C8019C
:10B250000E941A7431DD29833A834B835C836D83AA
:10B260007E838F83988749815A816B817C8121E01D
:10B27000CE010F960E946272BE01615F7F4FCE01C8
:10B2800009960E94EA726CE178E0CE0109960E946C
:10B290007071BC0188EC9FE00E940F72CE0109968C
:10B2A0000E945D72CE010F960E945D7263E278E0AB
:10B2B000CE010F960E94F27268EC7FE0CE010F96ED
:10B2C0000E948471BC01CE0109960E94EA72BE01FF
:10B2D000675F7F4FC8010E943374CE0109960E94B8
:10B2E0005D72CE010F960E945D724D815E816F810D
:10B2F000788521E0CE0109960E946272BE01675FE7
:10B300007F4F88EC9FE00E942472CE0109960E9434
:10B310005D7265E378E0CE010F960E94F27268ECF0
:10B320007FE0CE010F960E94847166E478E00E946F
:10B330007071BC01CE0109960E94EA72BE01675F7E
:10B340007F4FC8010E943374CE0109960E945D723E
:10B35000CE010F960E945D7240915F0C5091600C7F
:10B360006091610C7091620C22E0CE010F960E94F8
:10B3700062726DE478E0CE0145960E94F272BE01E1
:10B38000615F7F4FCE0145960E9484716FE578E042
:10B390000E947071BC01CE0109960E94EA72BE0142
:10B3A000675F7F4FC8010E943374CE0109960E94E7
:10B3B0005D72CE0145960E945D72CE010F960E948D
:10B3C0005D7240915B0C50915C0C60915D0C7091D2
:10B3D0005E0C22E0CE010F960E94627268E678E071
:10B3E000CE0145960E94F272BE01615F7F4FCE0191
:10B3F00045960E9484716FE578E00E947071BC01EF
:10B40000CE0109960E94EA72BE01675F7F4FC801B4
:10B410000E943374CE0109960E945D72CE0145965A
:10B420000E945D72CE010F960E945D72E6EF2E16AD
:10B43000EFEF3E062CF466E875E0C8010E94F316B3
:10B4400068E374E0C8010E94F31622EAC22E22E0EB
:10B45000D22EEE24E394F12CF2E0CF0ED11C809199
:10B46000A8029091A9028E159F050CF468C0B7013F
:10B47000CE010F960E945A706EE877E0CE01459695
:10B480000E94F272BE01615F7F4FCE0145960E941D
:10B49000847162EE75E00E947071BC01CE01099664
:10B4A0000E94EA72BE01675F7F4FC8010E94337439
:10B4B000B70183E0660F771F8A95E1F7625C7F4EE4
:10B4C000CE014B960E94F272BE01655E7F4FC801AD
:10B4D0000E94337466E778E0C8010E942C74F6017C
:10B4E00060817181660F771F660F771F6A5C7F4EE0
:10B4F000CE0181960E94F272BE016F5D7F4FC8013E
:10B500000E9433746BE778E0C8010E942C74CE016E
:10B5100081960E945D72CE014B960E945D72CE01B3
:10B5200009960E945D72CE0145960E945D72CE0121
:10B530000F960E945D72FFEFEF1AFF0A8DCFCE01CA
:10B5400087960E945D7281E08093790C6CE475E0CF
:10B55000C8010E94F3161092580CAC960FB6F894DE
:10B56000DEBF0FBECDBFDF91CF911F910F91FF9036
:10B57000EF90DF90CF90BF90AF909F908F907F9093
:10B580006F905F904F903F902F90089566E875E020
:10B59000C8010E94F316DACFAF92BF92CF92DF922A
:10B5A000EF92FF920F931F93CF93DF93CDB7DEB748
:10B5B000A0970FB6F894DEBF0FBECDBF65ED78E063
:10B5C00082EF9FE00E94517065ED78E086EE9FE08B
:10B5D0000E94517053E4E52E52E0F52E62EAC62E29
:10B5E00062E0D62E7BE3A72E72E0B72E01E010E0DA
:10B5F0008091A8029091A902801791070CF482C053
:10B60000F50181919191A191B1915F01892B8A2BD3
:10B610008B2B19F5F60182819381F7012281338109
:10B6200082179307D1F0880F991FFC01E952F44F5C
:10B63000D801AA0FBB1FA452B44F60818C910E9405
:10B640004375F60182819381F7019383828364E6D7
:10B6500070E080E090E00E948A76F7016281738159
:10B66000CE0145960E945A70B801CE010F960E94F5
:10B670005A70B80123E0660F771F2A95E1F7625CE4
:10B680007F4ECE0109960E94F27262EE75E0CE0105
:10B6900001960E94F272BE01675F7F4FCE01019654
:10B6A0000E94847160E878E00E947071BE01615F61
:10B6B0007F4F0E94847165EE75E00E947071BE013B
:10B6C0006B5E7F4F0E948471BC0182EF9FE00E94FD
:10B6D000E671CE0101960E945D72CE0109960E942C
:10B6E0005D72CE010F960E945D72CE0145960E945A
:10B6F0005D720F5F1F4FF2E0EF0EF11C22E0C20EF1
:10B70000D11C76CFE0914411F0914511EE0FFF1F4F
:10B71000ED5BFD4F60817181CE0101960E945A70F0
:10B7200046E050E0BE016F5F7F4FCE0109960E9458
:10B730006E17BE01675F7F4F86EE9FE00E94E67145
:10B74000CE0109960E945D72CE0101960E945D7243
:10B75000E0914611F0914711EE0FFF1FED5BFD4F99
:10B7600060817181CE0101960E945A7046E050E0DE
:10B77000BE016F5F7F4FCE0109960E946E17BE011A
:10B78000675F7F4F86EE9FE00E94E671CE010996CB
:10B790000E945D72CE0101960E945D7262EE75E0BC
:10B7A000CE0145960E94F2720E94447728EE33E063
:10B7B00040E050E00E946EA369017A0165ED78E0F7
:10B7C000CE014B960E94F27265ED78E088EF9FE023
:10B7D0000E945170CE0101960E94F71D44E150E095
:10B7E000BE016F5F7F4FCE0109960E946E17BE01AA
:10B7F000675F7F4F88EF9FE00E942472CE01099619
:10B800000E945D72CE0101960E945D722AE0B7012E
:10B81000A601CE0109960E94967248E050E0BE0152
:10B82000675F7F4FCE010F960E946E1768EF7FE033
:10B83000CE0101960E94EA72BE01615F7F4FCE0188
:10B8400001960E948471BC018CEE9FE00E940F72F1
:10B85000CE0101960E945D72CE010F960E945D722C
:10B86000CE0109960E945D722AE0B701A601CE01C1
:10B8700009960E94967263E878E0CE0101960E94D4
:10B88000F272BE01675F7F4FCE0101960E94847104
:10B89000BE016B5E7F4F0E948471BC0188EF9FE008
:10B8A0000E94E671CE0101960E945D72CE0109965A
:10B8B0000E945D7240915F0C5091600C6091610C30
:10B8C0007091620C21E0CE0101960E946272BE016D
:10B8D0006F5F7F4FCE014B960E942472CE0101967E
:10B8E0000E945D726AE878E0CE0101960E94F272D1
:10B8F000BE01655E7F4FCE0101960E948471BE013C
:10B900006B5E7F4F0E948471BC0188EF9FE00E94B4
:10B91000E671CE0101960E945D72BE01655E7F4FA9
:10B92000CE0101960E94EA7246E050E0BE016F5FD0
:10B930007F4FCE0109960E946E17BE01675F7F4F51
:10B940008CEE9FE00E94E671CE0109960E945D7226
:10B95000CE0101960E945D7240915B0C50915C0C8F
:10B9600060915D0C70915E0C21E0CE0101960E9409
:10B970006272BE016F5F7F4FCE014B960E942472B0
:10B98000CE0101960E945D7268E978E0CE010196D1
:10B990000E94F272BE01655E7F4FCE0101960E9449
:10B9A0008471BE016B5E7F4F0E948471BC0188EF81
:10B9B0009FE00E94E671CE0101960E945D72BE0179
:10B9C000655E7F4FCE0101960E94EA7246E050E02C
:10B9D000BE016F5F7F4FCE0109960E946E17BE01B8
:10B9E000675F7F4F8CEE9FE00E94E671CE01099663
:10B9F0000E945D72CE0101960E945D7200918302E9
:10BA00001091840267E370E0C8010E9423089093BC
:10BA10001F0C80931E0C892B49F067E370E0C8016E
:10BA20000E94230890931F0C80931E0C80911E0C83
:10BA300090911F0C8C3F9F4F0CF4EDC03DD9298392
:10BA40003A834B835C836D837E838F8398874981A0
:10BA50005A816B817C8121E0CE0109960E9462723D
:10BA6000BE01675F7F4FCE014B960E942472CE01CC
:10BA700009960E945D7262EA78E0CE0109960E9402
:10BA8000F272BE01655E7F4FCE0109960E948471FD
:10BA9000BE016B5E7F4F0E948471BC0188EF9FE006
:10BAA0000E94E671CE0109960E945D72BE01655E3C
:10BAB0007F4FCE0109960E94EA7246E050E0BE0137
:10BAC000675F7F4FCE010F960E946E17BE01615FC8
:10BAD0007F4F8CEE9FE00E94E671CE010F960E9490
:10BAE0005D72CE0109960E945D724D815E816F810B
:10BAF000788521E0CE0109960E946272BE01675FDF
:10BB00007F4FCE014B960E942472CE0109960E946F
:10BB10005D726DEA78E0CE0109960E94F272BE0174
:10BB2000655E7F4FCE0109960E948471BE016B5EF7
:10BB30007F4F0E948471BC0188EF9FE00E94E671F4
:10BB4000CE0109960E945D72BE01655E7F4FCE01F7
:10BB500009960E94EA7246E050E0BE01675F7F4F9F
:10BB6000CE010F960E946E17BE01615F7F4F8CEE73
:10BB70009FE00E94E671CE010F960E945D72CE0199
:10BB800009960E945D7262EF7FE088EF9FE00E945D
:10BB9000E67162EE75E0CE0101960E94F27266EEE9
:10BBA0007FE0CE0101960E948471BC018CEE9FE083
:10BBB0000E94E671CE0101960E945D726CEE7FE0FC
:10BBC000CE0101960E94EA72CE0101960E9494165F
:10BBD000CE0101960E945D726AE070E080E090E024
:10BBE0000E948A76CE014B960E945D72CE014596E8
:10BBF0000E945D72A0960FB6F894DEBF0FBECDBF57
:10BC0000DF91CF911F910F91FF90EF90DF90CF9038
:10BC1000BF90AF90089563EB78E088EF9FE00E94BB
:10BC2000DD7162EC78E08CEE9FE00E94DD7169ECE2
:10BC300078E088EF9FE00E94DD7162EC78E08CEEA6
:10BC40009FE00E94DD719FCFBF92CF92DF92EF9273
:10BC5000FF920F931F93CF93DF93CDB7DEB7C455F9
:10BC6000D1090FB6F894DEBF0FBECDBF6C018B01BA
:10BC700065965FAF4EAF65978091590C90915A0CC5
:10BC8000019690935A0C8093590C8091580C811115
:10BC90003BC0BB24B394B092580C10925A0C109233
:10BCA000590C65ED78E0CE01895B9F4F0E94F272DE
:10BCB00065ED78E0CE01835B9F4F0E94F27250E009
:10BCC00040E06AE074E0C6010E943F1701301105B0
:10BCD00009F0A5C065ED78E088EF9FE00E94517003
:10BCE0006596EEADFFAD65978081811123C054DC70
:10BCF000B092790CCE01835B9F4F0E945D72CE01A2
:10BD0000895B9F4F0E945D720FB6F894DEBF0FBE35
:10BD1000CDBFCC5ADF4F0FB6F894DEBF0FBECDBFFC
:10BD2000DF91CF911F910F91FF90EF90DF90CF9017
:10BD3000BF9008956596EEADFFAD6597808188232D
:10BD400009F467C000E210E09E012F5F3F4F40E220
:10BD500050E0BE016F5D7F4FCE018D5A9F4F0E9414
:10BD6000F26E049739F3BE016F5D7F4FCE018F5B9A
:10BD70009F4F0E94F272BE016F5B7F4FCE01895BC5
:10BD80009F4F0E942472CE018F5B9F4F0E945D7275
:10BD9000BE016F5F7F4FCE018F5B9F4F0E94F2729B
:10BDA000BE016F5B7F4FCE01835B9F4F0E94247269
:10BDB000CE018F5B9F4F0E945D72BE01695B7F4F1A
:10BDC00088EF9FE00E94E67163968EAD9FAD63970A
:10BDD000892B09F4AFCF65EE75E0CE018F5B9F4FE5
:10BDE0000E94F272BE01635B7F4FCE018F5B9F4F5B
:10BDF0000E94847162EE75E00E947071BC0188EF50
:10BE00009FE00E94E671CE018F5B9F4F0E945D72A2
:10BE100091CF68EF7FE084ED9FE00E940F72109257
:10BE2000580C68CF2F923F924F925F926F927F9201
:10BE30008F929F92AF92BF92CF92DF92EF92FF923A
:10BE40000F931F93CF93DF93CDB7DEB7C258D109BD
:10BE50000FB6F894DEBF0FBECDBF6C015B0188EE5C
:10BE6000482E83E0582E612C712C03EE13E09BE5E5
:10BE7000892E912C8C0E9D1E8CE0880E911C1B012E
:10BE80009FEF291A390AD6015996ED90FC90F701D7
:10BE90008581823008F493C082859385A485B58519
:10BEA0008F719927AA27BB27892B8A2B8B2B09F007
:10BEB00086C040E250E0BE016F5F7F4FC7010E9425
:10BEC0005383803209F07BC08981882309F477C0CD
:10BED000853E79F38E3269F38C8583FDEACF229615
:10BEE0001FAE1EAE22978DE693E09FAF8EAF2496D5
:10BEF0001FAE2497BE016F5F7F4FE0E080E04EE20F
:10BF0000DB019D91BD019032A1F0883049F426E714
:10BF100030E02C0F3D1F2E0F311DD9014C93EF5FE8
:10BF200026E730E02C0F3D1F2E0F311DD9019C93C9
:10BF3000EF5F8F5F8B3021F786E790E08C0F9D1FBE
:10BF40008E0F911DFC011082D60159966D917C9146
:10BF500021E0AE014A585F4FCE01CE960E94CF85B8
:10BF6000882369F1BE01625C7F4FCE0181960E94F9
:10BF7000398AAE014A585F4FBE016F5D7F4FCE01D7
:10BF8000855A9F4F0E94A68ACE01855A9F4F0E94D4
:10BF9000898A882309F4ABC0F12CFA141B042CF510
:10BFA00069E0CE0101960E94C272CE0101960E9404
:10BFB000AB16CE0101960E945D72F394EECF6F96A0
:10BFC0001FAE1EAE6F97A3964CAE5DAE6EAE7FAE4B
:10BFD000A3976D961FAF0EAF6D97E6961FAE1EAE80
:10BFE000E697A8961FAEA897CFCFB401CE010196D1
:10BFF0000E94F272CE0101960E94AB16CE0101960C
:10C000000E945D72E696EEADFFADE697309709F4BB
:10C0100046C08581823008F442C060E474E0CE01FD
:10C0200001960E94F272CE0101960E949416CE01F2
:10C0300001960E945D726F968EAD9FAD6F979C8347
:10C040008B83A3968CAD9DADAEADBFADA3978D8315
:10C050009E83AF83B887A7968CAD9DADAEADBFADC7
:10C06000A79789879A87AB87BC871A8309838DE056
:10C07000F401DE011D9601900D928A95E1F7E69696
:10C080008EAD9FADE6979B8F8A8FB101CE01019651
:10C09000C9DECE01855A9F4F0E94958AF4CE63ED8A
:10C0A00078E0CE0101960E94F272CE0101960E94C4
:10C0B000AB16CE0101960E945D72E696EEADFFAD25
:10C0C000E69740E050E0BA01309721F04389548967
:10C0D00065897689CE0101960E948570CE01019610
:10C0E0000E949416CE0101960E945D72D2CFCE5767
:10C0F000DF4F0FB6F894DEBF0FBECDBFDF91CF91FB
:10C100001F910F91FF90EF90DF90CF90BF90AF9075
:10C110009F908F907F906F905F904F903F902F9067
:10C1200008952F923F924F925F926F927F928F92DB
:10C130009F92AF92BF92CF92DF92EF92FF920F93B6
:10C140001F93CF93DF93CDB7DEB7C954D1090FB694
:10C15000F894DEBF0FBECDBF40E052EC61E070E06E
:10C1600086E59DE00E94826E40E855E260E070E066
:10C1700089EB9CE00E94826E61E088E00E94597623
:10C1800061E089E00E94597660E08AE30E94597676
:10C1900061E088E00E94437560E089E00E94437599
:10C1A00061E08AE00E94597661E08BE00E94597656
:10C1B00060E08BE30E94597661E08AE00E9443755B
:10C1C00060E08BE00E9443750E94717584EF91E0FE
:10C1D00090939B0280939A0268EE73E080E090E077
:10C1E0000E948A7686E59DE00E94D86AF82E6AE071
:10C1F000C62ED12CF1100BC086E59DE00E94D86AB6
:10C20000F82E6EE170E080E090E00E948A7621E0F6
:10C21000C21AD10879F780919A0290919B020AE2A2
:10C2200010E15801FC01EA52F0414F01C4018A0DAE
:10C230009B1D0E9449A3F50181935F01F4E5AF16B0
:10C24000F1E1BF0699F76091441170914511072EF5
:10C25000000C880B990B0E9436A29B01AC010E9436
:10C26000CDA4882331F081E090E090934511809334
:10C2700044116091461170914711072E000C880BF4
:10C28000990B0E9436A29B01AC010E94CDA4882389
:10C2900031F082E090E0909347118093461125E7BA
:10C2A000F216B1F0609140117091411180914211EC
:10C2B000909143110E9436A29B01AC010E94CDA433
:10C2C000811106C080912A1090912B108197E8F07F
:10C2D0008DB79EB78A5291400FB6F8949EBF0FBE9D
:10C2E0008DBFADB7BEB711968AE291E0EAE2F0E108
:10C2F00001900D920197E1F70E94D1230FB6F894B7
:10C30000DEBF0FBECDBF55E7F52E2DB73EB72A5283
:10C3100031400FB6F8943EBF0FBE2DBFADB7BEB7CC
:10C3200011968AE291E0EAE2F0E101900D92019724
:10C33000E1F70E947D190FB6F894DEBF0FBECDBFA6
:10C3400095E7F91619F0E3E7FE121BC02DB73EB7CB
:10C350002A5231400FB6F8943EBF0FBE2DBFADB785
:10C36000BEB711968AE291E0EAE2F0E101900D9207
:10C370000197E1F70E94FF280FB6F894DEBF0FBEC9
:10C38000CDBF64E07AE080EE9FE00E94EC716EEE3B
:10C3900079E08AED9FE00E94EC710E94717566ED74
:10C3A00078E086E59DE00E941A74B12CA12C47E24A
:10C3B000E42E992493949092B50CE092B70C1092CD
:10C3C000B60C1092B80C81E00E94256E8111B7C1A5
:10C3D00062EE78E086E59DE00E942C748E2D0E942E
:10C3E000A973E092DC116EEF78E086E59DE00E9493
:10C3F0002C748E2D0E94A9739FEFA91AB90AE39499
:10C40000E0E4EE12D8CF63E379E0AB2811F069E401
:10C4100079E086E59DE00E941A740E947175109281
:10C42000DD118091E111823018F098E09093DD11D8
:10C430009091E211992339F0813029F48091DD1136
:10C4400084608093DD1162E370E080E090E00E9400
:10C450008A766091E31188ED91E10E94F77868EEA9
:10C4600073E080E090E00E948A7660E388ED91E1DD
:10C470000E940B798BE4A82E86E4B82EC5010197A3
:10C48000F1F760E388ED91E10E940B79C501019716
:10C49000F1F760E388ED91E10E940B7983E592E08A
:10C4A0000197F1F760E288ED91E10E940B798091AC
:10C4B000DD1180620E94367984E08093DE118CE089
:10C4C0000E94367981E00E9436799BE3A92E9FE194
:10C4D000B92EC5010197F1F782E08093DF1186E064
:10C4E0000E94367982E00E943679C5010197F1F702
:10C4F00080E40E94367922E9A22E22E0B22E3AE9A7
:10C50000832E32E0932EF50161915F0188ED91E178
:10C510000E9421798A149B04B1F70E94FF070E94B0
:10C52000E30764E670E080E090E00E948A7666EDC2
:10C5300079E0CE0101960E94E272CE0101960E943E
:10C540009416CE0101960E945D7261E085E30E941F
:10C55000597661E085E30E94437561E08AE00E94BC
:10C56000597661E08AE00E94437561E084E00E94B0
:10C57000597661E084E00E94437561E089E30E949E
:10C5800059768091EB0E803308F052C061E089E368
:10C590000E9459768091EB0E282F30E0F901EE0FC2
:10C5A000FF1FE20FF31FE85AF14F9081907C9963CF
:10C5B00090831092EC0E1092ED0E2CE0622F0E94F0
:10C5C000D1A4829FB00111249B012C0D3D1DF901C6
:10C5D000EE0FFF1FE20FF31FE85AF14F908196FD17
:10C5E00019C0FFEFCF1ADF0A2CE0C216D10461F7A1
:10C5F000813009F0B1C01092800082E08093810008
:10C600001092850010928400B19A80916F00826030
:10C6100080936F00E091EB0E8E2F90E0FC01EE0F07
:10C62000FF1FE80FF91FE85AF14F80818064808373
:10C6300068EC70E080E090E00E948A7668EE73E03B
:10C6400080E090E00E948A7665EC79E0CE01019668
:10C650000E94E2724AE050E06FEF7FEFCE01019658
:10C660000E94B517CE0101960E945D7210920C0EC9
:10C6700010920A0E1092070E1092060E84E080931C
:10C68000050E0E9444776B0161E08091050E0E94C7
:10C69000597661E08091050E0E9443750E9437151E
:10C6A00082E58093FF0D1092000E8091FF0D909116
:10C6B000000E0E940B0B6AE0E62E8FEF0E94A90A83
:10C6C000EA94E110FACF81E09EE00E94EF7C20E046
:10C6D00030E0A90160E081E09EE00E942C7DE82E20
:10C6E00080930B0E31E0831709F462C00E944477F7
:10C6F0006C197D09613D774050F381E08093060E0F
:10C7000081E09EE00E94047D67EB79E0CE01019616
:10C710000E94E272CE0101960E949416CE0101960B
:10C720000E945D7266EA79E0CE0101960E94E27293
:10C730006AE070E0CE0101960E94717954C18430A4
:10C7400009F05DCE68E179E086E59DE00E942C74F9
:10C750008E2D0E94A97353CE823061F41092900006
:10C7600080939100109295001092940088BB809362
:10C77000710050CF833069F41092A00082E0809362
:10C78000A1001092A5001092A40089BB80937200B2
:10C7900041CF81113FCF1092200182E0809321018F
:10C7A00010922501109224018ABB8093730032CF2E
:10C7B0002AEA31E040E050E068E081E09EE00E943B
:10C7C0002C7D82FF2AC0E0920C0E80910C0E812CF1
:10C7D000912C5401823029F4812C912CA12C40E41D
:10C7E000B42E20E030E0A90167E381E09EE00E94E2
:10C7F0002C7DA501940169E281E09EE00E942C7DE0
:10C8000080930B0E8823D1F00E9444776C197D0928
:10C81000613D774030F388E071CF54E0E52E0E940F
:10C82000117D80930B0EEA94E110F9CF8A3A11F052
:10C8300082E064CF82E080930C0EC7CF80910C0E13
:10C840008230D1F420E030E0A9016AE381E09EE08B
:10C850000E942C7D882311F086E050CF0E94117D2C
:10C86000807C803C19F483E080930C0E0E94117D43
:10C870000E94117D0E94117D81E09EE00E94047D56
:10C8800080E58093FF0D1092000E81E00E94177FDB
:10C89000882309F463C18091300E811135CF8091D6
:10C8A000240E803109F061C182E08093300E109235
:10C8B000420E1092430E1092440E1092450E80913B
:10C8C000250E9091260EB0E0A0E035E0880F991F6C
:10C8D000AA1FBB1F3A95D1F780933E0E90933F0E4F
:10C8E000A093400EB093410E8DE09EE09093470ED2
:10C8F0008093460E81E080932F0E1092310E10929D
:10C90000320E1092330E1092340E1092350E109299
:10C91000360E1092370E1092380E1092390E109279
:10C920003A0E10923B0E10923C0E10923D0E6AE9A8
:10C9300079E0CE0101960E94E272CE0101960E943A
:10C940009416CE0101960E945D7241E060E474E0AD
:10C95000CE0101960E94DB8ABE016F5F7F4F81EAA4
:10C9600091E10E94C2168091A3119091A4119C8321
:10C970008B838091A5119091A611A091A711B091E0
:10C98000A8118D839E83AF83B8878091A911909160
:10C99000AA11A091AB11B091AC1189879A87AB878E
:10C9A000BC8783EE93E09A8389838DE0EDEAF1E121
:10C9B000DE011D9601900D928A95E1F78091BA11E2
:10C9C0009091BB119B8F8A8F70E060E0CE01019641
:10C9D00029DA64E979E0CE0101960E94E272CE0183
:10C9E00001960E949416CE0101960E945D7268EE37
:10C9F00073E080E090E00E948A7643E160ED72E0AF
:10CA0000CE0101960E94DB8ABE016F5F7F4F8CEBE7
:10CA100091E10E94C2166CE579E08EEC9FE00E94E5
:10CA2000EC7161E579E08EEC9FE00E9495718CEBF2
:10CA300091E10E94898A882309F4B6C068E178E808
:10CA400080ED92E00E946B87811122C060E579E061
:10CA5000CE0101960E94F272CE0101960E94AB16A1
:10CA6000CE0101960E945D7260ED72E0CE010196EA
:10CA70000E94F272CE0101960E949416CE01019698
:10CA80000E945D726EEC7FE08CEB91E10E9441743C
:10CA90008CEB91E10E94958A66E970E080E090E07D
:10CAA0000E948A7662E679E0CE0101960E94F272D7
:10CAB000CE0101960E949416CE0101960E945D72ED
:10CAC0001092750C6EE279E0CE0101960E94E2723E
:10CAD000CE0101960E949416CE0101960E945D72CD
:10CAE0000E941D8E5C0168EE73E080E090E00E9481
:10CAF0008A76D12CC12CAB2809F018C5EAE0CE16F5
:10CB0000D10409F4E4C2B601CE0101960E945A7024
:10CB1000CE0101960E949416CE0101960E945D728C
:10CB200060ED77E080E090E00E948A760E941D8EA2
:10CB30005C0168EE73E080E090E00E948A76CE01AE
:10CB400001960E94B66FBE016F5F7F4F86E59DE044
:10CB50000E940674FFEFCF1ADF0ACDCF80E00E945B
:10CB6000177F882309F4D0CD96CE803209F0CCCD42
:10CB700083E08093300E4091270E5091280E6091F3
:10CB8000290E70912A0E4093420E5093430E6093EB
:10CB9000440E7093450E2EE33EE08DE09EE00E9431
:10CBA0005F818111A1CEB0CD6CE379E0CE01019619
:10CBB0000E94E272CE0101960E94AB16CE01019650
:10CBC0000E945D7260ED72E06FCFF40111821082FD
:10CBD00066E370E1CE0188960E94F272B801645E4D
:10CBE0007F4FCE0182960E94F272B701CE014C9621
:10CBF0000E945A7068E679E0CE0101960E94F272B6
:10CC0000BE01645E7F4FCE0101960E94847166EC86
:10CC100076E00E947071BE016E5D7F4F0E9484714C
:10CC200065EE75E00E947071BE01685D7F4F0E94E5
:10CC30008471BC0129968FAD29972A969FAD2A97BA
:10CC40000E94E671CE0101960E945D72CE014C9663
:10CC50000E945D72CE0182960E945D72CE0188961E
:10CC60000E945D72F5011082118212821382F3011B
:10CC70001082118212821382C7010E946D15FFEF8C
:10CC8000EF1AFF0A81017FC3CE014C960E94F71D67
:10CC90006CE679E0CE0101960E94F272BE01645EFC
:10CCA0007F4FCE0101960E94847162EE75E00E9472
:10CCB0007071BE01605C7F4F0E948471BC0188EF7F
:10CCC0009FE00E940F72CE0101960E945D72CE011C
:10CCD0004C960E945D72CE0101960E94F71D46E1BE
:10CCE00050E0BE016F5F7F4FCE014C960E946E17E1
:10CCF000BE01645E7F4FCE0182960E94EA72BE0141
:10CD0000665C7F4FCE0182960E948471BC01CE0189
:10CD1000CA960E940F72CE0182960E945D72CE0169
:10CD20004C960E945D72CE0101960E945D7268EF82
:10CD30007FE0CE0101960E94EA72CE0101960E9428
:10CD40009416CE0101960E945D7268EF7FE0CE01DD
:10CD500001960E94EA72AE014F5F5F4F62E070E0A1
:10CD600086E792E00E947425182FCE0101960E945A
:10CD70005D72111121C068EF7FE0CE0101960E9423
:10CD8000EA7266ED77E0CE0101960E9470716AED5D
:10CD90007FE00E948471BC01CE014C960E94EA7231
:10CDA000CE014C960E949416CE014C960E945D7264
:10CDB000CE0101960E945D72BE01665C7F4FCE017E
:10CDC00001960E94EA72AE014F5F5F4F63E070E030
:10CDD00089E692E00E947425CE0101960E945D7260
:10CDE000CE01C4960E945D72CE01CA960E945D7209
:10CDF000CE01805C9F4F0E945D7201E010E01093B5
:10CE0000AB020093AA0210936802009367026CE3DE
:10CE100077E089E89FE00E945170109368020093C8
:10CE2000670269E87FE0CE0101960E94EA7262E043
:10CE300070E0CE0101960E94292CCE0101960E943D
:10CE40005D7265EC78E0CE0101960E94E272CE013F
:10CE500001960E949416CE0101960E945D7265EBC8
:10CE600078E0CE0101960E94E272CE0101960E9406
:10CE7000C61DCE0101960E945D7268E976E089E8E0
:10CE80009FE00E94517069E87FE0CE0101960E9408
:10CE9000EA7263E070E0CE0101960E94292CCE0177
:10CEA00001960E945D7282E090E09093AB028093C5
:10CEB000AA0264EA78E0CE0101960E94E272CE01F5
:10CEC00001960E949416CE0101960E945D7268E957
:10CED00078E0CE0101960E94E272CE0101960E9496
:10CEE000C61DCE0101960E945D726CE377E089E871
:10CEF0009FE00E945170809150119091511197FFC5
:10CF000006C060E477E089E89FE00E94517069E81C
:10CF10007FE0CE0101960E94EA7262E070E0CE01ED
:10CF200001960E94292CCE0101960E945D7268E94B
:10CF300076E089E89FE00E94517082E090E0909353
:10CF4000AB028093AA0269E87FE0CE0101960E94BD
:10CF5000EA7263E070E0CE0101960E94292CCE01B6
:10CF600001960E945D7284EF91E090939B02809302
:10CF70009A026AE270E10E94B20764E670E080E023
:10CF800090E00E948A7681E090E09093AB028093DB
:10CF9000AA0283EC97E59093610F8093600F209134
:10CFA000820F822F022E000C990B88309105C8F455
:10CFB000FC01EE0FFF1FEE0FFF1FEE59F04F46E78B
:10CFC00059E0518340832F5F2093820F880F991F70
:10CFD000880F991FFC01EC59F04F81E898E191838B
:10CFE00080832091820F822F022E000C990B8830B3
:10CFF0009105C8F4FC01EE0FFF1FEE0FFF1FEE5965
:10D00000F04F4CE759E0518340832F5F2093820F0C
:10D01000880F991F880F991FFC01EC59F04F84E28B
:10D020009EE59183808382EF9EE00E94B31266E8C2
:10D0300078E0CE0101960E94E272CE0101960E9434
:10D040009416CE0101960E945D720E94C179609390
:10D050004C0C70934D0C80934E0C90934F0C10928F
:10D06000580C0E94891D0E94C17960936F0C7093C7
:10D07000700C8093710C9093720C809129118093A5
:10D08000770C882351F00E94C1796093670C7093EC
:10D09000680C8093690C90936A0CC75BDF4F0FB6E6
:10D0A000F894DEBF0FBECDBFDF91CF911F910F91DE
:10D0B000FF90EF90DF90CF90BF90AF909F908F90B8
:10D0C0007F906F905F904F903F902F90089562E215
:10D0D00079E0CE0101960E94E272CE0101960E9493
:10D0E0009416CE0101960E945D7268EE73E080E0B6
:10D0F00090E00E948A7668E178E885E892E00E94F4
:10D100006B87882331F063E478E885E892E00E9439
:10D110006B8766E970E080E090E00E948A7643E1E8
:10D1200065E872E0CE0101960E94DB8ABE016F5F66
:10D130007F4F8CEB91E10E94C21681E08093750CC9
:10D14000CE01019613D7BE016F5F7F4F8CEB91E14B
:10D150000E9406748CEB91E10E94958A62E370E074
:10D1600080E090E00E948A761092750C0E94EA217D
:10D1700068EE73E080E090E00E948A760E941427B7
:10D1800024E6C22ED12CF1100AC086E59DE010D213
:10D19000F82E64E170E080E090E00E948A7621E061
:10D1A000C21AD10881F765E079E0CE0101960E94AC
:10D1B000E272CE0101960E94C61DCE0101960E9428
:10D1C0005D7232E781E0F31280E00E9420076BEF8E
:10D1D00078E088EF9FE00E94EC71CE0101960E94FA
:10D1E000F71DBE016F5F7F4F88EF9FE00E94E671E1
:10D1F000CE0101960E945D7268EE78E088EF9FE0B4
:10D200000E94957166ED78E0CE0101960E94E2726F
:10D21000CE0101960E94C61DCE0101960E945D724C
:10D2200067E370E080918302909184020E9423085A
:10D2300090931F0C80931E0C68EF7FE0CE01019647
:10D240000E94EA72AE014F5F5F4F62E070E086E7D6
:10D2500092E00E947425F82ECE0101960E945D7224
:10D26000F11021C068EF7FE0CE0101960E94EA72C2
:10D2700066ED77E0CE0101960E9470716AED7FE065
:10D280000E948471BC01CE014C960E94EA72CE01CC
:10D290004C960E949416CE014C960E945D72CE016F
:10D2A00001960E945D7268EF7FE0CE0101960E94B8
:10D2B000EA72AE014F5F5F4F63E070E089E692E093
:10D2C0000E947425F82ECE0101960E945D72F11025
:10D2D00020C068EF7FE0CE0101960E94EA7266ED01
:10D2E00077E0CE010196FCD76AED7FE00E94847161
:10D2F000BC01CE014C960E94EA72CE014C960E946F
:10D300009416CE014C960E945D72CE0101960E9449
:10D310005D7268EE73E080E090E00E948A761E0104
:10D3200080E4280E311C65ED78E0C1010E94F272A4
:10D3300065ED78E0CE01CA960E94F27265ED78E064
:10D34000CE01C4960E94F272E091A802F091A90267
:10D350002896FFAFEEAF2897A2EA8A2EA2E09A2E77
:10D36000BBE5CB2EB2E0DB2E8FE4482E82E0582EB8
:10D3700032015601EE24E394F12C29962FAE299721
:10D380002A963FAE2A97F2E08F0E911C180128E0F2
:10D39000220E311C34E0A30EB11C84E0680E711C17
:10D3A0002896EEADFFAD2897EE15FF050CF00DCCDD
:10D3B00073E4A72E72E0B72EE9E4EE2EE2E0FE2E33
:10D3C00001E010E0F8EE6F2EF3E07F2E812C912C1F
:10D3D00022E0A20EB11C34E0C30ED11C82E0E80EA4
:10D3E000F11C94E0490E511C8091A8029091A90271
:10D3F000801791070CF448CCF50160817181CE0152
:10D40000889658D642E050E0BE01685D7F4FCE015D
:10D410008E960E946E17B801CE014C964BD642E014
:10D4200050E0BE01645E7F4FCE0182960E946E176F
:10D430006EE877E0CE0101960E94F272BE016E5D49
:10D440007F4FCE01019660D7BE01625D7F4F5CD7F2
:10D45000BC01CE01C496E3D7CE0101960E945D7255
:10D46000CE0182960E945D72CE014C960E945D7242
:10D47000CE018E960E945D72CE0188960E945D72EA
:10D48000F6016081718182819381A40193010E94E0
:10D4900090A3BA01A90120E0CE0101960E949672E4
:10D4A00048E050E0BE016F5F7F4FCE014C960E9476
:10D4B0006E17BE01645E7F4FCE01C49687D7CE0142
:10D4C0004C96FBD7CE010196F8D7F70160817181A8
:10D4D000CE010196EFD543E050E0BE016F5F7F4F74
:10D4E000CE014C960E946E17BE01645E7F4FCE0146
:10D4F000C4966CD7CE014C96E0D7CE010196DDD70D
:10D50000BE016C5C7F4FCE01CA9660D7F6011082D7
:10D51000118212821382F20110821182128213820E
:10D52000C8010E946D150F5F1F4F52CF65E179E072
:10D53000D0CD089508950895AF92BF92CF92DF9213
:10D54000EF92FF920F931F93CF93DF936C017B01B8
:10D550008B01040F151FEB015E01AE18BF08C01749
:10D56000D10759F06991D601ED91FC910190F081BC
:10D57000E02DC6011995892B79F7C501DF91CF916F
:10D580001F910F91FF90EF90DF90CF90BF90AF90E1
:10D590000895FC01538D448D252F30E0842F90E0B9
:10D5A000821B930B541710F0CF960895019708959E
:10D5B000FC01918D828D981761F0A28DAE0FBF2F67
:10D5C000B11D5D968C91928D9F5F9F73928F90E0BD
:10D5D00008958FEF9FEF0895FC01918D828D98172C
:10D5E00031F0828DE80FF11D858D90E008958FEF69
:10D5F0009FEF0895FC01918D228D892F90E0805C32
:10D600009F4F821B91098F739927089589EB9CE0A6
:10D61000F1DF21E0892B09F420E0822F089586E5CF
:10D620009DE0E8DF21E0892B09F420E0822F0895B6
:10D63000FC01A48DA80FB92FB11DA35ABF4F2C9187
:10D64000848D90E001968F739927848FA689B7897E
:10D650002C93A089B1898C91837080648C93938D75
:10D66000848D981306C00288F389E02D80818F7D18
:10D6700080830895EF92FF920F931F93CF93DF93D0
:10D68000EC0181E0888F9B8D8C8D98131AC0E889FE
:10D69000F989808185FF15C09FB7F894EE89FF89CD
:10D6A0006083E889F98980818370806480839FBF6B
:10D6B00081E090E0DF91CF911F910F91FF90EF906B
:10D6C0000895F62E0B8D10E00F5F1F4F0F7311277B
:10D6D000E02E8C8D8E110BC00FB607FCFACFE889B7
:10D6E000F989808185FFF5CFCE01A2DFF2CFEB8DE6
:10D6F000EC0FFD2FF11DE35AFF4FF0829FB7F89416
:10D700000B8FEA89FB8980818062D0CFCF93DF9332
:10D71000EC01888D8823B1F0AA89BB89E889F98951
:10D720008C9185FD03C0808186FD0CC00FB607FC7F
:10D73000F7CF8C9185FFF2CF808185FFEDCFCE01B1
:10D7400077DFEACFDF91CF91089580E090E0892BD9
:10D7500021F065DF81110E94000080E090E0892BBC
:10D7600049F080E090E0892B29F00E9400008111AF
:10D770000E94000080E090E0892B49F080E090E07A
:10D78000892B29F00E94000081110E94000080E096
:10D7900090E0892B21F03ADF81110C94000008956C
:10D7A0008150823108F05AC0E82FF0E08827E45217
:10D7B000F4498F4F0C94F0A4FC6B006CEE6BF46B8F
:10D7C000F86B2E6C036C096C0D6C136C176C1B6C76
:10D7D000216C256C2E6C296C2F6C336C8091800031
:10D7E0008F77809380000895809180008F7DF9CF9E
:10D7F00080918000877FF5CF84B58F7784BD0895B1
:10D8000084B58F7DFBCF8091B0008F778093B0007F
:10D8100008958091B0008F7DF9CF809190008F772F
:10D82000809390000895809190008F7DF9CF809132
:10D830009000877FF5CF8091A0008F778093A00024
:10D8400008958091A0008F7DF9CF8091A000877FFF
:10D85000F5CF809120018F778093200108958091EA
:10D8600020018F7DF9CF80912001877FF5CFCF9365
:10D87000DF93282F30E0F901E050F54F8491F90152
:10D88000E654F54FD491F901EC58F54FC491CC23EF
:10D8900099F0811185DFEC2FF0E0EE0FFF1FE65AC3
:10D8A000F54FA591B491EC91ED2381E090E009F45E
:10D8B00080E0DF91CF91089580E090E0FACF3FB70C
:10D8C000F89480911F1390912013A0912113B0918F
:10D8D000221326B5A89B05C02F3F19F00196A11D64
:10D8E000B11D3FBFBA2FA92F982F8827BC01CD01AA
:10D8F000620F711D811D911D42E0660F771F881F09
:10D90000991F4A95D1F7089585ED8093BC008091C9
:10D91000BC0084FDFCCF1092B40C0895209110122D
:10D92000260F3327331F21323105ECF42091B40C3C
:10D93000FC0190E080E0243069F082E00895A0913D
:10D9400010122191AC0140515E4EA40FB52FB11DB4
:10D950002C930196861798F380911012680F6093AC
:10D96000101280E0089581E008950895E091740C0C
:10D970008091730CE81730F4F0E0ED5DF34F808197
:10D9800090E008958FEF9FEF08959091740C80912F
:10D99000730C2FEF3FEF981748F4E92FF0E0ED5D9F
:10D9A000F34F208130E09F5F9093740CC90108957C
:10D9B0008091730C9091740C891B990B0895CF92F0
:10D9C000DF92EF92FF920F931F93CF93DF937C012F
:10D9D000CB018A012091B50C222389F0EB016B0168
:10D9E000C40ED51ECC15DD0561F06991D701ED910E
:10D9F000FC910190F081E02DC7011995F3CF642FC0
:10DA00008DDFC801DF91CF911F910F91FF90EF90B3
:10DA1000DF90CF900895CF93DF931F92CDB7DEB7FD
:10DA200069832091B50C2223F9F02091B80C2032A3
:10DA300058F021E030E0FC013383228390E080E065
:10DA40000F90DF91CF9108958091B60CE82FF0E010
:10DA5000ED56FA4E998190838F5F8093B60C809338
:10DA6000B80C81E090E0ECCF61E0CE01019656DF8A
:10DA7000F8CFDC015996ED91FC913097B9F083898C
:10DA80009489A589B6894285538564857585841BEB
:10DA9000950BA60BB70B811520E89207A105B105E0
:10DAA00038F08FEF9FE7A0E0B0E0089590E080E0CD
:10DAB0000895CF93DF931F92CDB7DEB76983DC0162
:10DAC000ED91FC910280F381E02D41E050E0BE0138
:10DAD0006F5F7F4F19950F90DF91CF9108950E944E
:10DAE00014A70F931F93CF93DF93EC018881998143
:10DAF000009759F02A813B812617370730F081E0E3
:10DB0000DF91CF911F910F9108958B016F5F7F4F30
:10DB10000E9438A6009759F0998388831B830A8353
:10DB20002C813D81232B59F7FC011082E8CF80E046
:10DB3000E7CFEF92FF920F931F93CF93DF9361157F
:10DB4000710541F480E0DF91CF911F910F91FF901B
:10DB5000EF90089541155105A9F07B01EC010C816E
:10DB60001D81040F151FB801BCDF882359F32881DC
:10DB700039818C819D81B701820F931F0E9462A71A
:10DB80001D830C8381E0DFCFCF93DF93EC0188818D
:10DB90009981009711F00E94AFA5198218821D8209
:10DBA0001C821B821A82DF91CF910895EF92FF921F
:10DBB0000F931F93CF93DF93EC017B018A01BA018E
:10DBC00090DF81110AC0CE01DFDFCE01DF91CF915E
:10DBD0001F910F91FF90EF9008951D830C83B70163
:10DBE000888199810E9462A7F0CFCF92DF92EF9255
:10DBF000FF920F931F93CF93DF93EC017A018B0178
:10DC00006C01C40ED51ECC15DD05A9F00E94A70A33
:10DC10008FE00E94A90A8D2F0E94A90A8C2F0E94D2
:10DC2000A90A219680E00E94A90AF80181938F0138
:10DC30000E94A50AE8CFC701DF91CF911F910F91F4
:10DC4000FF90EF90DF90CF900895982F2091B80C1F
:10DC500081E0213208F043C08091B40C8111FCCFE7
:10DC60008091B70C32E03093B40C9093B30C9FEFDB
:10DC70009093B20C1092B10C2093B00CA3E9B5E1D3
:10DC8000E0E9FCE090E0291331C010928F0C9091F4
:10DC90008F0C880F892B80938F0C80918E0C813094
:10DCA00049F510928E0C80918F0C8093BB0080916F
:10DCB000BC0083FDF8CF85EC8093BC008091B40C50
:10DCC0008230E1F38091B20C8F3FB1F08091B20CC1
:10DCD0008032A1F08091B20C803391F084E01092F8
:10DCE000B60C1092B80C1092B50C08953D9131937A
:10DCF0009F5FC9CF85EEE0CF80E0F1CF82E0EFCF2C
:10DD000083E0EDCFCF93DF93EC019A01AB01E8897B
:10DD1000F98982E08083211581EE3807410551059C
:10DD200081F160E079E08DE390E00E946EA32150E4
:10DD30003109410951095695479537952795EC8545
:10DD4000FD851082EE85FF852083188EEC89FD8984
:10DD500086E08083EA89FB89808180618083EA890B
:10DD6000FB89808188608083EA89FB898081806863
:10DD70008083EA89FB8980818F7D8083DF91CF91C9
:10DD80000895E889F989108220E1D9CFCF93C82F6F
:10DD9000462F61E070E00E94B00A61E070E08C2FD5
:10DDA0000E94C90A8111F9CFCF910895FF920F9374
:10DDB0001F93CF93DF93F82E10E000E08F2D0E9489
:10DDC000F20AEC01892B21F08F2D0E94F20A8C01BE
:10DDD000C017D10799F7CE01DF91CF911F910F9115
:10DDE000FF9008954F925F926F927F928F929F92D1
:10DDF000AF92BF92CF92DF92EF92FF920F931F9359
:10DE0000CF93DF9300D0CDB7DEB72C015B014A0181
:10DE10003901FC01C080D18070E060E0C5010E9442
:10DE200047A7A80170E060E0C3010E9447A7F60180
:10DE30008081882309F493C07601FFEFEF1AFF0A6F
:10DE4000F60160816632A9F06CF5662389F06532CF
:10DE500009F447C0F2E08F16910444F0F5016083A5
:10DE6000F1E08F1A9108C50101965C016701E4CFCA
:10DE7000760181E090E0F201F182E0820F900F9054
:10DE80000F90DF91CF911F910F91FF90EF90DF9056
:10DE9000CF90BF90AF909F908F907F906F905F904A
:10DEA0004F9008956B3209F45DC06D3399F681810E
:10DEB0008823F9F26701FFEFCF1ADF0AF7016081CB
:10DEC000653279F144F56623B9F1023011053CF071
:10DED000F301608301501109C30101963C017601F1
:10DEE000E9CF81818983882321F282818A83760127
:10DEF000811104C0F2E0EF0EF11CBBCF83E0E80E0D
:10DF0000F11C1B8240E150E070E060E0CE01019620
:10DF10000E94AE9C9FCF663281F06B32B1F660E218
:10DF2000D4CF818189838823F9F082818A8381110A
:10DF300008C0F2E0EF0EF11C6701760183E090E08B
:10DF40009ACF670183E0C80ED11C1B8240E150E0EC
:10DF500070E060E0CE0101960E94AE9CB6CF84E0F6
:10DF600090E08CCF60E276CF7601E6CFCF93DF935F
:10DF7000EC0181E094E0998388831A821B821C82E1
:10DF80001D8280E590E00E940B0BBE016E5F7F4F0B
:10DF900044E050E08FE090E028DE0E940A0BCE01C2
:10DFA000DF91CF9108950F931F93CF93DF93411586
:10DFB000510541F0FC01048115810115110539F469
:10DFC000FB011082DF91CF911F910F910895415075
:10DFD00051094017510708F48A01EB01FC016081E7
:10DFE0007181A801CE010E9477A7C00FD11F1882AE
:10DFF000E9CFAF92BF92CF92DF92EF92FF920F9351
:10E000001F93CF93DF931F921F92CDB7DEB77A8312
:10E010006983BA01A901E981FA81F770082F10E03C
:10E02000000F111F0A57134FD8018D919C918E0F2D
:10E030009F1F9F01240F351F2130384098F05A014F
:10E040006B0160E078E07B01EE1AFF0AA701B601E0
:10E05000CCDDA5014E195F09B6016E0D7F1DF801DB
:10E06000808191810F900F90DF91CF911F910F913F
:10E07000FF90EF90DF90CF90BF90AF90B6CD20E3B0
:10E08000FC0120833296862F82958F706F706A30E4
:10E0900030F4605D6293682F8111F5CF0895695C5B
:10E0A000F9CFFB0101900020E9F73197AF01461B42
:10E0B000570B7CCD0F931F93CF93DF93CDB7DEB774
:10E0C00062970FB6F894DEBF0FBECDBF8C01CB01B7
:10E0D000F8011182108213821282158214824AE0A2
:10E0E000BE016F5F7F4F0E94EF9DBE016F5F7F4F4C
:10E0F000C801D7DF62960FB6F894DEBF0FBECDBF62
:10E10000DF91CF911F910F9108950F931F93CF939C
:10E11000DF93CDB7DEB7A1970FB6F894DEBF0FBE81
:10E12000CDBF8C01CB01BA01F8011182108213829C
:10E130001282158214822AE0AE014F5F5F4F0E9467
:10E14000269EBE016F5F7F4FC801ABDFA1960FB661
:10E15000F894DEBF0FBECDBFDF91CF911F910F911D
:10E160000895FC0180819181009711F00C94AE9D7F
:10E1700060E070E0CB010895FC01808191810097FF
:10E1800011F00C94B19D60E070E0CB010895AF9266
:10E19000BF92CF92DF92EF92FF920F931F93CF9394
:10E1A000DF93DC01CD90DC901197C114D10439F0DC
:10E1B0001496CD91DC918C017601209761F4DF916A
:10E1C000CF911F910F91FF90EF90DF90CF90BF9074
:10E1D000AF90089575015701BFEFAB1ABB0AF70165
:10E1E0008081082E000C990B0E94D79D892B91F7F6
:10E1F0002197CC0DDD1D8881082E000C990B0E9403
:10E20000D79D892B29F0CE15DF0510F02197F3CF8C
:10E21000AE014F5F5F4F4E195F09D80115965C93B1
:10E220004E931497CE14DF0420F4B701C6010E9468
:10E230002DA7D801ED91FC91119714968D919C9189
:10E24000E80FF91F1082BBCFFC01248135816217D2
:10E25000730748F480819181009729F0860F971FFA
:10E26000FC018081089580E00895FC0124813581BE
:10E27000FB014481558124173507A0F0FC01808102
:10E280009181009779F0FB016081718161157105C1
:10E2900049F0241B350B820F931F0E9459A721E0E0
:10E2A000892B09F020E0822F0895FB0144815581DC
:10E2B000FC01248135812417350778F08081918114
:10E2C000009759F0FB01608171816115710529F09A
:10E2D0000E9469A721E0892B09F020E0822F089590
:10E2E000CF93DF93EC01FB0101900020E9F7319718
:10E2F000AF01461B570B1DDC811102C0CE0144DC6F
:10E30000CE01DF91CF910895CF93DF93EC01FB0114
:10E3100044815581608171810CDC811102C0CE0184
:10E3200033DCCE01DF91CF910895EF92FF920F93EE
:10E330001F93CF93DF93EC017B01CB010E94E69DFD
:10E340000097A1F00C811D81080F191FB801CE01A3
:10E35000C8DB882361F0288139818C819D81B701D8
:10E36000820F931F0E94DF9D1D830C8381E0DF914C
:10E37000CF911F910F91FF90EF900895CF93DF936E
:10E380001F921F92CDB7DEB769831A8241E050E039
:10E39000BE016F5F7F4FCDDB0F900F90DF91CF916C
:10E3A0000895CF93DF93EC01E9DF811102C0CE0124
:10E3B000EBDBCE01DF91CF910895FB0101900020AE
:10E3C000E9F73197AF01461B570BB3CBFB014481F3
:10E3D000558160817181ADCBEF92FF920F931F93B6
:10E3E000CF93DF93EC018B01CB010E94E69D7C0172
:10E3F000BC01CE0176DB81110AC0CE01C5DBCE01A6
:10E40000DF91CF911F910F91FF90EF900895FD82C2
:10E41000EC82B801888199810E94DF9DF0CFCF9373
:10E42000DF93EC01FB018617970741F06081718152
:10E430006115710539F044815581B8DBCE01DF915A
:10E44000CF910895A1DBFACF0F931F93CF93DF9362
:10E450008C01EB01FC01808191810097E1F06881E2
:10E46000798161157105A9F0428153812C813D812B
:10E470004217530770F00E9462A78C819D81F801BA
:10E48000958384831D821C82DF91CF911F910F9110
:10E4900008950E94AFA588819981F80191838083B6
:10E4A0008A819B81938382838C819D8195838483E0
:10E4B000198218821B821A82E5CFFC01808191812A
:10E4C0000C94AFA5EF92FF920F931F93CF93DF931E
:10E4D000CDB7DEB7A1970FB6F894DEBF0FBECDBFA4
:10E4E0007C01CB01BA01F7011182108213821282E2
:10E4F0001582148242E0420F8E010F5F1F4F0E946F
:10E50000F39B009781F0BC01C701CBDDA1960FB64C
:10E51000F894DEBF0FBECDBFDF91CF911F910F9159
:10E52000FF90EF900895C7012FDBF0CF0F931F935B
:10E53000CF93DF93CDB7DEB7A2970FB6F894DEBFC7
:10E540000FBECDBF8C01CB01BA01F8011182108240
:10E55000138212821582148230E0AE014F5F5F4F4A
:10E560000E94F99DBE016F5F7F4FC8019ADDA296A0
:10E570000FB6F894DEBF0FBECDBFDF91CF911F91D4
:10E580000F910895CF93DF931F921F92CDB7DEB7FF
:10E59000FC01118210821382128215821482698317
:10E5A0001A82BE016F5F7F4F7CDD0F900F90DF916D
:10E5B000CF910895FC01118210821382128215827C
:10E5C000148242CFFC0111821082138212821582C2
:10E5D000148202CFFC0111821082138212821582F2
:10E5E00014821DCFFC0111821082138212821582C7
:10E5F00014826115710549F0FB0101900020E9F7D3
:10E600003197AF01461B570BD1CA0895AF92BF9205
:10E61000CF92DF92EF92FF920F931F93CF93DF93EE
:10E620006C015B017A0189012417350720F48F2DD5
:10E630007901042F182F65ED78E0C601D3DFD501ED
:10E640001496CD91DC91EC16FD06D8F40C171D073D
:10E6500008F4E801D501ED91FC911197EC0FFD1F35
:10E66000108110826D917C916E0D7F1DC601611528
:10E67000710599F016DDF50180819181C80FD91FD0
:10E680001883C601DF91CF911F910F91FF90EF90FA
:10E69000DF90CF90BF90AF90089576DAECCFFB017A
:10E6A00001900020E9F73197AF01461B570BDC01C1
:10E6B000ED91FC910280F381E02D19948F929F924D
:10E6C000AF92BF92EF92FF920F931F93CF93DF937E
:10E6D000CDB7DEB7A1970FB6F894DEBF0FBECDBFA2
:10E6E0007C01FA01CB0119A2223008F42AE08E0144
:10E6F0000F5D1F4F822E912CB12CA12CBF01A501C3
:10E7000094010E946EA3F901CA016A3004F5605DAC
:10E71000D8016E938D01232B242B252B79F790E0C4
:10E7200080E0109719F0BD01C701B9DFA1960FB6BF
:10E73000F894DEBF0FBECDBFDF91CF911F910F9137
:10E74000FF90EF90BF90AF909F908F900895695C7D
:10E75000DFCFCF93DF93482F50E070E060E020E1FF
:10E7600086E59DE0ABDFEC0169EE79E086E59DE0B2
:10E7700096DF8C0F9D1FDF91CF9108958F929F920E
:10E78000AF92BF92CF92DF92EF92FF920F931F93BF
:10E79000CF93DF937C01EB016C0182E0C80ED11CAA
:10E7A0004701E5E08E0E911C10E000E0F60141917A
:10E7B0006F0150E070E060E02AE0CE017FDF5C0195
:10E7C000E881F9810190F081E02D6EE2CE0119958A
:10E7D0008A0D9B1D080F191FC814D90439F7F701BA
:10E7E000458150E070E060E02AE0CE0167DF800FF5
:10E7F000911FDF91CF911F910F91FF90EF90DF90CC
:10E80000CF90BF90AF909F908F9008950F931F93DC
:10E81000CF93DF93EC01CB01BE01B0DF8C0169EE39
:10E8200079E0CE013CDF800F911FDF91CF911F91E6
:10E830000F9108950F931F93CF93DF93EC012FDF78
:10E840008C0169EE79E0CE012ADF800F911FDF9104
:10E85000CF911F910F9108956115710509F01FCF98
:10E8600090E080E00895DB0114964D915C9115973E
:10E870006D917C91DC01ED91FC910280F381E02DA2
:10E8800019940F931F93CF93DF93EC01ECDF8C016E
:10E8900069EE79E0CE0103DF800F911FDF91CF9108
:10E8A0001F910F910895EF92FF920F931F93CF93B3
:10E8B000DF938C017B01D0E0C0E0F701EC0FFD1F7E
:10E8C0006491662361F0D801ED91FC910190F08193
:10E8D000E02DC8011995892B11F02196EECFCE01BC
:10E8E000DF91CF911F910F91FF90EF900895DC0180
:10E8F00081E094E08D939D9384E0FB0101900D9263
:10E900008A95E1F708951F920F920FB60F92112486
:10E910000BB60F922F933F934F935F936F937F9319
:10E920008F939F93AF93BF93EF93FF9389EB9CE0FB
:10E930000E94186BFF91EF91BF91AF919F918F91C2
:10E940007F916F915F914F913F912F910F900BBEEF
:10E950000F900FBE0F901F9018951F920F920FB639
:10E960000F9211240BB60F922F938F939F93EF93D7
:10E97000FF93E091C90CF091CA0C8081E091CF0C1B
:10E98000F091D00C82FD1DC090818091D20C8F5FE0
:10E990008F732091D30C821741F0E091D20CF0E0FC
:10E9A000E754F34F958F8093D20CFF91EF919F9195
:10E9B0008F912F910F900BBE0F900FBE0F901F9055
:10E9C00018958081F2CF1F920F920FB60F921124EB
:10E9D0000BB60F922F933F934F935F936F937F9359
:10E9E0008F939F93AF93BF93EF93FF9386E59DE043
:10E9F0000E94186BFF91EF91BF91AF919F918F9102
:10EA00007F916F915F914F913F912F910F900BBE2E
:10EA10000F900FBE0F901F9018951F920F920FB678
:10EA20000F9211240BB60F922F938F939F93EF9316
:10EA3000FF93E091660DF091670D8081E0916C0D80
:10EA4000F0916D0D82FD1DC0908180916F0D8F5FE3
:10EA50008F732091700D821741F0E0916F0DF0E0FF
:10EA6000EA5AF24F958F80936F0DFF91EF919F912E
:10EA70008F912F910F900BBE0F900FBE0F901F9094
:10EA800018958081F2CF1F93CF93DF93282F30E02A
:10EA9000F901E050F54F8491F901E654F54FD49116
:10EAA000F901EC58F54FC491CC23A9F0162F811130
:10EAB0000E94D06BEC2FF0E0EE0FFF1FE05CF54FF3
:10EAC000A591B4918FB7F894EC91111108C0D0952D
:10EAD000DE23DC938FBFDF91CF911F910895DE2B52
:10EAE000F8CF1092740C1092730C1092B60C109216
:10EAF000B80C1092B40C81E08093B30C10928E0C81
:10EB000061E084E1C0DF61E085E1BDDFE9EBF0E0D9
:10EB100080818E7F808380818D7F808388E4809355
:10EB2000B80085E48093BC0089E99AE690932813A5
:10EB3000809327138AE99AE69093261380932513EE
:10EB40000895AF92BF92CF92DF92EF92FF920F9310
:10EB50001F93CF93DF936B017A01EC01CA5EDC4E09
:10EB600028813CE0389F8001399F100D1124A0902E
:10EB7000D115B12C27FF1FC0FB01118210828881A3
:10EB80008F5F888388819801280F311D87FD3A9512
:10EB9000F6012A153B051CF488818C30BCF180817C
:10EBA0009181049680349C4908F471C0F6018081FB
:10EBB000918104966EC088819801280F311D87FDD0
:10EBC0003A952A153B05DCF68881A801480F511DAE
:10EBD00087FD5A95FA01EE0FFF1FE40FF51FE85A63
:10EBE000F14F808186FFCBCF8881F801E80FF11DBE
:10EBF00087FDFA95CF01EE0FFF1FE80FF91FE85AC6
:10EC0000F14F808160E08F733EDFB9CF80819181C9
:10EC10002881A801420F511D27FD5A959A01FA013A
:10EC2000EE0FFF1FE20FF31FE85AF14F21813281EF
:10EC3000820F931FF7019183808388819801280FA9
:10EC4000311D87FD3A95F901EE0FFF1FE20FF31F0B
:10EC5000E85AF14F808186FF21C08881080F111D7D
:10EC600087FD1A95F801EE0FFF1FE00FF11FE85A1C
:10EC7000F14F808161E08F73DF91CF911F910F91F0
:10EC8000FF90EF90DF90CF90BF90AF90FCCE80E4EC
:10EC90009CE9F701918380838FEF8883DF91CF9187
:10ECA0001F910F91FF90EF90DF90CF90BF90AF90AA
:10ECB0000895CF93DF9390E0FC01E654F54F249143
:10ECC0008C58954FFC0184918823D1F090E0880FF7
:10ECD000991FFC01EA5DF54FA591B491FC01E05C40
:10ECE000F54FC591D49161110EC09FB7F8948C91E6
:10ECF000E22FE0958E238C932881E223E8839FBF47
:10ED0000DF91CF9108958FB7F894EC91E22BEC93BB
:10ED10008FBFF6CF8F929F92AF92BF92CF92DF922A
:10ED2000EF92FF926B017C010E945F6C4B015C01D2
:10ED3000C114D104E104F104B9F00E945F6C6819B8
:10ED400079098A099B09683E73408105910580F322
:10ED500021E0C21AD108E108F10888EE880E83E0AC
:10ED6000981EA11CB11CE4CFFF90EF90DF90CF90D4
:10ED7000BF90AF909F908F900895AF92BF92CF9227
:10ED8000DF92EF92FF920F931F93CF93DF93C82FE1
:10ED9000D62F10925C1110925D1110925E1110929C
:10EDA0005F111092601161E084DF60E08C2F6BDEF8
:10EDB0006D2F70E090E080E0ADDF60E08C2F79DFB8
:10EDC0008BE990E00197F1F700E911E08C2F0E94A8
:10EDD000376C892B81F401501109C1F78EEF9FEF39
:10EDE000DF91CF911F910F91FF90EF90DF90CF9027
:10EDF000BF90AF90089500E911E08C2F0E94376C0E
:10EE0000019721F401501109C1F7E8CF18E2D0E8C9
:10EE100000E090E9E92EFF24F3948C2F0E94376CD8
:10EE2000892B29F481E0E81AF108B9F7D7CF0E94BD
:10EE30005F6C6B017C0180E9A82EBB24B3948C2FFE
:10EE40000E94376C019729F481E0A81AB108B9F73C
:10EE5000C5CF0E945F6C6C197D098E099F096932CC
:10EE600071058105910538F0E02FF0E0EC5AFE4E77
:10EE700080858D2B8087D69511F40F5FD0E81150D7
:10EE800041F690E080E0ACCF2FB7F89460911B136F
:10EE900070911C1380911D1390911E132FBF089524
:10EEA000CF92DF92EF92FF92CF93DF938091040F86
:10EEB000843051F4CFEFDFEFCE01DF91CF91FF909F
:10EEC000EF90DF90CF900895E091270FE1113CC0C3
:10EED000DBDF6B017C0128EEC20E23E0D21EE11CB9
:10EEE000F11C88EF9EE00E94AC0D882319F38091FD
:10EEF0005D0F882331F08091280F9091290F892B85
:10EF0000C9F288EF9EE00E948F0CEC01CF3FDC0736
:10EF100071F080915D0F882379F28091280F909194
:10EF2000290F01979093290F8093280FC5CFACDF4D
:10EF3000C616D706E806F906A0F61092270F88EF46
:10EF40009EE00E941C13B8CFE150E093270F0E2ED5
:10EF5000000CFF0BE251F14FC18DD0E0ADCF0F930C
:10EF60001F93CF93DF93EC018C01F80181918F0106
:10EF70008823B9F195DFF8012291022E000C330BA2
:10EF80008217930791F38F3F980791F0A091270F75
:10EF900091E09A0F9093270F0A2E000CBB0BA25101
:10EFA000B14F59968C93903219F48FE18093270FCB
:10EFB0002FE1EC17FD07D9F092919F3FD1F3A0917B
:10EFC000270F81E08A0F8093270F0A2E000CBB0BBE
:10EFD000A251B14F59969C93803259F72093270F35
:10EFE000E8CF81E0DF91CF911F910F91089580E0EC
:10EFF000F9CF1F920F920FB60F9211242F933F93C8
:10F000008F939F93AF93BF9380911B1390911C1389
:10F01000A0911D13B0911E1330911A1323E0230FFA
:10F020002D3758F50196A11DB11D20931A13809319
:10F030001B1390931C13A0931D13B0931E13809168
:10F040001F1390912013A0912113B09122130196C8
:10F05000A11DB11D80931F1390932013A093211322
:10F06000B0932213BF91AF919F918F913F912F91B8
:10F070000F900FBE0F901F90189526E8230F029651
:10F08000A11DB11DD2CF1F920F920FB60F92112466
:10F090000BB60F922F933F934F935F936F937F9392
:10F0A0008F939F93AF93BF93EF93FF9348E251E009
:10F0B00064E271E090E080E044DDFF91EF91BF9168
:10F0C000AF919F918F917F916F915F914F913F9100
:10F0D0002F910F900BBE0F900FBE0F901F901895A1
:10F0E0001F920F920FB60F9211240BB60F922F930F
:10F0F0003F934F935F936F937F938F939F93AF93C0
:10F10000BF93EF93FF9348EA50E064EA70E083E036
:10F1100090E017DDFF91EF91BF91AF919F918F919B
:10F120007F916F915F914F913F912F910F900BBE07
:10F130000F900FBE0F901F9018951F920F920FB651
:10F140000F9211240BB60F922F933F934F935F931F
:10F150006F937F938F939F93AF93BF93EF93FF939F
:10F1600048E950E064E970E082E090E0EADCFF9179
:10F17000EF91BF91AF919F918F917F916F915F912F
:10F180004F913F912F910F900BBE0F900FBE0F909C
:10F190001F9018951F920F920FB60F9211240BB665
:10F1A0000F922F933F934F935F936F937F938F9320
:10F1B0009F93AF93BF93EF93FF9348E850E064E8C9
:10F1C00070E081E090E0BDDCFF91EF91BF91AF91E5
:10F1D0009F918F917F916F915F914F913F912F916F
:10F1E0000F900BBE0F900FBE0F901F901895FC0153
:10F1F000248131E03093B50C2093B70C1092B60CFB
:10F200001092B80C8385682B83EF9DE00E940B6DF4
:10F2100081E00C94256E0F931F93CF938C01C62F22
:10F22000E6DF6C2F6460C801E2DF6C2F6B7FC801E2
:10F23000DEDF83EC90E00197F1F7CF911F910F9102
:10F2400008950F931F93CF938C01C62F607F616049
:10F25000E2DF80E1C89FB00111246160C801DBDFFB
:10F2600081E090E0CF911F910F910895CF93C82F27
:10F27000682F607F88ED91E1CEDF80E1C89FB0010B
:10F28000112488ED91E1CF91C6CFCF93DF9300D0C9
:10F2900000D01F921F92CDB7DEB798E0E9E1F3E00E
:10F2A000DE01119601900D929A95E1F79091E1118E
:10F2B000961708F46FEF70E0660F771F21E030E0DB
:10F2C0002C0F3D1F620F731FFB019081890F806817
:10F2D00028960FB6F894DEBF0FBECDBFDF91CF9159
:10F2E000C5CF0F931F93CF93DF932091DE0222238C
:10F2F000F9F02091DD022223D9F0EB018C0161E0CD
:10F3000080E0C3DFB80188ED91E1ADDA6DE67CE025
:10F3100088ED91E1C8DA61E0F8018481B6DFBE01D1
:10F32000DD0F880B990BDF91CF911F910F91F2CCDC
:10F33000DF91CF911F910F910895609312137093F5
:10F3400013138093141390931513645D7E4F8F4FA6
:10F350009F4F60930E1370930F138093101390932D
:10F36000111382E090E090930D1380930C138CDDC9
:10F37000609308137093091380930A1390930B13EF
:10F380000895CF92DF92EF92FF920F931F937CDD4F
:10F390008B019C01C0900813D0900913E0900A13D0
:10F3A000F0900B136091121370911313809114134A
:10F3B000909115130C191D092E093F09083E1340A1
:10F3C00021053105E0F0DC01CB010196A11DB11D45
:10F3D0008093121390931313A0931413B0931513E7
:10F3E000B701A60148515C4F6F4F7F4F4093081300
:10F3F0005093091360930A1370930B13C8CF1F9196
:10F400000F91FF90EF90DF90CF9008954F925F9211
:10F410006F927F928F929F92AF92BF92CF92DF9224
:10F42000EF92FF920F931F93CF93DF934B015C01F9
:10F430008091041390910513A0910613B0910713C6
:10F4400088159905AA05BB0509F4C6C08CE3C82E2A
:10F45000D12CE12CF12CC501A70196010E946EA3CD
:10F460006093430CCA01B901A70196010E946EA3E3
:10F470006093440CC501B40120E13EE040E050E05F
:10F480000E946EA3CA01B90128E130E040E050E0DB
:10F490000E946EA36093450CC501B40120E831E5DC
:10F4A00041E050E00E946EA369017A01CA01B901EE
:10F4B0006C5F7F4F8F4F9F4F27E030E040E050E080
:10F4C0000E946EA36F5F6093460C412C512C320159
:10F4D00040E004E610E0C0E9D1E0242F30E02E54F3
:10F4E000384FF901E370FF273097F9F4C901B801EB
:10F4F0000E94DDA4892B31F4C901BE010E94DDA464
:10F50000892B99F48EE691E0A0E0B0E0480E591EF8
:10F510006A1E7B1ED301C201AA27BB27C816D906C3
:10F52000EA06FB0638F04F5FD8CF8DE691E0A0E009
:10F53000B0E0ECCF4093490CC90164E670E00E9452
:10F54000DDA4EC01C90160E971E00E94DDA43097FF
:10F5500021F42097D9F40097C9F04DE651E060E01E
:10F5600070E0441A550A660A770AC418D508E608F6
:10F57000F708A3E2B3E020E0213069F43097E9F521
:10F58000209711F40097C9F54DE106C04EE651E011
:10F5900060E070E0E6CF4C9150E070E060E031E078
:10F5A000320FC416D506E606F70640F0C41AD50A8F
:10F5B000E60AF70A1196232F3C30F1F62F5F2093CD
:10F5C000480CC394C092470C809204139092051388
:10F5D000A0920613B0920713DF91CF911F910F9164
:10F5E000FF90EF90DF90CF90BF90AF909F908F9063
:10F5F0007F906F905F904F9008954CE1CDCFC1DE2A
:10F6000005DF8091490C90E08E54984F0895B9DE43
:10F61000FDDE8091480C90E00895B3DEF7DE809126
:10F62000470C90E00895ADDEF1DE8091440C90E04F
:10F630000895A7DEEBDE8091450C90E008951F92BF
:10F640000F920FB60F9211240BB60F922F933F9388
:10F650004F935F936F937F938F939F93AF93BF93DA
:10F66000EF93FF93809134120E94376C20913712F0
:10F67000309138122F5F3F4F30933812209337125A
:10F6800090913612953618F096E09093331290913F
:10F690003312943009F46EC0F8F4923031F19330A3
:10F6A00009F44CC090913512992319F0811171C061
:10F6B0002F9AFF91EF91BF91AF919F918F917F9181
:10F6C0006F915F914F913F912F910F900BBE0F90D3
:10F6D0000FBE0F901F901895953009F457C09630C3
:10F6E00009F791E0909303134FC08111DBCF209174
:10F6F0003712309138122436310528F4109238121E
:10F7000010923712CFCF1092031310923612E0915D
:10F71000361291E09E0F90933612F0E0209137124E
:10F7200030913812EE0FFF1FE75CFD4E31832083CE
:10F73000109238121092371293E019C0813009F0FC
:10F74000B1CFE091361291E09E0F90933612F0E027
:10F750002091371230913812EE0FFF1FE75CFD4EFB
:10F7600031832083109238121092371294E09093D4
:10F77000331298CF882359F22091371230913812E2
:10F780002536310508F48ECF95E0F1CF81118ACF6F
:10F79000B5CF2F988ECF1F920F920FB60F921124D4
:10F7A0000BB60F922F933F934F935F936F937F937B
:10F7B0008F939F93AF93BF93EF93FF938091B90083
:10F7C000887F803609F44DC008F040C0883209F4C3
:10F7D000A9C028F5803109F49DC0C8F4882309F434
:10F7E000FBC0883009F496C0FF91EF91BF91AF91B3
:10F7F0009F918F917F916F915F914F913F912F9149
:10F800000F900BBE0F900FBE0F901F901895883170
:10F8100009F488C0803241F78093B20C14C0803460
:10F8200009F49DC040F48033B9F38833E9F680933E
:10F83000B20C85ECB0C0803509F485C0883509F478
:10F8400096C0883489F60E94846CCECF883909F43A
:10F850008CC038F5883729F050F4883611F080379D
:10F8600019F683E08093B40C1092321257C0883896
:10F8700009F47BC0803919F0803809F0B5CF809148
:10F880003212803208F071C0E091321281E08E0FA6
:10F89000809332128091BB00F0E0EE5EFD4E8083DB
:10F8A0003DC0803B39F0E0F4803A09F479C0883AF1
:10F8B00009F09ACF84E08093B40C10921112109248
:10F8C0001012E0912713F0912813199580911012CE
:10F8D00081110FC081E0809310121092F01109C0C5
:10F8E000803C09F4A6CF883C09F4A3CF883B09F0FB
:10F8F0007BCFE091111281E08E0F80931112F0E026
:10F90000E051FE4E80818093BB0090911112809156
:10F91000101229C080918F0C8093BB0085EC8093DE
:10F92000BC0062CF9091B10C8091B00C981758F543
:10F93000E091B10C81E08E0F8093B10CF0E0E057C4
:10F94000F34F8081E9CFE091B10C81E08E0F80937D
:10F95000B10C8091BB00F0E0E057F34F80839091B1
:10F96000B10C8091B00C9817C8F285E8D8CFE0911F
:10F97000B10C81E08E0F8093B10C8091BB00F0E060
:10F98000E057F34F80838091B30C81115CCF81E00D
:10F9900080938E0C84EA8093BC001092B40C24CF28
:10F9A00085EC8093BC001092B40C809132128032AE
:10F9B00030F4E0913212F0E0EE5EFD4E1082609184
:10F9C000321270E0E0912513F091261382E192E16A
:10F9D00019951092321208CF1092B20C34CFCF93F7
:10F9E000DF93EC018091EA11811109C081E08093DD
:10F9F000EA118091FF0D9091000E0E940B0B60E0C8
:10FA00008C81DF91CF913FC861E0FC0184813BD8BC
:10FA10008091EA11882321F01092EA110C940A0BCC
:10FA200008958FEF0C94A90A0F931F93CF93DF9340
:10FA3000EC012ADA8B01F5DF8F3F61F025DA601BDC
:10FA4000710B6C177D07B8F380E0DF91CF911F91A8
:10FA50000F91089581E0F9CF8F929F92AF92BF925C
:10FA6000FF920F931F93CF93DF93EC01F62E490182
:10FA70005A018E81882379F08F8198859C012F5FB0
:10FA80003F4F38872F838230924010F4CADFF4CF83
:10FA9000CE01BADF1E82CE01A2DF8CE291E0C4DF8C
:10FAA0008F2D80640E94A90A08E110E0D501C401ED
:10FAB000002E04C0B695A795979587950A94D2F71E
:10FAC0000E94A90A08501109083F8FEF180771F723
:10FAD00085E9FF2021F028E087E8F2128FEF0E94ED
:10FAE000A90A10E09EDF8A8787FF04C01F3F11F03C
:10FAF0001F5FF8CFDF91CF911F910F91FF90BF90C3
:10FB0000AF909F908F900895AF92BF92CF92DF9267
:10FB1000EF92FF920F931F93CF93DF93EC01690154
:10FB2000C801820F931F8130924048F58E8188234F
:10FB300079F088819981AA81BB8184179507A607EE
:10FB4000B70731F48F819885C816D90608F03CC0F4
:10FB5000488359836A837B838B85833039F089E0BE
:10FB6000440F551F661F771F8A95D1F79A01AB0185
:10FB700061E1CE0171DF882381F083E08D83CE01C6
:10FB800043DF80E0DF91CF911F910F91FF90EF90C5
:10FB9000DF90CF90BF90AF90089576D95B0141DFA1
:10FBA0008A878F3F59F470D96A197B096D32714089
:10FBB000B0F38FE08D83CE0127DFE1CF8E3F81F45C
:10FBC00018861F8281E08E838F8198858C159D0514
:10FBD00048F427DF8F819885019698878F83F4CF2B
:10FBE0008DE0E8CF6701E00EF11E1BDFF601819387
:10FBF0006F01EE15FF05C9F78F819885080F191F52
:10FC000018870F838985882319F00115124090F019
:10FC10008E81882379F08F8198859C012F5F3F4FDB
:10FC200038872F838230924010F4FBDEF4CFCE0170
:10FC3000EBDE1E8281E0A6CFEF92FF920F931F931F
:10FC4000CF93DF93EC01790182E141155105610504
:10FC5000710591F08B85833039F089E0440F551F91
:10FC6000661F771F8A95D1F79A01AB0168E1CE0133
:10FC7000F3DE882319F084E08D832CC08EEF0E9480
:10FC8000A90A87018EEFF81AF80181918F010E946D
:10FC9000A90A0E151F05C1F78FEF0E94A90A8FEF61
:10FCA0000E94A90ABEDE8A878F71853079F488E5C3
:10FCB00092E0BADE882391F020E030E0A9016DE007
:10FCC000CE01CADE882361F084E1D6CF81E18D8345
:10FCD000CE019ADECE0198DE80E008C085E1CCCF6F
:10FCE000A0DE8111F1CFCE018FDE81E0DF91CF91D7
:10FCF0001F910F91FF90EF900895CF93DF93809124
:10FD0000EB11882399F1C0912913D0912A134091C6
:10FD10009E0250919F026091A0027091A10223E97E
:10FD200033E1CE0189DF811104C080E0DF91CF9102
:10FD300008954091EC115091ED116091EE11709188
:10FD4000EF11411551056105710571F023E933E1AA
:10FD5000CE0172DF882349F31092EC111092ED115D
:10FD60001092EE111092EF111092EB1181E0DECFA4
:10FD70008F929F92AF92BF92EF92FF920F931F9339
:10FD8000CF934B015C01C42F80919E0290919F0202
:10FD9000A091A002B091A10288159905AA05BB0502
:10FDA00039F1ABDF81110BC080E0CF911F910F9132
:10FDB000FF90EF90BF90AF909F908F90089583E950
:10FDC000E82E83E1F82E00E012E030E020E0B501FB
:10FDD000A4018091291390912A1396DE882321F3A0
:10FDE00080929E0290929F02A092A002B092A102E5
:10FDF0004091EB114C2B4093EB1181E0D6CFCF9388
:10FE0000DF93EC016E857F858889998941E0B0DFB9
:10FE1000882351F08A8920E2829FC00111248D56E7
:10FE20009C4EDF91CF91089590E080E0FACF8F92C1
:10FE30009F92AF92BF92CF92DF92EF92FF92CF93B9
:10FE400021E03EE030932A1320932913882309F4FC
:10FE50006BC040E060E070E0CB018ADF81110BC035
:10FE600080E0CF91FF90EF90DF90CF90BF90AF9068
:10FE70009F908F900895809151158F7789F7809189
:10FE80005D1590915E15A0915F15B0916015843657
:10FE90009105A105B10520F3C0905915D0905A15D0
:10FEA000E0905B15F0905C15C114D104E104F104FD
:10FEB000B9F240E0C701B6015BDF882389F2809187
:10FEC0009E1390919F138115924051F6A091A31318
:10FED000AA2331F26091A1137091A21361157105EB
:10FEE00009F4BECF2091A013222309F4B9CFA09327
:10FEF0001F0E2093110E90E080E030E0E1E0F0E092
:10FF0000C82FAF01082E02C0440F551F0A94E2F714
:10FF10002417350769F041E0480F019689309105B3
:10FF200079F740931A0E9CCFC12CD12C7601C1CF0A
:10FF300080931A0E2091A9133091AA1350E040E04B
:10FF40002115310541F42091B7133091B813409138
:10FF5000B9135091BA132093120E3093130E40939D
:10FF6000140E5093150E46015701860E971EA11CC4
:10FF7000B11C8092200E9092210EA092220EB0927F
:10FF8000230EE091A413F091A513F093260EE093B5
:10FF9000250EB0E00E94ACA3DC01CB01880D991DB9
:10FFA000AA1DBB1D8093270E9093280EA093290EA7
:10FFB000B0932A0E25E0EE0FFF1F2A95E1F7E150DE
:10FFC000FE4FEF2FFF27E6958E0F9F1FA11DB11D3E
:10FFD00080931B0E90931C0EA0931D0EB0931E0ECB
:10FFE0008090A6139090A713B12CA12C811491049A
:10FFF00041F48090B3139090B413A090B513B090D7
:020000021000EC
:10000000B613C81AD90AEA0AFB0AC80CD91CEA1C9A
:10001000FB1C04C0F694E794D794C794CA95D2F712
:10002000C092160ED092170EE092180EF092190E92
:1000300085EFC8168FE0D806E104F10428F48CE0BF
:100040008093240E81E00DCF80E125EFC2162FEFC3
:10005000D206E104F104A0F38091BF139091C01384
:10006000A091C113B091C2138093270E9093280ED4
:10007000A093290EB0932A0E80E2E2CF4F925F92B6
:100080006F927F928F929F92AF92BF92CF92DF92A8
:10009000EF92FF920F931F93CF93DF93EC014230C7
:1000A00051056105710590F480E0DF91CF911F91BA
:1000B0000F91FF90EF90DF90CF90BF90AF909F9007
:1000C0008F907F906F905F904F90089589859A856B
:1000D000AB85BC850196A11DB11D84179507A607A8
:1000E000B70710F3CB88DC88ED88FE888F898031D4
:1000F00009F042C0BB27A72F962F852F4801590131
:100100002A013B01C80ED91EEA1EFB1E80919E02E9
:1001100090919F02A091A002B091A102C816D906A9
:10012000EA06FB0699F58F898031B9F5B301A20182
:10013000552766277727440F551F4D565C4EFA0109
:10014000918280828091EB1181608093EB118A898A
:10015000823080F08D819E81AF81B8858C0D9D1D90
:10016000AE1DBF1D8093EC119093ED11A093EE1185
:10017000B093EF1181E099CFDB01CA01E7E0B695BA
:10018000A79597958795EA95D1F7B8CF40E0C70135
:10019000B601EEDD8111C7CF87CFB301A2014F7742
:1001A000552766277727440F551F440F551F4D5677
:1001B0005C4EFA0180829182A282B382C3CF8F9279
:1001C0009F92AF92BF92CF92DF92EF92FF920F93E6
:1001D0001F93CF93DF93FC0181859285A385B4851E
:1001E0000196A11DB11D84179507A607B70770F4E6
:1001F00080E0DF91CF911F910F91FF90EF90DF9002
:10020000CF90BF90AF909F908F90089583889488EF
:10021000A588B6888789803189F5BB27A72F962FB7
:10022000852FE9016A017B018F01BC01CD01680DB9
:10023000791D8A1D9B1D80909E0290909F02A09028
:10024000A002B090A10286169706A806B90601F58D
:10025000F8018789803109F5DD24EE24FF24F601B9
:10026000EE0FFF1FED56FC4E80819181B0E0A0E0C3
:1002700088839983AA83BB8381E0BBCFDB01CA015A
:10028000C7E0B695A79597958795CA95D1F7C9CF39
:1002900040E06EDD8111DCCFABCFE894C7F8DD2400
:1002A000EE24FF24F601EE0FFF1FEE0FFF1FED56A9
:1002B000FC4E80819181A281B381BF70D9CF4F92D2
:1002C0005F926F927F92AF92BF92CF92DF92EF9246
:1002D000FF920F931F93CF93DF9300D01F92CDB760
:1002E000DEB78C0149835A836B837C835901C12C0F
:1002F000D12C7601412C82E0582E612C712C498141
:100300005A816B817C819E012F5F3F4FC80157DF6F
:10031000882339F1F8018585A301920104C0220FD9
:10032000331F441F551F8A95D2F7DA01C901C80E41
:10033000D91EEA1EFB1E49815A816B817C81878907
:10034000803111F188EF9FEFAFEFBFE048175907F9
:100350006A077B07A0F2F501C082D182E282F382B4
:1003600081E00F900F900F900F90DF91CF911F9130
:100370000F91FF90EF90DF90CF90BF90AF907F9064
:100380006F905F904F90089588EF9FEFA0E0B0E0EE
:10039000DDCF8F929F92AF92BF92CF92DF92EF927A
:1003A000FF920F931F93CF93DF93EC018D81811107
:1003B0000EC080E0DF91CF911F910F91FF90EF90E1
:1003C000DF90CF90BF90AF909F908F9008950B8952
:1003D0001C892D893E89041715072607370748F31E
:1003E0004A015B01823031F48A869B86AC86BD86E9
:1003F00081E0E0CF81149104A104B10449F41E828C
:100400001F82188619861A861B861C861D86F0CFC9
:100410000A851B852C853D85EB8DFC8D858590E0BF
:100420000996B901A8014150510961097109082EC5
:1004300004C076956795579547950A94D2F775014C
:100440006401E1E0CE1AD108E108F10804C0F69495
:10045000E794D794C7948A95D2F7C416D506E606D2
:10046000F70620F0012B022B032B09F58F89988DBD
:10047000A98DBA8D8E839F83A887B9878E010A5F65
:100480001F4FC114D104E104F10409F4ADCF4E8132
:100490005F816885798598018B8D9C8D90DE91E0D8
:1004A000C91AD108E108F1088111EBCF82CFC41A33
:1004B000D50AE60AF70AE2CF3F924F925F926F9217
:1004C0007F928F929F92AF92BF92CF92DF92EF92E4
:1004D000FF920F931F93CF93DF93CDB7DEB72C9787
:1004E0000FB6F894DEBF0FBECDBF5C01DC015B969A
:1004F0008D909C905C9716964D905D906D907C9041
:100500001997411451046104710409F467C0BFEFE5
:100510004B1A5B0A6B0A7B0A312CF40181859285A8
:10052000A385B4859C01AD012F5F3F4F4F4F5F4FB7
:1005300029873A874B875C87730162011D821E827F
:100540001F821886F40181859285A385B4852D814B
:100550003E814F815885281739074A075B0708F005
:1005600054C089859A85AB85BC858C159D05AE05E3
:10057000BF0550F482E0C82ED12CE12CF12C92E082
:10058000492E512C612C712C9E012F5F3F4FB701DA
:10059000A601C40114DE8823C1F189819A81AB814F
:1005A000BC81892B8A2B8B2B09F1260137019FEF08
:1005B000491A590A690A790A2D813E814F81588565
:1005C0002F5F3F4F4F4F5F4F2D833E834F835887A1
:1005D0003FEFC31AD30AE30AF30AB4CFF401408011
:1005E0005180628073803324339497CFC414D50430
:1005F000E604F70409F70FEF1FEF2FEF3FE0B70115
:10060000A601C4013BDD811119C080E02C960FB614
:10061000F894DEBF0FBECDBFDF91CF911F910F9138
:10062000FF90EF90DF90CF90BF90AF909F908F9012
:100630007F906F905F904F903F900895F5014681B5
:10064000578160857185411551056105710531F04E
:1006500097018601C40112DD8823B9F2D5011696EF
:10066000CD92DD92ED92FC921997332051F0D70193
:10067000C6010196A11DB11DF40180839183A2835F
:10068000B383F5018789908DA18DB28D892B8A2B3B
:100690008B2B39F4C78AD08EE18EF28E84818068EC
:1006A000848381E0B3CF2F923F924F925F926F92FB
:1006B0007F928F929F92AF92BF92CF92DF92EF92F2
:1006C000FF920F931F93CF93DF93EC015B012A01FD
:1006D0008D81811115C08FEF9FEFDF91CF911F9119
:1006E0000F91FF90EF90DF90CF90BF90AF909F90D1
:1006F0008F907F906F905F904F903F902F900895D4
:100700008C8180FFE8CF0B891C892D893E894A8521
:100710005B856C857D85C201B0E0A0E06801790150
:10072000C41AD50AE60AF70AC816D906EA06FB066D
:1007300018F42801441A550A42011E0126E0220E2F
:10074000311C8114910409F4B0C04A855B856C8525
:100750007D856A0181E0D8228B8D9C8D8A019B0169
:10076000E9E03695279517950795EA95D1F7ED813C
:10077000E230D9F5FC01628D738D848D958D600F0B
:10078000711F821F931F612C22E0722E6C187D084E
:100790008614970408F434012C8126FD04C06114EA
:1007A000F2E07F0671F400919E0210919F02209169
:1007B000A0023091A102061717072807390709F090
:1007C00051C040E0D5DA882309F485CFC6018D56A3
:1007D0009C4ED5019C01260D371DFC012E173F07AD
:1007E00009F45EC041914D93F9CFFC0174807A9475
:1007F0007022C114D10471F471100CC0452B462B2A
:10080000472B39F58F89988DA98DBA8D8E839F835B
:10081000A887B987EB8DFC8D6E817F81888599854E
:100820006250710981099109258504C0660F771FFF
:10083000881F991F2A95D2F7068517852089318947
:10084000600F711F821F931F670D711D811D911D08
:100850009ACF4E815F81688579859101B0DC8111E5
:10086000D9CF39CF750183019601AB01BC018091CD
:10087000291390912A1348D9882309F42CCFA60C68
:10088000B71C8A859B85AC85BD85860D971DA11DEE
:10089000B11D8A879B87AC87BD878618970851CF83
:1008A000281B390BA20EB31EECCFC20116CFCF937B
:1008B000DF931F92CDB7DEB741E050E0BE016F5F1E
:1008C0007F4FF1DE019731F4898190E00F90DF9145
:1008D000CF9108958FEF9FEFF9CFFC01818D928D1D
:1008E000009709F0E4CF8FEF9FEF08950F931F93C8
:1008F000CF93DF93EC01898D9A8D10E000E0009793
:1009000089F0D5DF8C010F3F100761F0898D9A8D3A
:10091000FC01428553856485758541505109610903
:10092000710937DDC801DF91CF911F910F910895B3
:10093000CF93DF93EC018D81882319F18C8187FFA0
:100940001DC0CE015CDAFC01892BD9F08D8182308B
:1009500040F48B899C89AD89BE89848F958FA68F41
:10096000B78F8F89988D938F828F8F89988DA98D5E
:10097000BA8DB58BA48B8C818F778C83DF91CF91CF
:10098000BCC980E0DF91CF9108958F929F92AF9282
:10099000BF92CF92DF92EF92FF920F931F93CF936C
:1009A000DF9300D01F92CDB7DEB7FC018581813087
:1009B00091F080E00F900F900F900F90DF91CF910A
:1009C0001F910F91FF90EF90DF90CF90BF90AF906D
:1009D0009F908F900895848181FFEBCF83899489C4
:1009E000A589B689892B8A2B8B2B09F459C07F01E5
:1009F00040E050E0BA01CF01CCDC8823D1F2F7010E
:100A0000C38CD48C8788908CA18CB28C82E090E0CF
:100A1000A0E0B0E0F60180839183A283B3839E01BE
:100A20002F5F3F4FB501A401C601C9DB882309F43C
:100A3000C0CF00E010E09801B501A401C6011EDBA3
:100A4000882309F4B6CF89809A80AB80BC80F601F8
:100A50008789803101F188EF9FEFAFEFBFE0881603
:100A60009906AA06BB06D8F2F701178A108E118ED6
:100A7000128E138A148A158A168A84818068848368
:100A8000C70156DF882309F494CF40E050E0BA0153
:100A9000C7017FDC8FCF88EF9FEFA0E0B0E0DFCF12
:100AA00081E088CFCF92DF92EF92FF921F93CF9396
:100AB000DF93EC0180E2689FF0011124ED56FC4EBB
:100AC0009385917161F0842F827449F080E0DF9109
:100AD000CF911F91FF90EF90DF90CF900895142F4A
:100AE0006A8B80919E0290919F02A091A002B0918A
:100AF000A1028E879F87A88BB98BC488D588F12CDB
:100B0000E12C7601DD24CC24CF8AD88EE98EFA8EB2
:100B1000828D938DB0E0A0E0AC01BD014C295D2930
:100B20006E297F294F8B588F698F7A8F83858871C3
:100B3000B1F4848D958DA68DB78D8B8B9C8BAD8BF1
:100B4000BE8B81E08D831F701C831E821F821886DE
:100B500019861A861B861C861D8681E0B8CF8031D7
:100B600009F0B4CF9E012D5E3F4F8B8D9C8DA7DB8E
:100B7000882309F4ABCF84E0E5CFCF93DF93EC017A
:100B8000D7DE882311F01D8281E0DF91CF91089597
:100B9000FC01818D928D009709F0CACE08953F9295
:100BA0004F925F926F927F928F929F92AF92BF927D
:100BB000CF92DF92EF92FF920F931F93CF93DF9329
:100BC00000D000D000D01F921F92CDB7DEB77C01BD
:100BD000DC0115968C91811115C0FE013196CE0174
:100BE0000C966F0130E23193E817F907E1F7DA016B
:100BF00030E087E09D91B92E992329F19E3239F496
:100C00008A3011F480E0D6C038E08AE0F3CFE6E124
:100C1000FAE04491442321F031969413FACFF2CFB5
:100C2000831780F34FED490F4E3560F74FE9490FB9
:100C30004A3118F440EEB42EB90EF601E30FF11D5F
:100C4000B0823F5FD7CF89818032E1F2322E8B01B3
:100C5000FB01838D948DD7015C969C938E935B975B
:100C600016821782108611861286138614861586C0
:100C7000F80182859385A485B58543895489658962
:100C8000768984179507A607B70708F04CC025E0BA
:100C9000B695A795979587952A95D1F7F82FFF7068
:100CA000AF2ED80115968C91823008F4ABCFC801D5
:100CB000FEDD97FDA7CFF80182859385A485B585D4
:100CC0004F96A11DB11D82879387A487B587F0E257
:100CD000AF9EB00111246D567C4E6115710509F46B
:100CE00091CFDB018C91882341F0853E09F056C0FD
:100CF000BB2029F0BB24B394BBCFB1100EC0F701C9
:100D0000A28A80919E0290919F02A091A002B09130
:100D1000A10286879787A08BB18BDB018C91811113
:100D2000E9CFBB24B394832D8271823109F06ACF5D
:100D3000BB2009F457C0C70162D8009709F462CFFD
:100D400020E2FC0111922A95E9F72BE0F601DC0183
:100D500001900D922A95E1F721E238E2DC015196EB
:100D60003C932E93509740E058E01F965C934E932F
:100D70001E9753963C932E93529759963C932E93DD
:100D8000589757965C934E9356970E947D7E882382
:100D900009F438CF432DF70162890AC04BE050E0D7
:100DA000C6010E9420A7892B09F062CF432D6A2D2E
:100DB000C70178DE2B960FB6F894DEBF0FBECDBF0D
:100DC000DF91CF911F910F91FF90EF90DF90CF9027
:100DD000BF90AF909F908F907F906F905F904F905B
:100DE0003F900895F8018581823009F40BCFC80146
:100DF00063DB882309F406CFD8015B96ED91FC9163
:100E00005C9716968D909D90AD90BC901997B2E02E
:100E10008B1A9108A108B108858504C0880C991C1B
:100E2000AA1CBB1C8A95D2F786859785A089B189B3
:100E3000880E991EAA1EBB1E848124013501480E0E
:100E4000511C611C711C84149504A604B70401F1A3
:100E5000E1E04E1A5108610871080E947D7E8823E6
:100E600009F4D0CEE3E9F3E1119283E995E18E171D
:100E70009F07D1F740929E0250929F026092A0027B
:100E80007092A1028091EB1181608093EB11DBCF16
:100E9000D8015B96ED91FC91258580E092E0A0E081
:100EA000B0E004C0880F991FAA1FBB1F2A95D2F774
:100EB000F8014389548965897689840F951FA61F97
:100EC000B71F838B948BA58BB68BD70152961C9240
:100ED00083E993E135CF5F926F927F928F929F92D9
:100EE000AF92BF92CF92DF92EF92FF920F931F9338
:100EF000CF93DF93CDB7DEB7C754D1090FB6F894BF
:100F0000DEBF0FBECDBF5C013B0119A218A28DE66A
:100F100093E09F8F8E8F1BA21C821B829A838983F2
:100F20001E8210E000E06E018EE1C80ED11C8BE243
:100F3000E82E8EE0F82EF501E00FF11F80818F3250
:100F400011F40F5F1F4FD501A00FB11FFE01FB96DB
:100F500090E080E04F012D912F3249F0222339F0AB
:100F60000F5F1F4F019621938C309105A1F7880DDB
:100F7000991DFC011082F501E00FF11F80818F3275
:100F800011F40F5F1F4FF501E00FF11F508041E09A
:100F9000511040E030E020E0B401C701F3011995A1
:100FA000811120C0FBE2EF16FEE0FF06C1F480E0F5
:100FB000C95BDF4F0FB6F894DEBF0FBECDBFDF9128
:100FC000CF911F910F91FF90EF90DF90CF90BF9046
:100FD000AF909F908F907F906F905F900895C70122
:100FE000CCDDE5CF552081F021E0A401B701C60199
:100FF000D6DD982E8BE2E8168EE0F80671F0C70178
:10100000BCDD91100FC0D3CF9BE2E9169EE0F9063C
:1010100011F0C701B2DD81E0CBCF992041F2FE0192
:1010200031967F019E2D8F2D7601C92ED82E83CF2C
:101030001F93CF93DF93CDB7DEB76D970FB6F894BC
:10104000DEBF0FBECDBFAB011C821B822DE633E09D
:101050003A8329831E8221E0BC01CE0101969FDDE7
:1010600011E081110CC010E0812F6D960FB6F8943D
:10107000DEBF0FBECDBFDF91CF911F910895CE018E
:1010800001967BDDF1CFCF93DF93CDB7DEB76D97C0
:101090000FB6F894DEBF0FBECDBF442381F1AB0184
:1010A000BC011C821B828DE693E09A8389831E8299
:1010B00022E0CE01019673DD81110EC090E081E047
:1010C000911101C080E06D960FB6F894DEBF0FBE9F
:1010D000CDBFDF91CF910895CE01019656DC8823D4
:1010E00069F3CE0101960E94FF7E009739F325EE49
:1010F000FC0120831E820E947D7E982FE0CF81E03C
:10110000E2CF2F923F924F925F926F927F928F9297
:101110009F92AF92BF92CF92DF92EF92FF920F9386
:101120001F93CF93DF9300D01F92CDB7DEB78C0112
:101130005B011A01DC0115968C911597813009F03D
:10114000C6C014968C9181FFC2C082FDADC0610102
:10115000D8011A964D915D916D917C911D97C114A6
:10116000D10409F427C15B968D919C915C97FC0199
:1011700074802FEF270D2A013B0139E076946794A4
:10118000579447943A95D1F7722E74207A01F1E082
:10119000FF2271101FC0E114F104E1F416964D9185
:1011A0005D916D917C91199741155105610571050E
:1011B00009F096C057968D919D910D90BC91A02DF0
:1011C0000097A105B10509F0ADC0C80175D9882304
:1011D00009F47DC080E092E08E199F0946018C15CC
:1011E0009D0508F44C01D8015B964D915C915C978C
:1011F00016968D919D910D90BC91A02D0297A109FD
:10120000B109FA01258504C0880F991FAA1FBB1FC9
:101210002A95D2F74685578560897189840F951F75
:10122000A61FB71F9C01AD01270D311D411D511D8A
:1012300029013A01811432E0930609F079C08091C6
:101240009E0290919F02A091A002B091A1028415EC
:101250009505A605B70559F48FEF9FEFDC01809344
:101260009E0290939F02A093A002B093A1029501C9
:10127000B301A2018091291390912A130E941C7E30
:10128000882329F19EEFB91AC818D908F801828578
:101290009385A485B585880D991DA11DB11D8287F3
:1012A0009387A487B58754CFF8014389548965890A
:1012B000768982859385A485B585481759076A077D
:1012C0007B0709F444CFC80164D8811140CF81E085
:1012D00090E0D80113969C938E93129780E007C0FC
:1012E0009E012F5F3F4F0E94DF80811102C090E07E
:1012F00077C089819A81AB81BC81F801238D348DBF
:10130000F901278948EF5FEF60E070E0203121F0BC
:1013100048EF5FEF6FEF7FE084179507A607B707E9
:1013200008F053CFF80186839783A087B18752CF07
:10133000E114F10491F5D8011A964D915D916D91EA
:101340007C911D9753968D919D910D90BC91A02DF0
:10135000481759076A077B0700F10E947D7E8823A2
:1013600009F4B5CF40929E0250929F026092A00273
:101370007092A1028091EB1181608093EB11970133
:101380002D563C4ED501C901880D991DF9018E17C6
:101390009F0759F04D914193FACF41E0C301B2014B
:1013A0000E94B87E8111EBCF92CF821B930BA80EC7
:1013B000B91E6ACFF80183899489A589B6898417F3
:1013C0009507A607B70738F48481438B548B658B48
:1013D000768B80688483F801848183FD18C0C10105
:1013E0000F900F900F900F90DF91CF911F910F9161
:1013F000FF90EF90DF90CF90BF90AF909F908F9035
:101400007F906F905F904F903F902F900895C8010C
:101410008FDA882309F45BCFE2CFCF93DF931F925B
:10142000CDB7DEB7698341E050E0BE016F5F7F4F0B
:1014300068DE0F90DF91CF910895CF93DF93EC0199
:10144000E98DFA8D309749F481E090E09B838A839F
:1014500090E080E0DF91CF91089513821282898D10
:101460009A8D4FDEE98DFA8D22813381232B61F72E
:10147000F1CFFC01DB0112968D919C911397938320
:1014800082838DE693E09183808314968C911497E8
:10149000848315968C911597858316964D915D9151
:1014A0006D917C91199746835783608771871A964F
:1014B0004D915D916D917C911D9742875387648713
:1014C00075871E964D915D916D917C9151974687E0
:1014D0005787608B718B52968C915297828B539663
:1014E0004D915D916D917C915697438B548B658B9B
:1014F000768B57964D915D916D917C915A97478B64
:10150000508F618F728F5B968D919C91948F838F9A
:101510000895DC015996ED91FC91309721F081E01E
:101520009581911101C080E00895CF93DF93EC0184
:10153000898D9A8D009739F020DB898D9A8D0E94D4
:10154000AFA51A8E198EDF91CF910895EF92FF9279
:101550000F931F93CF93DF93EC017B018A011B82D2
:101560001A8288EE93E0A0E0B0E08C839D83AE8386
:10157000BF8383EE93E0998388838DE190E00E949E
:1015800013A59A8F898F009779F02DE1F701DC017F
:1015900001900D922A95E1F74CE050E0B801CE01A0
:1015A0000C960E9477A7188EDF91CF911F910F9113
:1015B000FF90EF9008952F923F924F925F926F921B
:1015C0007F928F929F92AF92BF92CF92DF92EF92D3
:1015D000FF920F931F93CF93DF93CDB7DEB7C7561C
:1015E000D1090FB6F894DEBF0FBECDBF5C013B0141
:1015F000A6964FAFA6974E018EE1880E911C6BE226
:101600007EE0C40136DF1C821B828DE693E09A8364
:1016100089831E8263018E010F5F1F4F2401180111
:101620006FE270E0C6010E944EA7009709F454C013
:10163000F60120812F3271F4FFEFCF1ADF0A902FCD
:10164000812F8201492E582E942D852D2801092F96
:10165000182FE6CF8C198D3008F08CE0E82EF12C95
:10166000A701B601CE01885A9F4F0E9477A7E8E5EF
:10167000F0E0EC0FFD1FEE0DFF1D1082C8017DDABA
:1016800021E0AE01485A5F4FB201C80188DA8111EA
:101690001EC01EAE1DAE8DE693E09CAF8BAF2196B3
:1016A0001FAE2197A896EEADFFADA8976E0E7F1ED8
:1016B000F301808181111CC0BE01655C7F4FC101B7
:1016C000D8DE40E454E0B101C50140DF2FC0CE0CAC
:1016D000DF1CC20152DAB8CFC60186199709A89655
:1016E0009FAF8EAFA897B201CE01CB96C2DEDACF04
:1016F00019A218A28DE693E09F8F8E8F1BA22196D0
:101700008FAD219781112DC0F5011382128288EED1
:1017100093E0A0E0B0E084839583A683B78383EE53
:1017200093E091838083128E118E1486C501C9596E
:10173000DF4F0FB6F894DEBF0FBECDBFDF91CF9164
:101740001F910F91FF90EF90DF90CF90BF90AF90DF
:101750009F908F907F906F905F904F903F902F90D1
:1017600008958250A6962FADA697A3018230B8F4B3
:101770006BE27EE0C40113DA882331F2A6968FADC6
:10178000A697867039F049A95AA96BA97CA9C4010A
:101790000E94C981B401C1016CDEA30194CFBE01D6
:1017A000655C7F4FC401FBD9882309F4ADCFCE011E
:1017B000CB96E3D9E3CF0F931F93CF93DF93CDB7AE
:1017C000DEB7AD970FB6F894DEBF0FBECDBF8091E8
:1017D000790C882331F08091FC0F9091FD0F892BBB
:1017E00011F40E94CC5A65ED78E0CE0188960E94F3
:1017F000F2728091780C8823E1F06CE57CE0CE01F8
:1018000001960E94E272CE0101960E94AB16CE01B3
:1018100001960E945D7266EB72E0CE0101960E9415
:10182000F272CE0101960E949416CE0101960E949A
:101830005D728091790C81111BC08091770C8111B0
:101840007BC08091760C882309F442C10FE110E03F
:101850008091750C882309F4BAC00150110909F46C
:101860005CC064E170E080E090E00E948A76F0CF96
:101870008091FC0F9091FD0F892BF9F264E170E0EB
:1018800080E090E00E948A766EE47CE0CE0188964B
:101890000E94EC7168EF7FE0CE0101960E94EA722F
:1018A000AE014F5F5F4F63E070E086EB92E00E9415
:1018B0007425182FCE0101960E945D72111127C068
:1018C000BE01685D7F4FCE014C960E94EA726AEDC0
:1018D0007FE0CE014C960E948471BC01CE0101963E
:1018E0000E94EA72CE0101960E949416CE010196E2
:1018F0000E945D72CE014C960E945D7280919113A0
:101900009091921301969093921380939113109259
:10191000790C8091770C811190CFCE0188960E942E
:101920005D72AD960FB6F894DEBF0FBECDBFDF91EE
:10193000CF911F910F9108958091F00F9091F10F29
:10194000892B09F47ECF60E47CE0CE0188960E946A
:10195000EC716CEE7FE0CE0101960E94EA72AE015E
:101960004F5F5F4F62E070E080ED92E00E9474256F
:10197000182FCE0101960E945D72111162CFBE0137
:10198000685D7F4FCE014C960E94EA726AED7FE05F
:10199000CE014C960E948471BC01CE0101960E943A
:1019A000EA72CE0101960E949416CE0101960E9421
:1019B0005D72CE014C960E945D7280919113909160
:1019C0009213019690939213809391133ACF43E12F
:1019D00063EC72E0CE010196EEDDBE016F5F7F4FDA
:1019E0008CEB91E10E94C21681E08093750C8CEB28
:1019F00091E18FDD8823D9F168EF7FE08CEB91E1F5
:101A00000E9441748CEB91E190DD62E370E080E034
:101A100090E00E948A761092750C8091780C882351
:101A200031F1CE014C960E94F71D64E979E0CE01B8
:101A300082960E94F272BE01645E7F4FCE01829652
:101A40000E948471BC01CE0101960E94EA72CE010F
:101A500001960E949416CE0101960E945D72CE01FD
:101A600082960E945D72CE014C960E945D728CEB54
:101A700091E15BDD62E370E080E090E00E948A76B5
:101A80001092750C43E160ED72E0CE01019693DD9A
:101A9000BE016F5F7F4F8CEB91E10E94C21681E027
:101AA0008093750C8CEB91E134DD882331F06CEE82
:101AB0007FE08CEB91E10E9441748CEB91E135DD8C
:101AC00062E370E080E090E00E948A761092750CEC
:101AD00065ED78E08CEE9FE00E94517065ED78E056
:101AE00088EF9FE00E94517018CFCF92DF92EF9263
:101AF000FF920F931F93CF93DF93EC017A018B0139
:101B00006C01C40ED51ECC15DD05A1F00E94A70AFC
:101B100080EF0E94A90A8D2F0E94A90A8C2F0E9493
:101B2000A90A2196F80181918F010E94A90A0E94B9
:101B3000A50AE9CFC701DF91CF911F910F91FF90C7
:101B4000EF90DF90CF9008958F929F92AF92BF92C7
:101B5000CF92DF92EF92FF921F93CF93DF93182FD4
:101B60007B014A01590164E270E00E94C90AC82E53
:101B700065E270E0812F0E94C90A9C2DE80EF91ED3
:101B800097013770C12ED12CCC0CDD1CC6018258B8
:101B9000934F6C01FC0180819181820F931FA901F9
:101BA0004A0D5B1D4130584050F1C0E0D8E0C21BE7
:101BB000D30BAE01B40199DFA5014C1B5D0BB40141
:101BC0006C0F7D1FF601808191818FDFEA0CFB1C79
:101BD0004F2D64E270E0812F0E94B00A4E2D65E225
:101BE00070E0812FDF91CF911F91FF90EF90DF90F8
:101BF000CF90BF90AF909F908F900C94B00AA501AA
:101C0000B401E3CF1F93CF93DF93D82F192FC62FA3
